:020000040800F2
:1000000000060020E1010008E3010008E301000808
:10001000E3010008E3010008E3010008E301000830
:10002000E3010008E3010008E30100086D2F000868
:10003000E3010008E3010008E3010008E301000810
:10004000E3010008E3010008E3010008E301000800
:10005000E3010008E3010008153200083D32000802
:10006000653200088D320008B5320008E30100084F
:10007000E3010008E3010008E3010008E3010008D0
:10008000E3010008E3010008E3010008E3010008C0
:10009000E3010008E3010008E3010008DD32000885
:1000A000E3010008E3010008E3010008E3010008A0
:1000B000B1330008E3010008E3010008E301000890
:1000C000E3010008E3010008E3010008E301000880
:1000D000E3010008E3010008E3010008E301000870
:1000E00041330008E3010008E3010008E3010008D0
:1000F000E3010008E3010008E3010008E301000850
:10010000E3010008E3010008E3010008E30100083F
:10011000E3010008E3010008E3010008E30100082F
:10012000E3010008E3010008E3010008E30100081F
:10013000E3010008E3010008E3010008E30100080F
:10014000E3010008E3010008E3010008212700089B
:10015000E3010008E3010008E3010008E3010008EF
:10016000E3010008E3010008E3010008E3010008DF
:10017000E3010008E3010008E3010008E3010008CF
:10018000E3010008E3010008E3010008E3010008BF
:10019000E3010008E3010008E3010008E3010008AF
:1001A000E3010008E3010008E3010008E30100089F
:1001B000E3010008E3010008E3010008E30100088F
:1001C000E3010008E3010008E3010008E30100087F
:1001D000E3010008E3010008E3010008E30100086F
:1001E00002E000F000F8FEE772B6374880F30888B6
:1001F000364880F3098836483649086040F20000E6
:10020000CCF200004EF63471CEF200010860BFF36C
:100210004F8FBFF36F8F40F20000C0F2F0004EF638
:100220008851CEF200010860BFF34F8FBFF36F8F8C
:100230004FF00000E1EE100A4EF63C71CEF20001E4
:100240000860062080F31488BFF36F8F01F030FF41
:1002500002F02AFE4FF055301F491B4A91423CBF25
:1002600041F8040BFAE71D49184A91423CBF41F896
:10027000040BFAE71A491B4A1B4B9A423EBF51F83E
:10028000040B42F8040BF8E700201849184A914281
:100290003CBF41F8040BFAE701F00EFF02F058FEF4
:1002A000144C154DAC4203DA54F8041B8847F9E7A7
:1002B00000F042F8114C124DAC4203DA54F8041B22
:1002C0008847F9E701F0F6BE000600200022002072
:1002D0000000000808ED00E00000002000060020FB
:1002E0007837000800220020402200204022002011
:1002F000602E0020E0010008E0010008E001000895
:10030000E00100082DE9F04F2DED108AC1F80CD066
:10031000C3689D46BDEC108ABDE8F08F002383F3CF
:1003200011882846A047002001F074FAFEE701F08A
:1003300003FA00DFFEE7000038B500F0BFFB01F074
:1003400087FE054601F0AAFE0446C8B90E4B9D4241
:1003500018D001339D4218BF044641F2883504BFCE
:1003600001240025002001F07DFE0CB100F074F89E
:1003700000F002FD284600F0C3F800F06DF8F9E740
:100380000025EFE70546EDE7010007B008B500F0EE
:1003900067FBA0F120035842584108BD07B541F260
:1003A0001203022101A8ADF8043000F077FB03B07E
:1003B0005DF804FB38B5302383F3118817480368D0
:1003C0000BB101F0F3FA164A144800234FF47A7186
:1003D00001F0E2FA002383F31188124C236813B171
:1003E0002368013B2360636813B16368013B63606A
:1003F0000D4D2B7833B963687BB9022000F026FCE1
:10040000322363602B78032B07D163682BB902205A
:1004100000F01CFC4FF47A73636038BD402200206A
:10042000B50300086023002058220020084B1870F4
:1004300003280CD8DFE800F008050208022000F0CD
:10044000FDBB022000F0F0BB024B00225A60704757
:100450005822002060230020244B254A10B51C465A
:100460001968013140D004339342F9D16268214BBD
:100470009A4239D9204B9B6803F1006303F580331E
:100480009A4231D2002000F033FB0220FFF7CEFF6A
:100490001A4B1A6C00221A64196E1A66196E596C7E
:1004A0005A64596E5A665A6E5A6942F080025A610D
:1004B0005A6922F080025A615A691A6942F0005260
:1004C0001A611A6922F000521A611B6972B64FF064
:1004D000E0233021C3F8084DD4E9003281F31188BC
:1004E0009D4683F30888104710BD00BF0000010837
:1004F00020000108FFFF0008002200200038024011
:100500002DE9F04F93B0AA4B00902022FF210AA8BA
:100510009D6800F0DBFBA74A1378A3B9A648012128
:1005200003601170302383F3118803680BB101F06D
:100530003DFAA24AA04800234FF47A7101F02CFA48
:10054000002383F31188009B13B19D4B009A1A601E
:100550009C4A009C1378032B1EBF00231370984AFB
:100560004FF0000A18BF5360D3465646D1460120CB
:1005700000F064FB24B1924B1B68002B00F0118249
:10058000002000F06DFA0390039B002BF2DB0120AA
:1005900000F04AFB039B213B162BE8D801A252F83E
:1005A00023F000BF0106000829060008BD06000868
:1005B0006F0500086F0500086F0500084707000871
:1005C000170900083108000893080008BB08000854
:1005D000E10800086F050008F30800086F0500082F
:1005E00065090008A10600086F050008A9090008B0
:1005F0000D060008A10600086F0500089308000812
:100600000220FFF7C3FE002840F0F581009B022185
:10061000BAF1000F08BF1C4605A841F21233ADF82D
:10062000143000F03BFAA2E74FF47A7000F018FAA9
:10063000071EEBDB0220FFF7A9FE0028E6D0013FF2
:10064000052F00F2DA81DFE807F0030A0D101336F8
:1006500005230593042105A800F020FA17E054486B
:100660000421F9E758480421F6E758480421F3E744
:100670004FF01C08404600F03DFA08F104080590D0
:10068000042105A800F00AFAB8F12C0FF2D10120DC
:1006900000FA07F747EA0B0B5FFA8BFB4FF00009F4
:1006A00000F060FB26B10BF00B030B2B08BF0024FE
:1006B000FFF774FE5BE746480421CDE7002EA5D086
:1006C0000BF00B030B2BA1D10220FFF75FFE0746B7
:1006D00000289BD0012000F00BFA0220FFF7A6FEB5
:1006E00000261FFA86F8404600F012FA044690B140
:1006F0000021404600F01CFA01360028F1D1BA462C
:10070000044641F21213022105A8ADF814303E460A
:1007100000F0C4F92BE70120FFF788FE2546244BA3
:100720009B68AB4207D9284600F0E4F9013040F05D
:1007300067810435F3E7234B00251D70204BBA4633
:100740005D603E46ACE7002E3FF460AF0BF00B035C
:100750000B2B7FF45BAF0220FFF768FE322000F026
:100760007FF9B0F10008FFF651AF18F003077FF4EE
:100770004DAF0F4A926808EB050393423FF646AF30
:10078000B8F5807F3FF742AF124B0193B84523DDA8
:100790004FF47A7000F064F90390039A002AFFF690
:1007A00035AF019B039A03F8012B0137EDE700BF3A
:1007B000002200205C23002040220020B503000816
:1007C000602300205822002004220020082200205C
:1007D0000C2200205C220020C820FFF7D7FD07462E
:1007E00000283FF413AF1F2D11D8C5F12002424558
:1007F0000AAB25F0030028BF424683490192184402
:1008000000F03EFA019A8048FF2100F05FFA4FEABB
:10081000A8037D490193C8F38702284600F05EFAD9
:10082000064600283FF46DAF019B05EB830537E7D3
:100830000220FFF7ABFD00283FF4E8AE00F0A4F97A
:1008400000283FF4E3AE0027B846704B9B68BB42DC
:1008500018D91F2F11D80A9B01330ED027F003039C
:1008600012AA134453F8203C05934046042205A9DC
:1008700000F0ACFA04378046E7E7384600F03AF972
:100880000590F2E7CDF81480042105A800F006F9E0
:1008900006E70023642104A8049300F0F5F800287B
:1008A0007FF4B4AE0220FFF771FD00283FF4AEAE36
:1008B000049800F051F90590E6E70023642104A8AC
:1008C000049300F0E1F800287FF4A0AE0220FFF7C7
:1008D0005DFD00283FF49AAE049800F04DF9EAE778
:1008E0000220FFF753FD00283FF490AE00F05CF9C2
:1008F000E1E70220FFF74AFD00283FF487AE05A993
:10090000142000F057F904210746049004A800F0D1
:10091000C5F83946B9E7322000F0A2F8071EFFF605
:1009200075AEBB077FF472AE384A926807EB0903D5
:1009300093423FF66BAE0220FFF728FD00283FF4FC
:1009400065AE27F003074F44B9453FF4A9AE4846CA
:1009500000F0D0F80421059005A800F09FF809F1F7
:100960000409F1E74FF47A70FFF710FD00283FF417
:100970004DAE00F009F9002844D00A9B01330BD09A
:1009800008220AA9002000F0A9F900283AD0202264
:10099000FF210AA800F09AF9FFF700FD1C4800F0BB
:1009A0003FFF13B0BDE8F08F002E3FF42FAE0BF0E9
:1009B0000B030B2B7FF42AAE0023642105A80593BB
:1009C00000F062F8074600287FF420AE0220FFF70F
:1009D000DDFC804600283FF419AEFFF7DFFC41F252
:1009E000883000F01DFF059800F0EEF9464600F053
:1009F000B9F93C46BBE5064652E64FF0000905E66C
:100A0000BA467EE637467CE65C22002000220020C3
:100A1000A086010070B50F4B1B780133DBB2012BB0
:100A20000C4611D80C4D29684FF47A730E6AA2FB5C
:100A30000332014622462846B047844204D1074B80
:100A400000221A70012070BD4FF4FA7000F0E8FE29
:100A50000020F8E710220020082600209423002020
:100A600007B50023024601210DF107008DF807307C
:100A7000FFF7D0FF20B19DF8070003B05DF804FB3D
:100A80004FF0FF30F9E700000A4608B50421FFF7F0
:100A9000C1FF80F00100C0B2404208BD30B4054C37
:100AA0002368DD69044B0A46AC460146204630BC4B
:100AB000604700BF08260020A086010070B501F045
:100AC000CDF9094E094D30800024286833888342CF
:100AD00008D901F0BDF92B6804440133B4F5803F17
:100AE0002B60F2D370BD00BF962300206823002046
:100AF00001F062BA00F1006000F5803000687047D4
:100B000000F10060920000F5803001F0EDB90000C6
:100B1000054B1A68054B1B889B1A834202D9104467
:100B200001F096B90020704768230020962300202A
:100B300038B5084D044629B128682044BDE838403E
:100B400001F0A6B92868204401F08AF90028F3D002
:100B500038BD00BF6823002010F003030AD1B0F5B0
:100B6000047F05D200F10050A0F51040D0F8003805
:100B7000184670470023FBE700F10050A0F5104035
:100B8000D0F8100A70470000064991F8243033B1BC
:100B90000023086A81F824300822FFF7B1BF012042
:100BA000704700BF6C230020014B1868704700BFDE
:100BB000002004E070B5194B1D68194B0138C5F3CE
:100BC0000B0408442D0C04221E88A6420BD15C683D
:100BD0000A46013C824213460FD214F9016F4EB10E
:100BE00002F8016BF6E7013A03F10803ECD1814208
:100BF0000B4602D22C2203F8012B0A4A0524168840
:100C0000AE4204D1984284BF967803F8016B013C50
:100C100002F10402F3D1581A70BD00BF002004E0B5
:100C20009434000880340008022802BF024B4FF4BD
:100C300000129A61704700BF00040240022802BF00
:100C4000014B20229A61704700040240022801BF34
:100C5000024A536983F02003536170470004024045
:100C600070B504464FF47A764CB1412C254628BF26
:100C7000412506FB05F000F0D3FD641BF4E770BDD1
:100C800010B50023934203D0CC5CC4540133F9E780
:100C900010BD000010B5013810F9013F3BB191F9CA
:100CA00000409C4203D11AB10131013AF4E71AB174
:100CB00091F90020981A10BD1046FCE70346024641
:100CC000D01A12F9011B0029FAD1704702440346D9
:100CD000934202D003F8011BFAE770472DE9F8436D
:100CE0001F4D144695F824200746884652BBDFF86E
:100CF00070909CB395F824302BB92022FF214846F0
:100D00002F62FFF7E3FF95F82400C0F10802A2422A
:100D100028BF2246D6B24146920005EB8000FFF77D
:100D2000AFFF95F82430A41B1E44F6B2082E1744DA
:100D30009044E4B285F82460DBD1FFF725FF00285A
:100D4000D7D108E02B6A03EB82038342CFD0FFF7B1
:100D50001BFF0028CBD10020BDE8F8830120FBE772
:100D60006C230020024B1A78024B1A70704700BFA8
:100D7000942300201022002010B5104C104800F0E1
:100D8000B5F821460E4800F0DDF82468626DD2F80F
:100D9000043843F00203C2F804384FF47A70FFF7C6
:100DA0005FFF0849204600F0D3F9626DD2F804389D
:100DB00023F00203C2F8043810BD00BF60350008FC
:100DC00008260020683500087047000030B5094D3E
:100DD0000A4491420DD011F8013B5840082340F3DA
:100DE0000004013B2C4013F0FF0384EA5000F6D1CD
:100DF000EFE730BD2083B8ED02684368114301601E
:100E000003B118477047000013B5446BD4F894340D
:100E10001A681178042915D1217C022912D1197977
:100E2000128901238B4013420CD101A904F14C001B
:100E300001F0F6FED4F89444019B21790246206823
:100E400000F0D0F902B010BD143001F079BE0000FE
:100E50004FF0FF33143001F073BE00004C3001F04E
:100E60004BBF00004FF0FF334C3001F045BF000096
:100E7000143001F047BE00004FF0FF31143001F094
:100E800041BE00004C3001F017BF00004FF0FF32B0
:100E90004C3001F011BF00000020704710B5D0F8B1
:100EA00094341A6811780429044617D1017C022968
:100EB00014D15979528901238B4013420ED1143039
:100EC00001F0DAFD024648B1D4F894444FF480733F
:100ED00061792068BDE8104000F072B910BD0000D3
:100EE000406BFFF7DBBF0000704700007FB5124B7F
:100EF000036000234360C0E90233012502260F4B43
:100F0000057404460290019300F18402294600967C
:100F10004FF48073143001F08BFD094B0294CDE93E
:100F2000006304F523724FF48073294604F14C00EA
:100F300001F052FE04B070BDB4340008E10E0008A8
:100F4000090E00080B68302282F311880A7903EB3E
:100F5000820290614A79093243F822008A7912B1FB
:100F600003EB820398610223C0F8941403740020F9
:100F700080F311887047000038B5037F044613B131
:100F800090F85430ABB9201D01250221FFF734FF42
:100F900004F1140025776FF0010100F069FC84F87A
:100FA000545004F14C006FF00101BDE8384000F0EE
:100FB0005FBC38BD10B5012104460430FFF71CFFAB
:100FC0000023237784F8543010BD000038B5044660
:100FD0000025143001F044FD04F14C00257701F0A8
:100FE00013FE201D84F854500121FFF705FF204611
:100FF000BDE83840FFF752BF90F8443003F060037B
:10100000202B07D190F84520212A4FF0000303D868
:101010001F2A06D800207047222AFBD1C0E90E33D0
:1010200003E0034A82630722C2630364012070471E
:101030001122002037B5D0F894341A6811780429A9
:1010400004461AD1017C022917D11979128901238A
:101050008B40134211D100F14C05284601F094FE5B
:1010600058B101A9284601F0DBFDD4F89444019B56
:1010700021790246206800F0B5F803B030BD0000C9
:10108000F0B500EB810385B09E6904460D46FEB1C4
:10109000302383F3118804EB8507301D0821FFF707
:1010A000ABFEFB685B691B6806F14C001BB101904D
:1010B00001F0C4FD019803A901F0B2FD024648B158
:1010C000039B2946204600F08DF8002383F3118806
:1010D00005B0F0BDFB685A691268002AF5D01B8A7A
:1010E000013B1340F1D104F14402EAE7093138B57C
:1010F00050F82140DCB1302383F31188D4F89424D4
:101100001368527903EB8203DB689B695D6845B124
:1011100004216018FFF770FE294604F1140001F065
:10112000B5FC2046FFF7BAFE002383F3118838BDD3
:101130007047000001F014B8012303700023C0E9D8
:101140000133C36183620362C36243620363704716
:1011500038B50446302383F311880025C0E90355D0
:10116000C0E90555416001F00BF80223237085F3B7
:101170001188284638BD000070B500EB8103054694
:101180005069DA600E46144618B110220021FFF7AC
:101190009DFDA06918B110220021FFF797FD31468F
:1011A0002846BDE8704001F0B5B80000826802F042
:1011B000011282600022C0E90422826101F036B986
:1011C000F0B400EB81044789E4680125A4698D40EF
:1011D0003D43458123600023A2606360F0BC01F0C1
:1011E00051B90000F0B400EB81040789E4680125DF
:1011F00064698D403D43058123600023A2606360E4
:10120000F0BC01F0CBB9000070B502230025044604
:101210000370C0E90255C0E90455C564856180F8D2
:10122000345001F013F863681B6823B12946204647
:10123000BDE87040184770BD0378052B10B5044613
:101240000AD080F850300523037043681B680BB147
:10125000042198470023A36010BD000001780529F0
:1012600006D190F85020436802701B6803B11847FC
:101270007047000070B590F83430044613B1002375
:1012800080F8343004F14402204601F0F1F863683C
:101290009B68B3B994F8443013F0600535D0002151
:1012A000204601F091FB0021204601F083FB63689A
:1012B0001B6813B1062120469847062384F8343072
:1012C00070BD204698470028E4D0B4F84A30E26B5D
:1012D0009A4288BFE36394F94430E56B002B4FF0EA
:1012E000300380F20381002D00F0F280092284F89F
:1012F000342083F311880021D4E90E232046FFF720
:1013000071FF002383F31188DAE794F8452003F096
:101310007F0343EA022340F20232934200F0C58089
:1013200021D8B3F5807F48D00DD8012B3FD0022BB8
:1013300000F09380002BB2D104F14C02A263022290
:10134000E2632364C1E7B3F5817F00F09B80B3F5CE
:10135000407FA4D194F84630012BA0D1B4F84C3092
:1013600043F0020332E0B3F5006F4DD017D8B3F568
:10137000A06F31D0A3F5C063012B90D8636894F8B7
:1013800046205E6894F84710B4F848302046B047CD
:10139000002884D04368A3630368E3631AE0B3F5CD
:1013A000106F36D040F6024293427FF478AF5C4B28
:1013B000A3630223E3630023C3E794F84630012BC1
:1013C0007FF46DAFB4F84C3023F00203C4E90E553E
:1013D000A4F84C30256478E7B4F84430B3F5A06F36
:1013E0000ED194F8463084F84E30204600F086FF47
:1013F00063681B6813B101212046984703232370BB
:101400000023C4E90E339CE704F14F03A3630123D7
:10141000C3E72378042B10D1302383F311882046AF
:10142000FFF7C4FE85F311880321636884F84F50E9
:1014300021701B680BB12046984794F84630002B6A
:10144000DED084F84F300423237063681B68002BC0
:10145000D6D0022120469847D2E794F848301D069E
:1014600003F00F0120460AD500F0F4FF012804D054
:1014700002287FF414AF2B4B9AE72B4B98E700F030
:10148000DBFFF3E794F84630002B7FF408AF94F8C5
:10149000483013F00F01B3D01A06204602D501F0F0
:1014A000A7FAADE701F09AFAAAE794F84630002BC4
:1014B0007FF4F5AE94F8483013F00F01A0D01B066E
:1014C000204602D501F080FA9AE701F073FA97E717
:1014D000142284F8342083F311882B462A462946A7
:1014E0002046FFF76DFE85F31188E9E65DB1152210
:1014F00084F8342083F311880021D4E90E23204698
:10150000FFF75EFEFDE60B2284F8342083F311889A
:101510002B462A4629462046FFF764FEE3E700BF34
:10152000E4340008DC340008E034000838B590F8F2
:1015300034300446002B3ED0063BDAB20F2A34D8B2
:101540000F2B32D8DFE803F0373131082232313146
:101550003131313131313737C56BB0F84A309D42C6
:1015600014D2C3681B8AB5FBF3F203FB12556DB9A5
:10157000302383F311882B462A462946FFF732FE93
:1015800085F311880A2384F834300EE0142384F89C
:101590003430302383F3118800231A46194620463D
:1015A000FFF70EFE002383F3118838BD036C03B1EF
:1015B00098470023E7E70021204601F005FA0021C3
:1015C000204601F0F7F963681B6813B10621204635
:1015D00098470623D7E7000010B590F83430142B55
:1015E000044629D017D8062B05D001D81BB110BD51
:1015F000093B022BFBD80021204601F0E5F9002130
:10160000204601F0D7F963681B6813B10621204614
:101610009847062319E0152BE9D10B2380F83430C5
:10162000302383F3118800231A461946FFF7DAFDA9
:10163000002383F31188DAE7C3689B695B68002B9A
:10164000D5D1036C03B19847002384F83430CEE73A
:1016500000230375826803691B6899689142FBD275
:101660005A68036042601060586070470023037539
:10167000826803691B6899689142FBD85A680360C5
:10168000426010605860704708B50846302383F305
:1016900011880B7D032B05D0042B0DD02BB983F3C0
:1016A000118808BD8B6900221A604FF0FF338361F7
:1016B000FFF7CEFF0023F2E7D1E9003213605A6052
:1016C000F3E70000FFF7C4BF054BD9680875186839
:1016D00002681A60536001220275D860FEF712BEDC
:1016E0009823002030B50C4BDD684B1C87B00446B6
:1016F0000FD02B46094A684600F04EF92046FFF706
:10170000E3FF009B13B1684600F050F9A86907B0E9
:1017100030BDFFF7D9FFF9E79823002089160008AC
:10172000044B1A68DB6890689B68984294BF00205D
:101730000120704798230020084B10B51C68D8681A
:1017400022681A60536001222275DC60FFF78EFF69
:1017500001462046BDE81040FEF7D4BD9823002086
:1017600038B5074C074908480123002523706560F8
:1017700001F042FB0223237085F3118838BD00BFBE
:1017800000260020EC3400089823002000F044B923
:10179000034A516853685B1A9842FBD8704700BFF0
:1017A000001000E08B60022308618B8208467047BE
:1017B0008368A3F1840243F8142C026943F8442C93
:1017C000426943F8402C094A43F8242CC26843F884
:1017D000182C022203F80C2C002203F80B2C044ACC
:1017E00043F8102CA3F12000704700BF1D03000830
:1017F0009823002008B5FFF7DBFFBDE80840FFF79E
:1018000061BF0000024BDB6898610F20FFF75CBFEF
:1018100098230020302383F31188FFF7F3BF0000E3
:1018200008B50146302383F311880820FFF75AFFDB
:10183000002383F3118808BD064BDB6839B1426889
:1018400018605A60136043600420FFF74BBF4FF0ED
:10185000FF307047982300200368984206D01A682A
:101860000260506099611846FFF72CBF7047000076
:1018700038B504460D462068844200D138BD03685F
:1018800023605C608561FFF71DFFF4E710B5036816
:101890009C68A2420CD85C688A600B604C60216036
:1018A000596099688A1A9A604FF0FF33836010BDBF
:1018B0001B68121BECE700000A2938BF0A2170B52B
:1018C00004460D460A26601901F090FA01F07CFAF0
:1018D000041BA54203D8751C2E460446F3E70A2EC6
:1018E00004D9BDE87040012001F0C6BA70BD000007
:1018F000F8B5144B0D46D96103F1100141600A2A75
:101900001969826038BF0A22016048601861A8180E
:10191000144601F05DFA0A2701F056FA431BA34270
:10192000064606D37C1C281901F060FA2746354686
:10193000F2E70A2F04D9BDE8F840012001F09CBA73
:10194000F8BD00BF98230020F8B506460D4601F00B
:101950003BFA0F4A134653F8107F9F4206D12A469E
:1019600001463046BDE8F840FFF7C2BFD169BB6809
:10197000441A2C1928BF2C46A34202D92946FFF746
:101980009BFF224631460348BDE8F840FFF77EBF83
:1019900098230020A823002010B4C0E903230023CB
:1019A0005DF8044B4361FFF7CFBF000010B5194C41
:1019B000236998420DD0D0E90032816813605A60E3
:1019C0009A680A449A60002303604FF0FF33A361D2
:1019D00010BD2346026843F8102F536000220260B6
:1019E00022699A4203D1BDE8104001F0F9B9936829
:1019F00081680B44936001F0E7F92269E16992681C
:101A0000441AA242E4D91144BDE81040091AFFF774
:101A100053BF00BF982300202DE9F047DFF8BC80BA
:101A200008F110072C4ED8F8105001F0CDF9D8F875
:101A30001C40AA68031B9A423ED81444D5E90032E0
:101A40004FF00009C8F81C4013605A60C5F80090B8
:101A5000D8F81030B34201D101F0C2F989F31188EE
:101A6000D5E9033128469847302383F311886B6901
:101A7000002BD8D001F0A8F96A69A0EB04094A4507
:101A800082460DD2022001F0F7F90022D8F810307A
:101A9000B34208D151462846BDE8F047FFF728BFBA
:101AA000121A2244F2E712EB090938BF4A462946C6
:101AB0003846FFF7EBFEB5E7D8F81030B34208D050
:101AC0001444211AC8F81C00A960BDE8F047FFF7CC
:101AD000F3BEBDE8F08700BFA823002098230020B4
:101AE00000207047FEE70000704700004FF0FF3015
:101AF0007047000002290CD0032904D001290748AF
:101B000018BF00207047032A05D8054800EBC20023
:101B10007047044870470020704700BFC435000874
:101B2000202200207835000870B59AB00546084696
:101B300001A9144600F0C2F801A8FFF7BFF8431C42
:101B40005B00C5E900340022237003236370C6B232
:101B500001AB02341046D1B28E4204F1020401D826
:101B60001AB070BD13F8011B04F8021C04F8010C34
:101B70000132F0E708B5302383F311880348FFF7FB
:101B800059FA002383F3118808BD00BF08260020FE
:101B900090F8443003F01F02012A07D190F8452045
:101BA0000B2A03D10023C0E90E3315E003F06003D4
:101BB000202B08D1B0F848302BB990F84520212AC5
:101BC00003D81F2A04D8FFF717BA222AEBD0FAE766
:101BD000034A82630722C26303640120704700BF87
:101BE0001822002007B5052917D8DFE801F01916DB
:101BF00003191920302383F31188104A0190012121
:101C0000FFF7BAFA01980E4A0221FFF7B5FA0D481C
:101C1000FFF7DCF9002383F3118803B05DF804FBC0
:101C2000302383F311880748FFF7A6F9F2E7302342
:101C300083F311880348FFF7BDF9EBE71835000877
:101C40003C3500080826002038B50C4D0C4C0D49D9
:101C50002A4604F10800FFF767FF05F1CA0204F104
:101C600010000949FFF760FF05F5CA7204F118007A
:101C70000649BDE83840FFF757BF00BFD02A002013
:101C800020220020F8340008023500080D35000835
:101C900070B5044608460D46FFF710F8C6B2204658
:101CA000013403780BB9184670BD32462946FEF759
:101CB000F1FF0028F3D10120F6E700002DE9F047FD
:101CC00005460C46FEF7FAFF2A49C6B22846FFF73A
:101CD000DFFF08B10936F6B227492846FFF7D8FFDB
:101CE00008B11036F6B2632E0BD8DFF88880DFF823
:101CF0008890224FDFF890A02E7846B92670BDE874
:101D0000F08729462046BDE8F04701F09BBB252E11
:101D10002CD1072241462846FEF7BCFF60B9184B7C
:101D2000224603F1100153F8040B42F8040B8B42D6
:101D3000F9D107351034DFE7082249462846FEF777
:101D4000A9FF98B90F4BA21C197809090232C95D85
:101D500002F8041C13F8011B01F00F015345C95D83
:101D600002F8031CF0D118340835C5E704F8016BFC
:101D70000135C1E7E43500080D350008FD350008E0
:101D8000EC350008107AFF1F1C7AFF1FBFF34F8F3E
:101D9000024AD368DB03FCD4704700BF003C02401A
:101DA00008B5094B1B7873B9FFF7F0FF074B1A69A9
:101DB000002ABFBF064A5A6002F188325A601A6888
:101DC00022F480621A6008BD2E2D0020003C0240E3
:101DD0002301674508B50B4B1B7893B9FFF7D6FF76
:101DE000094B1A6942F000421A611A6842F48052A3
:101DF0001A601A6822F480521A601A6842F48062EB
:101E00001A6008BD2E2D0020003C02400B28F0B5C2
:101E100016D80C4C0C4923787BB90C4D0E460C237C
:101E20004FF0006255F8047B46F8042B013B13F099
:101E3000FF033A44F6D10123237051F82000F0BD8E
:101E40000020FCE7602D0020302D00201036000817
:101E5000014B53F820007047103600080C207047E3
:101E60000B2810B5044601D9002010BDFFF7CEFFA6
:101E7000064B53F824301844C21A0BB90120F4E77A
:101E800012680132F0D1043BF6E700BF10360008BB
:101E90000B2810B5044621D8FFF778FFFFF780FF25
:101EA0000F4AF323D360C300DBB243F4007343F063
:101EB00002031361136943F480331361FFF766FF74
:101EC000FFF7A4FF074B53F8241000F0D9F8FFF7F1
:101ED00081FF2046BDE81040FFF7C2BF002010BDC3
:101EE000003C024010360008F8B512F00103144619
:101EF00042D18218B2F1016F57D82D4B1B6813F0F5
:101F0000010352D02B4DFFF74BFFF323EB60FFF79C
:101F10003DFF40F20127032C15D824F00104661878
:101F2000244C401A40F20117B142236900EB01052D
:101F300024D123F001032361FFF74CFF0120F8BDFA
:101F4000043C0430E7E78307E7D12B6923F44073AF
:101F50002B612B693B432B6151F8046B0660BFF387
:101F60004F8FFFF713FF03689E42E9D02B6923F0E0
:101F700001032B61FFF72EFF0020E0E723F44073FD
:101F8000236123693B4323610B882B80BFF34F8F71
:101F9000FFF7FCFE2D8831F8023BADB2AB42C3D057
:101FA000236923F001032361E4E71846C7E700BF74
:101FB00000380240003C0240084908B50B7828B1BF
:101FC0001BB9FFF7EDFE01230B7008BD002BFCD001
:101FD000BDE808400870FFF7FDBE00BF2E2D0020B1
:101FE00010B50244064BD2B2904200D110BD441C41
:101FF00000B253F8200041F8040BE0B2F4E700BF50
:10200000502800400F4B30B51C6F240407D41C6FC0
:1020100044F400741C671C6F44F400441C670A4CB1
:10202000236843F4807323600244084BD2B2904289
:1020300000D130BD441C00B251F8045B43F820507D
:10204000E0B2F4E700380240007000405028004041
:1020500007B5012201A90020FFF7C2FF019803B0D4
:102060005DF804FB13B50446FFF7F2FFA04205D06C
:10207000012201A900200194FFF7C4FF02B010BDA6
:1020800070470000034B1A681AB9034AD2F8742843
:102090001A607047642D00200030024008B5FFF739
:1020A000F1FF024B1868C0F3407008BD642D00209A
:1020B00070470000FEE700000A4B0B480B4A9042B5
:1020C0000BD30B4BDA1C121AC11E22F003028B42F7
:1020D00038BF00220021FEF7F9BD53F8041B40F879
:1020E000041BECE7B8370008602E0020602E0020AB
:1020F000602E002070B5D0E915439E6800224FF095
:10210000FF3504EB42135101D3F800090028BEBF8C
:10211000D3F8000940F08040C3F80009D3F8000B61
:102120000028BEBFD3F8000B40F08040C3F8000B7E
:10213000013263189642C3F80859C3F8085BE0D22D
:102140004FF00113C4F81C3870BD0000890141F044
:102150002001016103699B06FCD41220FFF718BB24
:1021600010B5054C2046FEF7E7FF4FF0A04363652E
:10217000024BA36510BD00BF682D00206436000827
:1021800070B50378012B054650D12A4B446D984217
:102190001BD1294B5A6B42F080025A635A6D42F0B0
:1021A00080025A655A6D5A6942F080025A615A6932
:1021B00022F080025A610E2143205B6900F022FC6C
:1021C0001E4BE3601E4BC4F800380023C4F8003EE9
:1021D000C02323606E6D4FF40413A3633369002B97
:1021E000FCDA012333610C20FFF7D2FA3369DB07F5
:1021F000FCD41220FFF7CCFA3369002BFCDA00265E
:10220000A6602846FFF776FF6B68C4F81068DB68A5
:10221000C4F81468C4F81C684BB90A4BA3614FF0AA
:10222000FF336361A36843F00103A36070BD064BF5
:10223000F4E700BF682D0020003802404014004041
:1022400003002002003C30C0083C30C0F8B5446DAB
:10225000054600212046FFF779FFA96D00234FF0C6
:1022600001128F68C4F834384FF00066C4F81C2897
:102270004FF0FF3004EB431201339F42C2F8006974
:10228000C2F8006BC2F80809C2F8080BF2D20B685A
:102290006A6DEB65636210231361166916F0100610
:1022A000FBD11220FFF774FAD4F8003823F4FE6350
:1022B000C4F80038A36943F4402343F01003A3613A
:1022C0000923C4F81038C4F814380A4BEB604FF0F7
:1022D000C043C4F8103B084BC4F8003BC4F8106975
:1022E000C4F80039EB6D03F1100243F48013EA6582
:1022F000A362F8BD4036000840800010426D90F89F
:102300004E10D2F8003823F4FE6343EA0113C2F8FA
:10231000003870472DE9F84300EB8103456DDA681A
:10232000166806F00306731E022B05EB41130C46DC
:1023300080460FFA81F94FEA41104FF00001C3F8CF
:10234000101B4FF0010104F1100398BFB60401FA0D
:1023500003F391698EBF334E06F1805606F50046B1
:1023600000293AD0578A04F15801490137436F5088
:10237000D5F81C180B43C5F81C382B180021C3F8DE
:10238000101953690127611EA7409BB3138A928BD2
:102390009B08012A88BF5343D8F85C20981842EA6A
:1023A000034301F1400205EB8202C8F85C002146BC
:1023B00053602846FFF7CAFE08EB8900C3681B8AF2
:1023C00043EA8453483464011E432E51D5F81C3827
:1023D0001F43C5F81C78BDE8F88305EB4917D7F80B
:1023E000001B21F40041C7F8001BD5F81C1821EA96
:1023F0000303C0E704F13F0305EB83030A4A5A6075
:1024000028462146FFF7A2FE05EB4910D0F8003917
:1024100023F40043C0F80039D5F81C3823EA070735
:10242000D7E700BF0080001000040002826D126830
:10243000C265FFF75FBE00005831436D49015B582C
:1024400013F4004004D013F4001F0CBF022001203D
:10245000704700004831436D49015B5813F4004058
:1024600004D013F4001F0CBF0220012070470000AD
:1024700000EB8101CB68196A0B6813604B685360ED
:102480007047000000EB810330B5DD68AA6913686E
:10249000D36019B9402B84BF402313606B8A146842
:1024A000426D1C44013CB4FBF3F46343033323F05B
:1024B000030302EB411043EAC44343F0C043C0F8B6
:1024C000103B2B6803F00303012B09B20ED1D2F8A5
:1024D000083802EB411013F4807FD0F8003B14BFA2
:1024E00043F0805343F00053C0F8003B02EB41122D
:1024F000D2F8003B43F00443C2F8003B30BD00007B
:102500002DE9F041244D6E6D06EB40130446D3F8DF
:10251000087BC3F8087B38070AD5D6F814381907A2
:1025200006D505EB84032146DB6828465B6898479F
:10253000FA071FD5D6F81438DB071BD505EB840343
:10254000D968CCB98B69488A5A68B2FBF0F600FBAF
:1025500016228AB91868DA6890420DD2121AC3E9B5
:102560000024302383F311880B482146FFF78AFFAC
:1025700084F31188BDE8F081012303FA04F26B892A
:1025800023EA02036B81CB68002BF3D0214602487B
:10259000BDE8F041184700BF682D002000EB810323
:1025A00070B5DD68436D6C692668E6604A0156BB0C
:1025B0001A444FF40020C2F810092A6802F00302FE
:1025C000012A0AB20ED1D3F8080803EB421410F422
:1025D000807FD4F8000914BF40F0805040F00050D4
:1025E000C4F8000903EB4212D2F8000940F004409D
:1025F000C2F80009D3F83408012202FA01F10143BC
:10260000C3F8341870BD19B9402E84BF4020206033
:1026100020682E8A8419013CB4FBF6F440EAC440D9
:1026200040F000501A44C6E72DE9F8433B4D6E6D6B
:1026300006EB40130446D3F80889C3F8088918F05C
:10264000010F4FEA40171AD0D6F81038DB0716D51D
:1026500005EB8003D9684B691868DA68904230D27C
:10266000121A4FF000091A60C3F80490302383F364
:10267000118821462846FFF791FF89F3118818F049
:10268000800F1CD0D6F834380126A640334216D02D
:1026900005EB84036D6DD3F80CC0DCF81420013415
:1026A000E4B2D2F800E005EB04342F4451687145E0
:1026B00015D3D5F8343823EA0606C5F83468BDE8E2
:1026C000F883012303FA04F22B8923EA02032B8106
:1026D0008B68002BD3D0214628469847CFE7BCF81B
:1026E0001000AEEB0103834228BF0346D7F8180958
:1026F00080B2B3EB800FE2D89068A0F1040959F8DA
:10270000048FC4F80080A0EB09089844B8F1040FC6
:10271000F5D818440B4490605360C7E7682D00203B
:102720002DE9F74FA24C656D6E69AB691E4016F43A
:1027300080586E6107D02046FEF766FD03B0BDE805
:10274000F04F00F047BC002E12DAD5F8003E984852
:102750009B071EBFD5F8003E23F00303C5F8003EDB
:10276000D5F8043823F00103C5F80438FEF776FDE8
:10277000370505D58E48FFF7BDFC8D48FEF75CFD9B
:10278000B0040CD5D5F8083813F0060FEB6823F425
:1027900070530CBF43F4105343F4A053EB60310764
:1027A0001BD56368DB681BB9AB6923F00803AB6119
:1027B0002378052B0CD1D5F8003E7D489A071EBF23
:1027C000D5F8003E23F00303C5F8003EFEF746FDB2
:1027D0006368DB680BB176489847F30274D4B7029C
:1027E00027D5D4F85490DFF8C8B100274FF0010A7C
:1027F00009EB4712D2F8003B03F44023B3F5802FD6
:1028000011D1D2F8003B002B0DDA62890AFA07F3E6
:1028100022EA0303638104EB8703DB68DB6813B1FF
:10282000394658469847A36D01379B68FFB29F42CF
:10283000DED9F00617D5676D3A6AC2F30A1002F0C6
:102840000F0302F4F012B2F5802F00F08580B2F58C
:10285000402F08D104EB83030022DB681B6A07F5D5
:10286000805790426AD13003D5F8184813D5E10358
:1028700002D50020FFF744FEA20302D50120FFF796
:102880003FFE630302D50220FFF73AFE270302D57D
:102890000320FFF735FE75037FF550AFE00702D543
:1028A0000020FFF7C1FEA10702D50120FFF7BCFE03
:1028B000620702D50220FFF7B7FE23077FF53EAF80
:1028C0000320FFF7B1FE39E7636DDFF8E4A0019361
:1028D00000274FF00109A36D9B685FFA87FB9B45BA
:1028E0003FF67DAF019B03EB4B13D3F8001901F4C6
:1028F0004021B1F5802F1FD1D3F8001900291BDA30
:10290000D3F8001941F09041C3F80019D3F8001929
:102910000029FBDB5946606DFFF718FC218909FA95
:102920000BF321EA0303238104EB8B03DB689B6831
:1029300013B15946504698470137CCE7910708BF75
:10294000D7F80080072A98BF03F8018B02F1010233
:1029500098BF4FEA182884E7023304EB830207F597
:1029600080575268D2F818C0DCF80820DCE9001C57
:10297000A1EB0C0C002188420AD104EB83046368AC
:102980009B699A6802449A605A6802445A606AE7EE
:1029900011F0030F08BFD7F800808C4588BF02F8FC
:1029A000018B01F1010188BF4FEA1828E3E700BF5E
:1029B000682D0020436D03EB4111D1F8003B43F437
:1029C0000013C1F8003B7047436D03EB4111D1F890
:1029D000003943F40013C1F800397047436D03EB2D
:1029E0004111D1F8003B23F40013C1F8003B7047BC
:1029F000436D03EB4111D1F8003923F40013C1F802
:102A00000039704700F1604303F561430901C9B221
:102A100083F80013012200F01F039A4043099B0032
:102A200003F1604303F56143C3F880211A607047E6
:102A300030B5039C0172043304FB0325C0E906533F
:102A4000049B03630021059BC160C0E90000C0E94D
:102A50000422C0E90842C0E90A11436330BD000006
:102A6000416A0022C0E90411C0E90A22C2606FF085
:102A70000101FEF7FDBE0000D0E90432934201D10E
:102A8000C2680AB9181D70470020704703691960B1
:102A9000C2680132C260C269134482690361934211
:102AA00024BF436A03610021FEF7D6BE38B5044651
:102AB0000D46E3683BB16269131D1268A3621344BB
:102AC000E362002007E0237A33B929462046FEF767
:102AD000B3FE0028EDDA38BD6FF00100FBE700001F
:102AE000C368C269013BC36043691344826943619F
:102AF000934224BF436A436100238362036B03B1A3
:102B00001847704770B53023044683F31188866AEE
:102B10003EB9FFF7CBFF054618B186F3118828466A
:102B200070BDA36AE26A13F8015BA362934202D309
:102B30002046FFF7D5FF002383F31188EFE700005D
:102B40002DE9F84F04460E46174698464FF03009D7
:102B500089F311880025AA46D4F828B0BBF1000FEC
:102B600009D141462046FFF7A1FF20B18BF3118820
:102B70002846BDE8F88FD4E90A12A7EB050B521AD4
:102B8000934528BF9346BBF1400F1BD9334601F153
:102B9000400251F8040B43F8040B9142F9D1A36AA7
:102BA00040334036A3624035D4E90A239A4202D327
:102BB0002046FFF795FF8AF31188BD42D8D289F3EA
:102BC0001188C9E730465A46FEF75AF8A36A5B44B3
:102BD0005E44A3625D44E7E710B5029C01720433D2
:102BE00003FB0421C0E906130023C0E90A33039B59
:102BF0000363049BC460C0E90000C0E90422C0E98B
:102C00000842436310BD0000026AC260426AC0E924
:102C100004220022C0E90A226FF00101FEF728BE5B
:102C2000D0E904239A4201D1C26822B9184650F86B
:102C3000043B0B60704700231846FAE7C368C2697B
:102C40000133C3604369134482694361934224BFE3
:102C5000436A43610021FEF7FFBD000038B504461A
:102C60000D46E3683BB123691A1DA262E269134471
:102C7000E362002007E0237A33B929462046FEF7B5
:102C8000DBFD0028EDDA38BD6FF00100FBE7000046
:102C900003691960C268013AC260C269134482695B
:102CA0000361934224BF436A036100238362036B81
:102CB00003B118477047000070B530230D46044635
:102CC000114683F31188866A2EB9FFF7C7FF10B14A
:102CD00086F3118870BDA36A1D70A36AE26A01338E
:102CE0009342A36204D3E16920460439FFF7D0FF81
:102CF000002080F31188EDE72DE9F84F04460D46DA
:102D0000904699464FF0300A8AF311880026B34660
:102D1000A76A4FB949462046FFF7A0FF20B187F3C5
:102D200011883046BDE8F88FD4E90A073A1AA8EBB3
:102D30000607974228BF1746402F1BD905F14003CD
:102D400055F8042B40F8042B9D42F9D1A36A403377
:102D5000A3624036D4E90A239A4204D3E1692046AB
:102D60000439FFF795FF8BF311884645D9D28AF3D2
:102D70001188CDE729463A46FDF782FFA36A3B4416
:102D80003D44A3623E44E5E7D0E904239A4217D1CB
:102D9000C3689BB1836A8BB1043B9B1A0ED013604E
:102DA000C368013BC360C3691A44836902619A42E4
:102DB00024BF436A036100238362012318467047DE
:102DC0000023FBE700F030B94FF08043586A7047AA
:102DD0004FF08043002258631A610222DA60704784
:102DE0004FF080430022DA60704700004FF08043CC
:102DF00058637047FEE7000070B51B4B0163002568
:102E0000044686B0586085620E4600F0BFF804F1B3
:102E10001003C4E904334FF0FF33C4E90635C4E9B5
:102E20000044A560E562FFF7CFFF2B460246C4E9E8
:102E3000082304F134010D4A256580232046FEF75E
:102E4000B1FC0123E0600A4A0375009272680192A6
:102E5000B268CDE90223074B6846CDE90435FEF799
:102E6000C9FC06B070BD00BF002600207036000807
:102E700075360008F52D0008024AD36A1843D0625F
:102E8000704700BF982300204B6843608B688360C5
:102E9000CB68C3600B6943614B6903628B69436212
:102EA0000B6803607047000008B5264B26481A6976
:102EB00040F2FF110A431A611A6922F4FF7222F0EC
:102EC00001021A611A691A6B0A431A631A6D0A43DE
:102ED0001A651E4A1B6D1146FFF7D6FF02F11C0151
:102EE00000F58060FFF7D0FF02F1380100F5806047
:102EF000FFF7CAFF02F1540100F58060FFF7C4FF3D
:102F000002F1700100F58060FFF7BEFF02F18C0155
:102F100000F58060FFF7B8FF02F1A80100F58060BE
:102F2000FFF7B2FF02F1C40100F58060FFF7ACFFCC
:102F300002F1E00100F58060FFF7A6FFBDE8084060
:102F400000F0EEB800380240000002407C36000875
:102F500008B500F059FAFEF703FCFFF793F8BDE857
:102F60000840FEF771BE000070470000EFF30983D0
:102F700005494A6B22F001024A63683383F30988EA
:102F8000002383F31188704700EF00E0302080F3C6
:102F9000118862B60C4B0D4AD96821F4E06109042E
:102FA000090C0A43DA60D3F8FC20094942F0807228
:102FB000C3F8FC200A6842F001020A602022DA7796
:102FC00083F82200704700BF00ED00E00003FA051F
:102FD000001000E010B5302383F311880E4B5B68BE
:102FE00013F4006314D0F1EE103AEFF30984683C57
:102FF0004FF08073E361094BDB6B236684F3098830
:10300000FEF78EFB10B1064BA36110BD054BFBE72D
:1030100083F31188F9E700BF00ED00E000EF00E066
:103020002F030008320300080F4B1A6C42F0010214
:103030001A641A6E42F001021A660C4A1B6E9368FB
:1030400043F0010393604FF0804353229A624FF0A4
:10305000FF32DA6200229A615A63DA605A60012212
:103060005A611A60704700BF00380240002004E037
:103070004FF0804208B51169D3680B40D9B2C943FB
:103080009B07116107D5302383F31188FEF77EFB80
:10309000002383F3118808BD1F4B1A696FEAC252DF
:1030A0006FEAD2521A611A69C2F308021A614FF02C
:1030B000FF301A695A69586100215A6959615A6981
:1030C0001A6A62F080521A621A6A02F080521A6218
:1030D0001A6A5A6A58625A6A59625A6A1A6C42F0F3
:1030E00080521A641A6E42F080521A661A6E0B4AA7
:1030F000106840F480701060186F00F44070B0F5F4
:10310000007F1EBF4FF4803018671967536823F49F
:103110000073536000F054B9003802400070004062
:10312000334B4FF080521A64324A4FF440411160E1
:103130001A6842F001021A601A689107FCD59A6871
:1031400022F003029A602A4B9A6812F00C02FBD11B
:10315000196801F0F90119609A601A6842F4803226
:103160001A601A689203FCD55A6F42F001025A673E
:103170001F4B5A6F9007FCD51F4A5A601A6842F0DD
:1031800080721A601B4A53685904FCD5184B1A68A0
:103190009201FCD5194A9A60194B1A68194B9A4248
:1031A000194B21D1194A1168194A91421CD140F298
:1031B00005121A60144A136803F00F03052BFAD1A5
:1031C0000B4B9A6842F002029A609A6802F00C0275
:1031D000082AFAD15A6C42F480425A645A6E42F478
:1031E00080425A665B6E704740F20572E1E700BFAD
:1031F00000380240007000400854400700948838AE
:10320000002004E011640020003C024000ED00E0DA
:1032100041C20F41074A08B5536903F001035361E6
:1032200023B1054A13680BB150689847BDE80840C0
:10323000FFF7D0BE003C0140E02D0020074A08B552
:10324000536903F00203536123B1054A93680BB13C
:10325000D0689847BDE80840FFF7BCBE003C01407D
:10326000E02D0020074A08B5536903F004035361B9
:1032700023B1054A13690BB150699847BDE808406E
:10328000FFF7A8BE003C0140E02D0020074A08B52A
:10329000536903F00803536123B1054A93690BB1E5
:1032A000D0699847BDE80840FFF794BE003C014054
:1032B000E02D0020074A08B5536903F0100353615D
:1032C00023B1054A136A0BB1506A9847BDE808401C
:1032D000FFF780BE003C0140E02D0020164B10B5EA
:1032E0005C6904F478725A61A30604D5134A936AA0
:1032F0000BB1D06A9847600604D5104A136B0BB126
:10330000506B9847210604D50C4A936B0BB1D06BD8
:103310009847E20504D5094A136C0BB1506C9847E5
:10332000A30504D5054A936C0BB1D06C9847BDE852
:103330001040FFF74FBE00BF003C0140E02D0020D1
:10334000194B10B55C6904F47C425A61620504D5DE
:10335000164A136D0BB1506D9847230504D5134AD7
:10336000936D0BB1D06D9847E00404D50F4A136EEE
:103370000BB1506E9847A10404D50C4A936E0BB163
:10338000D06E9847620404D5084A136F0BB1506F92
:103390009847230404D5054A936F0BB1D06F984723
:1033A000BDE81040FFF716BE003C0140E02D0020B4
:1033B00008B5FFF75DFEBDE80840FFF70BBE000053
:1033C000062108B50846FFF71DFB06210720FFF779
:1033D00019FB06210820FFF715FB06210920FFF73E
:1033E00011FB06210A20FFF70DFB06211720FFF72E
:1033F00009FB06212820FFF705FBBDE8084007214F
:103400001C20FFF7FFBA000008B5FFF745FE00F0EB
:103410000BF8FDF78FFEFDF767FDFFF7A5FDBDE893
:103420000840FFF7CFBC00000023054A19460133CE
:10343000102BC2E9001102F10802F8D1704700BF59
:10344000E02D0020034611F8012B03F8012B002A80
:10345000F9D1704753544D3332463F3F3F005354E8
:103460004D3332463430780053544D333246343283
:10347000780053544D3332463434365858000000E7
:10348000012033000010410001105A0003105900C0
:10349000071031000000000054340008130400003D
:1034A0005E3400081904000068340008210400009C
:1034B0007234000800000000650E0008510E00087C
:1034C0008D0E0008790E0008850E0008710E0008A8
:1034D0005D0E0008490E0008990E0008000000006B
:1034E000010000000000000063300000E834000824
:1034F000F0230020002600204172647550696C6F33
:10350000740025424F415244252D424C002553451D
:103510005249414C2500000002000000000000005C
:1035200081100008ED10000840004000A02A002093
:10353000B02A00200200000000000000030000008C
:103540000000000031110008000000001000000021
:10355000C02A002000000000010000000000000060
:10356000682D002001010200E51B0008F51A000883
:10357000911B0008751B00084300000080350008FF
:1035800009024300020100C03209040000010202E6
:103590000100052400100105240100010424020299
:1035A0000524060001070582030800FF0904010045
:1035B000020A000000070501024000000705810221
:1035C0004000000012000000CC350008120110017C
:1035D00002000040091241570002010203010000ED
:1035E0000403090425424F41524425006F6D6E6962
:1035F000627573663470726F2D6F6E650030313294
:1036000033343536373839414243444546000000AB
:1036100000400000004000000040000000400000AA
:103620000000010000000200000002000000020093
:103630000000020000000200000002000000020082
:1036400000000000751200082D150008D9150008AB
:1036500040004000C82D0020C82D002001000000BF
:10366000D82D002080000000400100000300000071
:103670006D61696E0069646C650000000001804244
:1036800000000000AAAAAAAA00010040FFFF000053
:103690000000000000A00A0040050001000000003A
:1036A000AAAAAAAA40020001CFFF00000000000061
:1036B000000000000000000000000000AAAAAAAA62
:1036C00000000000FFFF00000000000000000000FC
:1036D0000000000000000000AAAAAAAA0000000042
:1036E000FFFF0000000000000000000000000000DC
:1036F00000000000AAAAAAAA00000000FFFF000024
:1037000000000000000000000000000000000000B9
:10371000AAAAAAAA00000000FFFF00000000000003
:10372000000000000000000000000000AAAAAAAAF1
:1037300000000000FFFF000000000000000000008B
:1037400000000000000000000A000000000000006F
:103750000300000000000000000000000000000066
:103760000000000000000000000000000000000059
:1037700000000000000000008300000000000000C6
:1037800000000F0000000000FF009600000000088D
:10379000009600000000080004000000E03500086A
:1037A0000000000000000000000000000000000019
:1037B0000000000000000000FFFFFFFFFFFFFFFF11
:1037C000FFFFFFFFFFFFFFFFFFFFFFFFFFFFFFFF09
:1037D000FFFFFFFFFFFFFFFFFFFFFFFFFFFFFFFFF9
:1037E000FFFFFFFFFFFFFFFFFFFFFFFFFFFFFFFFE9
:1037F000FFFFFFFFFFFFFFFFFFFFFFFFFFFFFFFFD9
:020000040801F1
:10000000000600209912010871E00808CDDF0808F9
:1000100039E00808CDDF080805E008089B12010850
:100020009B1201089B1201089B120108F57F0B0827
:100030009B1201089B1201089B1201089B120108E8
:100040009B1201089B1201089B1201089B120108D8
:100050009B1201089B1201088D8B0B08B58B0B08B6
:10006000DD8B0B08058C0B082D8C0B08B9300B08A9
:10007000E1300B080D310B0839310B0865310B08E5
:100080008D310B08B9310B083D300B089B1201086C
:100090009B1201089B1201089B120108558C0B084A
:1000A000798D0B087D8D0B08918D0B08958D0B08B4
:1000B000998D0B08AD8D0B08C18D0B089B120108A3
:1000C0009B12010845370B08ED380B089B120108FD
:1000D0009B120108298D0B089B1201083D8D0B080E
:1000E000B98C0B089B1201089B120108E58D0B08C7
:1000F000E98D0B08FD8D0B08018E0B08E5310B080F
:100100009B1201089B120108D58D0B089B12010858
:10011000518D0B089B1201089B1201089B120108CC
:1001200011320B0839320B0865320B0891320B087B
:10013000BD320B089B1201089B1201089B1201089B
:100140009B1201089B1201089B12010821870B08D2
:10015000E5320B0811330B083D330B08658D0B0896
:100160009B1201089B1201089B1201089B120108B7
:100170009B1201089B1201089B1201089B120108A7
:100180009B1201089B1201089B1201089B12010897
:100190009B1201089B1201089B1201089B12010887
:1001A0009B1201089B1201089B1201089B12010877
:1001B0009B1201089B1201089B1201089B12010867
:1001C0009B1201089B1201089B1201089B12010857
:1001D0009B1201089B1201089B1201089B12010847
:1001E000113F0108ED88010819280208958A0308C3
:1001F000DD4F050835550508D1C40508B5280608A2
:1002000079300608B1330608C9980608A1B7060870
:10021000316E070861990708B9A6070825D20808B2
:1002200009D70808E5210A084D7B0A08A5A10A0894
:100230005DAC0A0825DC0A0805E30A080000000096
:1002400081F0004102E000BF83F0004330B54FEA87
:1002500041044FEA430594EA050F08BF90EA020FF4
:100260001FBF54EA000C55EA020C7FEA645C7FEA87
:10027000655C00F0E2804FEA5454D4EB5555B8BFAA
:100280006D420CDD2C4480EA020281EA030382EA1B
:10029000000083EA010180EA020281EA0303362DAD
:1002A00088BF30BD11F0004F4FEA01314FF4801C80
:1002B0004CEA113102D0404261EB410113F0004F92
:1002C0004FEA03334CEA133302D0524263EB430349
:1002D00094EA050F00F0A780A4F10104D5F1200EE7
:1002E0000DDB02FA0EFC22FA05F2801841F1000142
:1002F00003FA0EF2801843FA05F359410EE0A5F116
:1003000020050EF1200E012A03FA0EFC28BF4CF046
:10031000020C43FA05F3C01851EBE37101F00045FC
:1003200007D54FF0000EDCF1000C7EEB00006EEB09
:100330000101B1F5801F1BD3B1F5001F0CD3490893
:100340005FEA30004FEA3C0C04F101044FEA4452EA
:1003500012F5800F80F09A80BCF1004F08BF5FEA71
:10036000500C50F1000041EB045141EA050130BD51
:100370005FEA4C0C404141EB0101013C28BFB1F563
:10038000801FE9D291F0000F04BF01460020B1FAAE
:1003900081F308BF2033A3F10B03B3F120020CDA81
:1003A0000C3208DD02F1140CC2F10C0201FA0CF05F
:1003B00021FA02F10CE002F11402D8BFC2F1200CC4
:1003C00001FA02F120FA0CFCDCBF41EA0C0190407A
:1003D000E41AA2BF01EB0451294330BD6FEA0404C3
:1003E0001F3C1CDA0C340EDC04F11404C4F12002AE
:1003F00020FA04F001FA02F340EA030021FA04F3C0
:1004000045EA030130BDC4F10C04C4F1200220FA16
:1004100002F001FA04F340EA0300294630BD21FA54
:1004200004F0294630BD94F0000F83F4801306BF1A
:1004300081F480110134013D4EE77FEA645C18BF0E
:100440007FEA655C29D094EA050F08BF90EA020FA5
:1004500005D054EA000C04BF1946104630BD91EA9D
:10046000030F1EBF0021002030BD5FEA545C05D1A0
:100470004000494128BF41F0004130BD14F58004DF
:100480003CBF01F5801130BD01F0004545F0FE4153
:1004900041F470014FF0000030BD7FEA645C1ABF88
:1004A000194610467FEA655C1CBF0B46024650EABF
:1004B000013406BF52EA033591EA030F41F40021EB
:1004C00030BD00BF90F0000F04BF0021704730B571
:1004D0004FF4806404F132044FF000054FF0000146
:1004E00050E700BF90F0000F04BF0021704730B507
:1004F0004FF4806404F1320410F0004548BF4042DC
:100500004FF000013EE700BF42004FEAE2014FEA30
:1005100031014FEA02701FBF12F07F4393F07F4F0B
:1005200081F06051704732F07F4208BF704793F00E
:100530007F4F04BF41F40021704730B54FF4607421
:1005400001F0004521F000411CE700BF50EA010224
:1005500008BF704730B54FF000050AE050EA0102CD
:1005600008BF704730B511F0004502D5404261EB3D
:1005700041014FF4806404F132045FEA915C3FF47E
:10058000D8AE4FF003025FEADC0C18BF03325FEA1B
:10059000DC0C18BF033202EBDC02C2F1200300FACC
:1005A00003FC20FA02F001FA03FE40EA0E0021FAF1
:1005B00002F11444BDE600BF70B54FF0FF0C4CF4DF
:1005C000E06C1CEA11541DBF1CEA135594EA0C0F91
:1005D00095EA0C0F00F0DEF82C4481EA030621EACC
:1005E0004C5123EA4C5350EA013518BF52EA033507
:1005F00041F4801143F4801338D0A0FB02CE4FF0B9
:100600000005E1FB02E506F00042E0FB03E54FF0E8
:100610000006E1FB03569CF0000F18BF4EF0010EE0
:10062000A4F1FF04B6F5007F64F5407404D25FEADC
:100630004E0E6D4146EB060642EAC62141EA55518F
:100640004FEAC52040EA5E504FEACE2EB4F1FD0CD1
:1006500088BFBCF5E06F1ED8BEF1004F08BF5FEA4F
:10066000500E50F1000041EB045170BD06F0004601
:1006700046EA010140EA020081EA0301B4EB5C04AE
:10068000C2BFD4EB0C0541EA045170BD41F48011A6
:100690004FF0000E013C00F3AB8014F1360FDEBFCB
:1006A000002001F0004170BDC4F10004203C35DAA7
:1006B0000C341BDC04F11404C4F1200500FA05F32A
:1006C00020FA04F001FA05F240EA020001F00042CB
:1006D00021F0004110EBD37021FA04F642EB060141
:1006E0005EEA430E08BF20EAD37070BDC4F10C046B
:1006F000C4F1200500FA04F320FA05F001FA04F22F
:1007000040EA020001F0004110EBD37041F100011A
:100710005EEA430E08BF20EAD37070BDC4F1200525
:1007200000FA05F24EEA020E20FA04F301FA05F28D
:1007300043EA020321FA04F001F0004121FA04F235
:1007400020EA020000EBD3705EEA430E08BF20EA05
:10075000D37070BD94F0000F0FD101F0004640003F
:1007600041EB010111F4801F08BF013CF7D041EAC1
:10077000060195F0000F18BF704703F000465200C5
:1007800043EB030313F4801F08BF013DF7D043EA96
:100790000603704794EA0C0F0CEA135518BF95EA4C
:1007A0000C0F0CD050EA410618BF52EA4306D1D1D3
:1007B00081EA030101F000414FF0000070BD50EAF2
:1007C000410606BF1046194652EA430619D094EA7C
:1007D0000C0F02D150EA013613D195EA0C0F05D166
:1007E00052EA03361CBF104619460AD181EA0301BA
:1007F00001F0004141F0FE4141F470014FF0000072
:1008000070BD41F0FE4141F4780170BD70B54FF00C
:10081000FF0C4CF4E06C1CEA11541DBF1CEA13558C
:1008200094EA0C0F95EA0C0F00F0A7F8A4EB05046E
:1008300081EA030E52EA03354FEA013100F0888065
:100840004FEA03334FF0805545EA131343EA12632E
:100850004FEA022245EA111545EA10654FEA0026E3
:100860000EF000419D4208BF964244F1FD0404F59C
:10087000407402D25B084FEA3202B61A65EB0305F8
:100880005B084FEA32024FF480104FF4002CB6EBB5
:10089000020E75EB030E22BFB61A754640EA0C0035
:1008A0005B084FEA3202B6EB020E75EB030E22BF75
:1008B000B61A754640EA5C005B084FEA3202B6EBB6
:1008C000020E75EB030E22BFB61A754640EA9C0075
:1008D0005B084FEA3202B6EB020E75EB030E22BF45
:1008E000B61A754640EADC0055EA060E18D04FEA03
:1008F000051545EA16754FEA06164FEAC30343EAA3
:1009000052734FEAC2025FEA1C1CC0D111F4801F6F
:100910000BD141EA00014FF000004FF0004CB6E768
:1009200011F4801F04BF01430020B4F1FD0C88BF07
:10093000BCF5E06F3FF6AFAEB5EB030C04BFB6EB12
:10094000020C5FEA500C50F1000041EB045170BD05
:100950000EF0004E4EEA113114EB5C04C2BFD4EB32
:100960000C0541EA045170BD41F480114FF0000EB6
:10097000013C90E645EA060E8DE60CEA135594EA32
:100980000C0F08BF95EA0C0F3FF43BAF94EA0C0F35
:100990000AD150EA01347FF434AF95EA0C0F7FF4AA
:1009A00025AF104619462CE795EA0C0F06D152EAFE
:1009B00003353FF4FDAE1046194622E750EA4106E2
:1009C00018BF52EA43067FF4C5AE50EA41047FF4F3
:1009D0000DAF52EA43057FF4EBAE12E74FF0FF3C58
:1009E00006E000BF4FF0010C02E000BF4FF0010C29
:1009F0004DF804CD4FEA410C7FEA6C5C4FEA430CA2
:100A000018BF7FEA6C5C1BD001B050EA410C0CBFF0
:100A100052EA430C91EA030F02BF90EA020F002052
:100A2000704710F1000F91EA030F58BF994208BFB9
:100A300090422CBFD8176FEAE37040F00100704776
:100A40004FEA410C7FEA6C5C02D150EA013C07D1CD
:100A50004FEA430C7FEA6C5CD6D152EA033CD3D018
:100A60005DF8040B704700BF8446104662468C4612
:100A70001946634600E000BF01B5FFF7B7FF002845
:100A800048BF10F1000F01BD4DF808EDFFF7F4FF6E
:100A90000CBF012000205DF808FB00BF4DF808EDF9
:100AA000FFF7EAFF34BF012000205DF808FB00BF1C
:100AB0004DF808EDFFF7E0FF94BF012000205DF83E
:100AC00008FB00BF4DF808EDFFF7CEFF94BF0120F3
:100AD00000205DF808FB00BF4DF808EDFFF7C4FFEC
:100AE00034BF012000205DF808FB00BF4FEA410C35
:100AF0007FEA6C5C02D150EA013C0AD14FEA430C18
:100B00007FEA6C5C02D152EA033C02D14FF0000054
:100B100070474FF0010070474FEA410212F5001292
:100B200015D211D56FF47873B3EB625212D94FEA34
:100B3000C12343F0004343EA505311F0004F23FA1E
:100B400002F018BF404270474FF00000704750EA73
:100B5000013005D111F0004008BF6FF00040704730
:100B60004FF00000704700BF4A0011D212F500128A
:100B700011D20DD56FF47873B3EB62520ED44FEAF5
:100B8000C12343F0004343EA505323FA02F0704775
:100B90004FF00000704750EA013002D14FF0FF30B3
:100BA00070474FF0000070474FEA4102B2F1E04356
:100BB00024BFB3F5001CDCF1FE5C0DD901F0004C44
:100BC0004FEAC0024CEA5070B2F1004F40EB830094
:100BD00008BF20F00100704711F0804F21D113F1C0
:100BE0003872BCBF01F00040704741F480114FEAF9
:100BF0005252C2F11802C2F1200C10FA0CF320FA82
:100C000002F018BF40F001004FEAC1234FEAD3239E
:100C100003FA0CFC40EA0C0023FA02F34FEA430308
:100C2000CCE77FEA625307D150EA01331EBF4FF091
:100C3000FE4040F44000704701F0004040F0FE40AC
:100C400040F40000704700BF80F0004002E000BFA9
:100C500081F0004142001FBF5FEA410392EA030FA7
:100C60007FEA226C7FEA236C6AD04FEA1262D2EBF1
:100C70001363C1BFD218414048404140B8BF5B42F6
:100C8000192B88BF704710F0004F40F4000020F08F
:100C90007F4018BF404211F0004F41F4000121F0A5
:100CA0007F4118BF494292EA030F3FD0A2F10102EF
:100CB00041FA03FC10EB0C00C3F1200301FA03F12D
:100CC00000F0004302D5494260EB4000B0F5000F50
:100CD00013D3B0F1807F06D340084FEA310102F10F
:100CE0000102FE2A51D2B1F1004F40EBC25008BFC1
:100CF00020F0010040EA03007047490040EB00008B
:100D0000013A28BFB0F5000FEDD2B0FA80FCACF18B
:100D1000080CB2EB0C0200FA0CF0AABF00EBC250B8
:100D200052421843BCBFD0401843704792F0000FA6
:100D300081F4000106BF80F400000132013BB5E7F9
:100D40004FEA41037FEA226C18BF7FEA236C21D06F
:100D500092EA030F04D092F0000F08BF08467047D4
:100D600090EA010F1CBF0020704712F07F4F04D1A2
:100D7000400028BF40F00040704712F100723CBFB5
:100D800000F50000704700F0004343F0FE4040F4DF
:100D9000000070477FEA226216BF08467FEA23639D
:100DA0000146420206BF5FEA412390EA010F40F488
:100DB000800070474FF0000304E000BF10F00043D4
:100DC00048BF40425FEA000C08BF704743F09643BB
:100DD00001464FF000001CE050EA010208BF7047D6
:100DE0004FF000030AE000BF50EA010208BF70475D
:100DF00011F0004302D5404261EB41015FEA010C72
:100E000002BF84460146002043F0B64308BFA3F169
:100E10008053A3F50003BCFA8CF2083AA3EBC2534B
:100E200010DB01FA02FC634400FA02FCC2F120026A
:100E3000BCF1004F20FA02F243EB020008BF20F0A1
:100E40000100704702F1200201FA02FCC2F1200207
:100E500050EA4C0021FA02F243EB020008BF20EAFC
:100E6000DC7070477BB972B90029BEBF00204FF01B
:100E7000004106E008BF00281CBF6FF000414FF0A2
:100E8000FF3000F007BAADF1080C6DE904CE00297F
:100E900009DB002B1ADB00F095F8DDF804E0DDE952
:100EA000022304B07047404261EB4101002B1BDB81
:100EB00000F088F8DDF804E0DDE9022304B04042E8
:100EC00061EB4101524263EB43037047524263EBD3
:100ED000430300F077F8DDF804E0DDE9022304B015
:100EE000404261EB41017047524263EB430300F023
:100EF00069F8DDF804E0DDE9022304B0524263EB57
:100F00004303704753B94AB9002908BF00281CBFE2
:100F10004FF0FF314FF0FF3000F0BCB9ADF1080CDD
:100F20006DE904CE00F04EF8DDF804E0DDE90223BF
:100F300004B07047430803F05533C01A830803F028
:100F4000333300F03330184400EB101000F00F3052
:100F500000EB002000EB0040000E704707EE900A07
:100F6000F5EEC07AF1EE10FA01D400F00BB8F1EE14
:100F7000677A08B517EE900A00F004F8404261EB7A
:100F8000410108BDD0B5FFF7BFFA0C4B0022064661
:100F90000F46FFF711FBFFF7E7FD0446FFF792FA54
:100FA000074B0022FFF708FB02460B463046394646
:100FB000FFF74AF9FFF7D8FD2146D0BD0000F03D0C
:100FC0000000F0412DE9F047089D04468E46002BB5
:100FD0004DD18A42944669D9B2FA82F252B101FAED
:100FE00002F3C2F1200120FA01F10CFA02FC41EAFD
:100FF000030E94404FEA1C48210CBEFBF8F61FFA82
:101000008CF708FB16E341EA034306FB07F199421C
:101010000AD91CEB030306F1FF3080F01F819942CF
:1010200040F21C81023E63445B1AA4B2B3FBF8F0A9
:1010300008FB103344EA034400FB07F7A7420AD930
:101040001CEB040400F1FF3380F00A81A74240F258
:1010500007816444023840EA0640E41B00261DB1C3
:10106000D4400023C5E900433146BDE8F0878B42F8
:1010700009D9002D00F0EF800026C5E900013046B7
:101080003146BDE8F087B3FA83F6002E4AD18B4291
:1010900002D3824200F2F980841A61EB030301203B
:1010A0009E46002DE0D0C5E9004EDDE702B9FFDE27
:1010B000B2FA82F2002A40F09280A1EB0C014FEAD2
:1010C0001C471FFA8CFE0126200CB1FBF7F307FB2F
:1010D000131140EA01410EFB03F0884208D91CEBD2
:1010E000010103F1FF3802D2884200F2CB8043466F
:1010F000091AA4B2B1FBF7F007FB101144EA01444E
:101100000EFB00FEA64508D91CEB040400F1FF31DC
:1011100002D2A64500F2BB800846A4EB0E0440EACA
:1011200003409CE7C6F12007B34022FA07FC4CEAD3
:10113000030C20FA07F401FA06F31C43F9404FEAC6
:101140001C4900FA06F3B1FBF9F8200C1FFA8CFEDB
:1011500009FB181140EA014108FB0EF0884202FA2F
:1011600006F20BD91CEB010108F1FF3A80F08880F0
:10117000884240F28580A8F102086144091AA4B2AD
:10118000B1FBF9F009FB101144EA014100FB0EFE2E
:101190008E4508D91CEB010100F1FF346CD28E455D
:1011A0006AD90238614440EA0840A0FB0294A1EBEE
:1011B0000E01A142C846A64656D353D05DB1B3EB4B
:1011C000080261EB0E0101FA07F722FA06F3F1407B
:1011D0001F43C5E9007100263146BDE8F087C2F122
:1011E0002003D8400CFA02FC21FA03F3914001439A
:1011F0004FEA1C471FFA8CFEB3FBF7F007FB1036D3
:101200000B0C43EA064300FB0EF69E4204FA02F47E
:1012100008D91CEB030300F1FF382FD29E422DD9D1
:10122000023863449B1B89B2B3FBF7F607FB163306
:1012300041EA034106FB0EF38B4208D91CEB010186
:1012400006F1FF3816D28B4214D9023E6144C91A06
:1012500046EA004638E72E46284605E70646E3E616
:101260001846F8E64B45A9D2B9EB020864EB0C0E20
:101270000138A3E74646EAE7204694E74046D1E72F
:10128000D0467BE7023B614432E7304609E76444DD
:10129000023842E7704700BF02E000F000F8FEE7C6
:1012A00072B6374880F30888364880F30988364894
:1012B0003649086040F20000CCF200004EF634716E
:1012C000CEF200010860BFF34F8FBFF36F8F40F283
:1012D0000000C0F2F0004EF68851CEF20001086026
:1012E000BFF34F8FBFF36F8F4FF00000E1EE100A96
:1012F0004EF63C71CEF200010860062080F314889F
:10130000BFF36F8FA6F0D4FEA5F03EFF4FF055302F
:101310001F491B4A91423CBF41F8040BFAE71D49A3
:10132000184A91423CBF41F8040BFAE71A491B4A9C
:101330001B4B9A423EBF51F8040B42F8040BF8E7EE
:1013400000201849184A91423CBF41F8040BFAE7C3
:10135000A6F0B2FEA5F06CFF144C154DAC4203DABA
:1013600054F8041B8847F9E700F060FC114C124D5B
:10137000AC4203DA54F8041B8847F9E7A6F09ABE9A
:1013800000060020002200200000010808ED00E017
:10139000000000200006002000E60D0800220020CA
:1013A0003827002038270020C8400120E00101082C
:1013B0003C0201083C0201083C0201082DE9F04F03
:1013C0002DED108AC1F80CD0C3689D46BDEC108A83
:1013D000BDE8F08F002383F311882846A047002042
:1013E000A5F058FCFEE7A5F0B5FA00DFFEE7000027
:1013F00001F0FF01102A2BDB10F0070F08D010F8C6
:10140000013B013A8B422DD010F0070F42B3F6D1C9
:10141000F0B441EA012141EA014122F007047FF0E2
:1014200000070023F0E80256083C85EA010586EA39
:10143000010685FA47F5A3FA87F586FA47F6A5FA75
:1014400087F68EB9EED1F0BC01F0FF0102F0070281
:1014500032B110F8013B013A83EA010313B1F8D12C
:101460000020704701387047002D06BF354603380D
:10147000073815F0010F07D1013015F4807F02BF46
:10148000013015F4C03F0130F0BC0138704700BF97
:1014900010F8012B11F8013B012A28BF9A42F7D01E
:1014A000D01A7047034613F8012B002AFBD1181AF3
:1014B0000138704738B50022002304460D46FFF777
:1014C000EDFA28B920462946BDE8384000F00AB8B0
:1014D000204605F1004100F005F8404261EB410172
:1014E00038BD00BFD0B50C4B002206460F46FFF7B3
:1014F00063F8FFF739FB0446FEF7E4FF074B0022D1
:10150000FFF75AF802460B4630463946FEF79CFE76
:10151000FFF72AFB2146D0BD0000F03D0000F0415E
:10152000036800221B6818471FB5094BD3F85C29D4
:101530000092D3F860290192D3F864290292D3F87B
:10154000683903936A4672F021FC05B05DF804FB2C
:101550005047002070B50024144E2546E1B23046B5
:1015600003F0DCFE002178F067FD02281CD004287F
:101570001AD0012804F1010408BF0125102CEDD177
:101580000DB9002070BD094D0024E1B2284603F0DA
:10159000C5FE012178F050FD022805D0042803D0B3
:1015A0000134102CF1D1ECE70120EBE750270020AB
:1015B00037B5C47F0191054644B9FFF7CBFF0199C8
:1015C000044630B9064A284671F086FD204603B02D
:1015D00030BD284603B0BDE8304072F03DBC00BFCE
:1015E0007C030C08F0B591B005460E4671F01CFE68
:1015F0000446D8B11021284671F066FBB0B1002135
:101600002E2204A803AF0391AAF088FC0BF004FF7C
:1016100032233A4600210BF05BFA044630B9054B01
:10162000009732461021284671F056FB204611B033
:10163000F0BD00BFA8030C08F8B5394F3B7806464B
:10164000002B6AD101253D7072F0C0FC044630B910
:10165000344A387013782B4313702046F8BD4CF091
:10166000ADFE29464BF096FE2F4803F0D5F92F4BDF
:101670001D710B253FF0A4F8013D3FF057F815F020
:10168000FF05F7D10BF0C8FE294BD0F80022C3F8B4
:10169000F02090F87C22D10706D5920704D4294681
:1016A000A3F5405002F07EFC224B234D1B68D86A04
:1016B000036801211B6898471B4808F067FB01215C
:1016C0001E4879F03DFD4CF079FE95F8EC2095F838
:1016D000841D4CF03BF8A5F5005003F08FF948F05D
:1016E0000DFF48F04DFA0023A5F500503B7000F0C7
:1016F0002FFA0028B1D156F013FE0421104A4FF002
:1017000069FF2021304671F0DFFA0028A5D00D4B8B
:1017100001222021304671F0DFFA00249DE700BF4E
:1017200038270020EC7E002050270020CD7E0020AE
:10173000505700204827002050470020FC5400202C
:10174000B4030C08D1030C0830B5204B93F8773E56
:1017500085B01BB90024204605B030BD72F0ECFC0A
:1017600004460028F6D00BF057FE05460AF0AEFC02
:10177000A8B111F025FB90F91830022B0FD10023EE
:1017800001AA002128460193029303930BF03CF831
:1017900028B111F015FB01AA002111F0E3F8002196
:1017A0000B4879F0CDFC0B4826F014FF4CF006FEF8
:1017B00000214BF0EFFD084B1B68D86A036800213D
:1017C0001B689847054803F03BFFC4E750470020DB
:1017D000FC5400206C510020482700205027002096
:1017E00009F070B85AF0ACBA48F0D2BD1FF0D6B9C3
:1017F0004BF052BF0FF0A4BB5AF0ECBD57F0F4BE53
:1018000056F042B809F082B808F0F6BC40F00ABAC7
:1018100019F0CABB5AF0EEBD08F0F0BD02F0B0BB43
:1018200004F056BE00F0E0BB03F034BD08F0AEBBE0
:101830001FF0A6BD034808601F21117008221A601E
:10184000704700BFC4060C0810B5044603F044FB03
:10185000204603F01BFC204603F09EFA204603F0CE
:1018600047FA58F031FABDE8104058F00DB90000C1
:10187000FFF7EABF38B5044600F5445004300EF0D7
:10188000BDFE11F09DFA90F91530F3B190F8F431E6
:10189000DBB104F5375030304FF04AFA034693ED90
:1018A000000ADFED0A0A9F20B7EE001A21F0ACFC17
:1018B00094F9BC3304F56575012B08BF84EDF00A7B
:1018C0002846BDE8384011F0AFB938BD000000002F
:1018D000FFF7D0BF37B50121044608F0D7FF88B322
:1018E00004F55F552046183501F00AFE284672F0CF
:1018F00049FC04F570512031284672F0A9FC4FF4E0
:101900008051204608F0C2FFE0B104F5675204F6AA
:10191000A8603032692101904BF01CFC04F56B5239
:10192000019818326A214BF015FC019804F56F52AA
:101930006B214BF00FFC04F57B52019808326C21AF
:101940004BF008FC8021204608F0A0FF60B14FF466
:101950000021204608F09AFF30B920F00DFF03B0B7
:10196000BDE830401EF034BD03B030BDFFF7B2BF5C
:1019700010B5044600F52550343078F0B5FB20460C
:1019800003F0DEF8204603F04DF8204603F090F80F
:10199000204603F0EFFA204603F024FC204603F033
:1019A00059FC04F585500830BDE810405FF038B8A8
:1019B000FFF7DEBF10B5044600F58850083001215E
:1019C0000BF09CFC04F55C501C30BDE8104009F0A5
:1019D00033BF0000FFF7EEBF10B5044608F0C0FBB0
:1019E0001021204608F052FF40B1204601F0DAFCF9
:1019F00020F0C2FEBDE810401EF0E6BD10BD0000A4
:101A0000FFF7EABF10B500F5005292F8813D13F0E0
:101A1000010408D1084A00F52D50183004214FF078
:101A2000D9FD002010BD92F8A53DDB0701D5034A82
:101A3000F1E70120F6E700BF40040C085F040C0842
:101A400000230B600120704710B5044604F50054D4
:101A50006BF0E8FA94F8771EBDE810406BF0BEBA60
:101A6000FFF7F2BF13B500F50053044693F8813D2C
:101A7000DA0729D500F5885001A908300AF0FEFBE5
:101A8000B8B104F5805494F88433DB070BD594ED9A
:101A9000DE7ADFED0F6ADDED017AB8EEC77AE7EEA8
:101AA000667ACDED017A9DED010AB1EE400A02B0F1
:101AB00010BD0EF039F8437C242202FB0300D0ED68
:101AC0000B7AF1EE677AECE79FED020AEFE700BFD1
:101AD0000AD7233C0000000010B500F5005386B083
:101AE00093F8813DDB07044603D49FED170A06B047
:101AF00010BD04F5885402A8083410F045FB02A973
:101B000020460BF07BFA0028EFD001A920460AF00E
:101B1000B5FB58B90EF008F8437C242202FB030001
:101B2000D0ED0B7AF1EE677ACDED017ADDED037A37
:101B30009FED067A9DED010AF8EEE77AA7EEC70A57
:101B4000B1EE400AD3E700BF000000000AD7233CF3
:101B500070B505468AB005F5885602A8083610F01B
:101B600013FB02A930460BF049FA044688BB05F581
:101B7000907018F083F960BB254ADFED267AD2ED2C
:101B8000006A12ED017A9FED246A66EEA76A52EDB3
:101B9000027A009427EE067A67EE867AFDEEE66A10
:101BA000BDEEC77AFDEEE77A16EE903A17EE102AF0
:101BB00017EE901A06A810F007FB089805F52D55AA
:101BC000183508B1099939B9144A042128464FF04B
:101BD00001FD20460AB070BD21F07CFD044608B925
:101BE0000F4AF2E706A930460BF02EF8044608B972
:101BF0000C4AEAE70C4A062128464FF0EBFC304637
:101C00000BF0EAFD4521284657F0A8F9E1E700BFAF
:101C1000A85000200000C8428096184B74040C089D
:101C2000A3040C08CC040C08FB040C0838B5054BC5
:101C30001C6823680A461D68034B01462046A847D6
:101C4000002038BD482700205027002010B504464A
:101C500048F054FC04F5005101F6AC53426FDA60D1
:101C600004F5405303F5FB6003F542638266C3F855
:101C7000FC2291F8843D133B012B06D904F55F50FB
:101C80001830BDE8104072F0CBBE10BDFFF7DEBFCC
:101C900037B50221044608F0F9FDB0B30121204612
:101CA00008F0F4FD88BB04F55F552046183501F0B7
:101CB00027FC284672F066FA04F570512031284658
:101CC00072F0C6FA4FF48051204608F0DFFDE0B113
:101CD00004F5675204F6A8603032692101904BF098
:101CE00039FA04F56B52019818326A214BF032FA36
:101CF000019804F56F526B214BF02CFA04F57B52DE
:101D0000019808326C214BF025FA4FF4003120463F
:101D100008F0BCFD20B104F536502C307AF004FAFE
:101D20004021204608F0B2FD18B104F6A8604AF040
:101D3000AFFE4FF48061204608F0A8FD18B104F60C
:101D4000A8604AF03FFF2021204608F09FFD58B1CF
:101D5000224DD5F8980303689B68984728B304F58B
:101D60007050203075F01AFD8021204608F08EFD5D
:101D700018B320F001FD1EF04FFB1021204608F0A3
:101D800085FD20B104F55F50183072F04BFF4FF421
:101D90000041204608F07AFDF0B104F5944020306F
:101DA00003B0BDE830405AF04DBCD5F89803036845
:101DB000DB6898470028D2D0D6E74FF48021204630
:101DC00008F064FD0028D4D14FF40021204608F02B
:101DD0005DFD0028CDD1D0E703B030BD50770020A5
:101DE000FFF756BF70B500F500552C4BB5F8322102
:101DF0001A70044600F5595000213830FFF7D8FB1F
:101E000095F8803D264E60F3000385F8803DB07163
:101E1000204608F029FD95F8773EF0714FF6FF71E6
:101E20002046737108F032FD28B1D5F8802D0721C6
:101E3000204601F083FB95F8773E23B904F5365030
:101E40002C307AF07BFB59F0A5FC59F073F9204651
:101E500008F04EFD134B1B68DB6A93F89C6036B1AB
:101E600095F8EE301BB97CF039F9C5F8F00085F82B
:101E7000EE6048F043FB47F0ABFF04F55F501830CD
:101E800072F03CFB48F03AFB47F0A2FF04F57850B3
:101E90003430BDE870406AF02FB900BF7C230020C9
:101EA000CD7E002048270020FFF79CBF10B50648D4
:101EB0000C4676F0FDFEDFED057A20EE270A0120C4
:101EC00084ED000A10BD00BF846700200AD7233CC0
:101ED00010B508480C4676F0FFFE07EE900A9FED1D
:101EE000067AF8EEE77A012067EE877AC4ED007A89
:101EF00010BD00BF846700200AD7233C70B52DEDCC
:101F0000048B00F5005482B00E4615464FF47A71EA
:101F10004FF4FA52B4F92C018DED011AF0EE408A1B
:101F2000B0EE608A21F0AEF9034607EE903ADFED9D
:101F3000240AA4F82C01B8EEE71A0B209DED010A43
:101F4000DFED209A21F060F9B4F92C31DFED1E6A43
:101F500007EE103AB8EEC77AB0EE409AC7EE267A8E
:101F600067EEA88A27EE888A28EEA80AA8EE080A53
:101F7000A7F024FFB4EEC09AF1EE10FA42BFC9EE0A
:101F8000007A28EE278A68EEA78A28EE290AA7F0A9
:101F9000A9FBB0EE409A28EEA90AA7F033FD29EE7E
:101FA000000AA7F07FFADFED097A20EE270A86ED16
:101FB000000A85ED008A02B0BDEC048B70BD00BF45
:101FC00000007A44D402373900A08C459F0CB345F9
:101FD00007EE901A00F50050F8EEE77A90ED740ADB
:101FE00027EE800A7047000073B5044600F588505C
:101FF00001A9083004F500560AF0C8FDD6F8543B94
:102000008342054606D004F55F50183073F0DCFEBD
:10201000C6F8545B02B070BD38B50F4A137801336F
:10202000DBB2032B044600F5405505D8137005F2CA
:10203000E46595ED000A38BD002300F55C5013708F
:1020400077F0E2FF04F55B51183121F0C1FA05F297
:10205000E46383ED000AEAE73927002038B5044637
:102060002DED028B00F55C5077F0D4FF054623F090
:10207000C9F92046B0EE408A08F0F6FB04F540545A
:10208000C0B1DFED107AB4EEE78AF1EE10FA11DD9F
:10209000D5ED000A95ED010AA7F046FDDFED0A7ABD
:1020A00020EE270ADFED097A20EE270A04F2F46316
:1020B00083ED000ABDEC028B04F2F46494ED000A97
:1020C00038BD00BF00401C46E02E65420000C842FB
:1020D00000F58050D0EDD65AD2ED007AD0EDD96A15
:1020E00091ED006A26EEE77A67EEA57AA6EE257AEC
:1020F000E6EE267A81ED007AC2ED007A70470000A4
:1021000000F50050B0F95E3133B9B0F95C01002838
:10211000B8BF404280B2704783EAE370A0EBE3703F
:10212000F8E7000070B52DED068B00F5005482B085
:1021300094F8A41D8DED010A11F0010105460091EE
:1021400062D1D4F864099FED329A57F017FEB4F9C2
:102150006231DFED300A9DED010A07EE900A08EECC
:10216000103A05F5405606F2BC63F8EEE79AB8EE71
:10217000C88AD3ED007A6720B0EE491A28EE278A84
:1021800021F042F839EEC8AA0099B4F962014FF47F
:10219000C872F0EE408A21F075F8B4EEE8AAF1EECC
:1021A00010FAA4F8620116DD2846FFF7A9FF07EE32
:1021B000900A78EECA8AB8EEE70A60EE288A88EEBE
:1021C0008A0AFDEEC07A17EE903AA6F8F43002B013
:1021D000BDEC068B70BD78EE297AF4EEE87AF1EE6C
:1021E00010FA49BFB4F95C319FED0A0A00EE103ACB
:1021F00078EEE78A41BFB8EEC00A79EE677A60EE02
:10220000288A88EEA70ADCE79FED020ADFE700BF15
:1022100000007A4400000000002070477047000072
:102220007047000070470000002070470020704792
:102230000020704701207047002070477047000061
:102240007047000070470000002070470C4991F86B
:10225000843D102B0FD801229A400A4B1340002BCB
:102260000CBF1020182091F8773E33B940F04000A1
:1022700040F0010070471020F5E740F0C000F7E79C
:102280005047002098000100014B93F8340170473B
:10229000504700207047000010B5044652F08CFCF7
:1022A000054879F033F8054A034606212046BDE883
:1022B000104052F069BC00BFFC54002038090C08E3
:1022C00000B513EE103A8DB06222CDF8253013EE32
:1022D000903ACDF829302123CDE900328DF8241031
:1022E000192303AAC2218DED030ACDED040A8DED59
:1022F000051ACDED061A8DED072ACDED082A50F00E
:102300009DF90DB05DF804FB08B50B484EF010FDCB
:102310000346DFED0A0A93ED000A9F20B7EE001A8C
:1023200020F072FFDFED067A20EE270ABDEEC00A2C
:1023300010EE103A18B208BD405500200000000011
:102340000000C8420148FFF7C7BB00BF502700206C
:1023500008B50648FFF7C0FBDFED057A20EE270A37
:10236000FDEEC07A17EE900A08BD00BF502700208E
:1023700000007A44F8B5704E04460BF04DF8B6F8FC
:1023800070310546D80736D56C4BDFED6D7AD3ED4D
:10239000002A9FED6C7AD5EDC50A207C06F5D05356
:1023A00093ED002A53ED011A93ED021A13ED040A7E
:1023B000D3ED043A93ED053A62EEA72A22EE272ADE
:1023C00061EEA71A21EE271A60EE870A20EE270A8F
:1023D0000121FFF775FF207C50F0C6F80746207CEE
:1023E00050F0C6FF00F121039F4204D2207CBDE8DB
:1023F000F8404FF00FBBB6F8703199072FD5524B0C
:10240000DFED4F7A53ED032A13ED042A53ED051A3D
:1024100013ED021A13ED080A9FED4A7AD5EDC60AAC
:10242000D3ED003A93ED013A207C62EEA72A22EE2A
:10243000272A61EEA71A21EE271A60EE870A20EEFE
:10244000270A0221FFF73CFF207C50F08DF8074659
:10245000207C50F08DFF00F121039F42C6D3B6F8D7
:1024600070315A072FD5394BDFED357A53ED032AFA
:1024700013ED042A53ED051A13ED021A13ED080AA1
:102480009FED307AD5EDC70AD3ED003A93ED013ACE
:10249000207C62EEA72A22EE272A61EEA71A21EEFF
:1024A000271A60EE870A20EE270A0321FFF708FFAC
:1024B000207C50F059F80746207C50F059FF00F17D
:1024C00021039F4292D3B6F870311B0732D5204BBF
:1024D0009FED207AD5EDD60ADFED197A53ED032A68
:1024E00013ED042A53ED051A13ED021A13ED080A31
:1024F000D3ED003A93ED013A207C70EE870A62EE4C
:10250000A72A22EE272A61EEA71A21EE271A20EE2B
:10251000270AF1EE600A0421FFF7D2FE207C50F07A
:1025200023F80546207C50F023FF00F121039D4253
:10253000FFF45CAFF8BD00BF50470020546100209D
:102540000AD7233CE02E6542486200203063002019
:10255000386600200AE81C41014802F093B800BF29
:102560005027002007B5084601910FF015FF38B13C
:102570000448019904F05CFE002003B05DF804FB00
:102580000420FAE7DC7B002038B5C5780B46352DF2
:10259000044628BF3525352200211846A9F0BEFC87
:1025A0002A4604F10C01BDE83840A9F06DBC0000DA
:1025B0002DE9F0472DED028B8A7A4B7A43EA02230C
:1025C000CA7A43EA0243522BA2B005460C4600F0F9
:1025D000568111D8452B00F0E680462B00F03C8157
:1025E000012B00F062822146284622B0BDEC028B0E
:1025F000BDE8F04755F0B4BE562B00F0DA8100F28A
:10260000C080542BEFD114A92046FFF7BDFFAE4B7D
:1026100093F8842D042A09D0032A40F0188103F589
:10262000405393F83C36032B40F011819DF88420F1
:102630000C2A00F20C8141F28234D440E44314F0BD
:10264000010440F00481BDF88030002613F0070734
:1026500003F0380A03F4E07903F4806803F40065BA
:102660000D960E960F962CD19FED986A9DED167AD9
:10267000DDED177ADDED156A27EE067A67EEC67A8C
:1026800066EE866AA2F10803012BCDED0D6A8DED91
:102690000E7ACDED0F7A01D90C2A04D18C480EAAFE
:1026A0000DA9FFF715FD9DF88430DA1F022A01D924
:1026B0000C2B06D1874877F0A5FC01460DA823F026
:1026C0007FF9109611961296BAF1000F20D19FED66
:1026D0007F6A9DED197ADDED1A7ADDED186A9DF8B5
:1026E000843027EE067A67EEC67A66EE866AA3F134
:1026F0000802012ACDED106A8DED117ACDED127A26
:1027000001D90C2B04D1724811AA10A9FFF7E0FCE3
:10271000B8F1000F40F02381DFED6F7A9DED1E0AC6
:102720009DF8844020EE270ADFED687AA4F10906BF
:10273000744220EE270A7441002D40F01381DFED32
:10274000667ADDED1F0A60EEA70ADFED607A60EEC3
:10275000A70A002F40F00981BAF1000F40F019815B
:10276000B9F1000F73D0B5FA85F56D09B8FA88F3A1
:10277000019400955B0910AA0DA9584805F08CFC3E
:1027800065E003F18073863B23F07F43012B3FF626
:102790002AAF0A46017C524822B0BDEC028BBDE84C
:1027A000F04748F0EDBB484DCA79B5F934319A424B
:1027B0004DD1CE781E2E28BF1E261E22002114A821
:1027C000A9F0ACFB324604F10C0114A8A9F05CFBA3
:1027D0009DF85A20B5F932319A4238D1BDF96C30A2
:1027E0000B93BDF96A300A93BDF968300993BDF9BE
:1027F00066300893BDF964300793BDF962300693E3
:10280000BDF960300593BDF95E3004939DF85D30ED
:102810000393BDF85B300293BDF858300193BDF9C6
:102820005630BDF95220BDF950100093A5F5005067
:10283000BDF9543003F0EAFB7BF050FCC5F8900D75
:1028400055F06EFD04467BF049FCC4F8B80122B097
:10285000BDEC028BBDE8F0871B4ECA79B6F9343166
:102860009A42F4D17BF03AFC2146C6F8900D2846F6
:1028700022B0BDEC028BBDE8F04753F0F3BFCD783A
:10288000272D28BF27252722002114A8A9F046FBC1
:102890002A4604F10C0114A8A9F0F6FA9DF8763046
:1028A0005F0623D57BF01AFC0E4D14ACC5F854031B
:1028B0000FCC05F556750FC50FCC0FC594E8030076
:1028C00085E80300C3E700BF504700200000C8426E
:1028D00050270020505E0020E02E6542187C00202A
:1028E00008720020507700200000000013F0C00F95
:1028F000ADD15FED030A9DED1C0A40F2C120B7EE99
:10290000001A20F081FCF6EE000AB0EE408A20F0BA
:1029100079FB08BBB6EE007A834BB4EEC78AF1EEC2
:1029200010FA78EE477AD4BF93ED150A93ED140AA6
:1029300077EEA77AD8BFB0EEC00A20EE270A159B23
:102940001093169B1193179B12937848189B13931F
:1029500010A905F067FC7AE79FED750AEFE79FED98
:10296000740AE9E6DFED720AF3E6BAF1000F7FF4CC
:102970006EAFB9F1000F3FF46AAFB5FA85F3B8FA5C
:1029800088F26A4800945B09520910A905F0B6FA6A
:102990005DE7B9F1000F3FF45AAFB5FA85F3B8FA25
:1029A00088F200945B0952090DA9604806F07CF892
:1029B0004DE714A92046FFF7E7FD5E4A92F8843DF3
:1029C000042B08D0032B1CD102F5405292F83C2670
:1029D000032A7FF43CAFBDF88020500702F00701C6
:1029E00002F0380602F4E0740DD4022B0BD1DDEDB9
:1029F000177A9FED517A514B67EE877AC3ED007AD3
:102A000025E7022BE5E700230D930E930F93002992
:102A10006AD1DDE9150120F05DFE00283FF417AF13
:102A20009DF884100CAA284655F010F800283FF4B1
:102A30000EAFDDED177A9FED408A0C9B009367EE99
:102A4000887ADDE91512FDEEE77A10A817EE903AC4
:102A50000FF0BAFB0DA910A80FF058FD00283FF4A5
:102A6000F6AED6B9002C3FF4F2AEDDED186A9DED5E
:102A7000197ADDED1A7A2D4866EE886A27EE087A13
:102A800027EEC88A10AA0DA9CDED106A8DED117A36
:102A90008DED128A05F094FAD9E6002C3FF4D7AEFA
:102AA0000DA9224805F0C8FFD1E6CD781F2D28BF1B
:102AB0001F251F22002114A8A9F030FA2A4604F18C
:102AC0000C0114A8A9F0E0F9159B9A007FF5BFAEA0
:102AD000169B9B003FF5BBAE194822B0BDEC028BA4
:102AE000BDE8F04777F01EBB002E7FF4B0AE002C9F
:102AF0003FF4ADAE9FED106ADDED186A9DED197AD9
:102B0000DDED1A7A094866EE866A27EE067A67EEE8
:102B1000C67A10A9CDED106A8DED117ACDED127A3D
:102B200005F0D2F993E600BF50670020187C002022
:102B300000000000504700200000C842C46600208A
:102B4000C450002010B5074B93F9B82A40F6C5349D
:102B500040F6C513002A08BF1C4651F0A7F82043D1
:102B600010BD00BF5067002008B50648FEF77AFF89
:102B7000DFED057A20EE270AFDEEC07A17EE900A07
:102B800008BD00BF5027002000007A4410B504465D
:102B90000FF050FE204610BD08B54B69012B03D045
:102BA000BDE8084051F0E6B855F0BAFB024A0621EC
:102BB0004EF010FD032008BD44090C0810B50C4868
:102BC00090F8774E3CB155F0ABFB0A4A06214EF027
:102BD00001FD04200BE0A0F50050FEF713FF0028D4
:102BE000F7D00CF0A1FF01210CF048FE204610BDEB
:102BF000504700206C090C080E4B93F8A42DD20707
:102C000014D403F5805292F875267AB9B3F8A42D3E
:102C100002F4FF7252B993F8772E4AB993F8803DC7
:102C200013F0100F14BF03200120704705207047D8
:102C3000042070475047002010B588B00446002299
:102C4000134803A96FF000FFF8B1247C7BF046FA2B
:102C5000DDED037A9FED0F7A049067EE877A00230B
:102C6000FDEEE77A0593069317EE903AADF81C3027
:102C700000238322ADF81E301023CDE900328F21CE
:102C80000E2304AA20464FF0D9FC08B010BD00BFA7
:102C9000E44700200000C8420C207047014B93F825
:102CA000840D70475047002038B512212DED028B5E
:102CB00004464EF0C1FE20B90025BDEC028B28462B
:102CC00038BD072058F0E0FAB6EE008AF0EE487AF8
:102CD000E0EE087A4B49F7EE008A204638EEE70A24
:102CE00053F068F8122120464EF0A6FE0028E3D0EB
:102CF000062058F0C9FAF0EE487AE0EE087A424928
:102D0000204638EEE70A53F055F8122120464EF0DF
:102D100093FE0028D0D03D4D3D49D5F8B436002B68
:102D2000B8BF03339B1000EE103A2046B8EEC00A3D
:102D300053F040F8122120464EF07EFE0028BBD012
:102D40003B2058F0A1FAF0EE487AE0EE087A3149DB
:102D50002046B0EE670A53F02DF8122120464EF0BF
:102D60006BFE0028A8D03C2058F08EFAA0EE088A0E
:102D700029492046B0EE480A53F01CF8122120469B
:102D80004EF05AFE002897D005F2BC63234993ED1C
:102D9000000A204653F00EF8122120464EF04CFE59
:102DA000002889D095F8C0361D4900EE103A20461B
:102DB000B8EE400A52F0FEFF122120464EF03CFED3
:102DC00000283FF479AF95F8C136164900EE103A65
:102DD0002046B8EE400A52F0EDFF122120464EF098
:102DE0002BFE054600283FF467AF0F4BDFED0F7A4F
:102DF00093ED000A0E4980EE270A204652F0DAFFD2
:102E00005BE700BF88090C0890090C0850570020A8
:102E100097090C08A1090C08A9090C08B1090C08AC
:102E2000BB090C08C5090C08807D00200000C842C1
:102E3000CF090C08282938B5054614D0472908D0F1
:102E400027291BD112214EF0F7FD044630B900248A
:102E500002E0FFF729FF0124204638BD297C0948FC
:102E600047F0ECFEF8E716214EF0E6FD0446002898
:102E7000EDD0297C034847F0BBFFEDE7BDE83840C3
:102E800054F0B8BF08720020024B93F8800DC0F3D5
:102E9000001070475047002070B5254E2DED028B75
:102EA0000546D6F8980391ED018A036884B09B69C2
:102EB0000C46984750B9BDEEC88A18EE103ADB07A9
:102EC00004D4022004B0BDEC028B70BDD4E904012F
:102ED00020F000FC0028F4D068460FF055F96A464F
:102EE0002146284654F0C8FD0028EAD0114968461A
:102EF0000FF05EFA0028E4D10F48694605F052FD54
:102F000098B1D6F8980303689B69984708B10020E8
:102F1000D8E70A480222042103F002FB28B1064840
:102F2000694605F03FFD0028F1D10420CAE700BF43
:102F300050770020145E0020187C002050270020CD
:102F400008B502221021044803F0EAFA00280CBF59
:102F50000420002008BD00BF5027002008B5022231
:102F60000921044803F0DCFA00280CBF04200020EB
:102F700008BD00BF5027002013B5D1ED007AF5EE53
:102F8000C07AF1EE10FA0C4602DA022002B010BD4F
:102F90009FED187AF4EEC77AF1EE10FAF5D891EDBC
:102FA000030ADFED157AB0EEC07AB4EEE77AF1EEFF
:102FB00010FA18D5D4ED037A1048D4ED010A94ED37
:102FC000000AFCEEE77ACDED007AD4ED027A9DF8A6
:102FD0000020FDEEE77ACDED017A9DF9041004F0B2
:102FE000B3F80020D2E7F7EE000A20F00BF8002833
:102FF000CBD0DFE70000B44300000034DC7B0020CE
:1030000008B5D1ED017AF5EEC07AF1EE10FA08DDDF
:103010009FED050A054827EE800A75F08FFF002016
:1030200008BD0420FCE700BF0000C8428467002000
:1030300008B5084890F8773E0BB9042008BD022275
:103040000321A0F5005003F06BFA0028F5D0002012
:10305000F4E700BF5047002070B501F10C050E46A3
:103060000FCD86B06C460FC495E8030084E80300DA
:1030700096E80E00044806F0D3FE00280CBF04209A
:10308000002006B070BD00BF5027002030B48B8BED
:10309000B22B05460C4618D00AD8152B35D0732B09
:1030A00010D0112B2ED02146284630BC55F07EBFC3
:1030B000D12B0DD0B3F5967F0DD0C02BF3D130BC02
:1030C000FFF7EABE30BCFFF757BF30BCFFF798BF31
:1030D00030BCFFF7C1BFD1ED007A9FED0F7AF0EE63
:1030E000E77AF4EEC77AF1EE10FA11D5D1ED017A54
:1030F000F0EEE77AF4EEC77AF1EE10FA08D530BCBC
:10310000FFF796BF30BCFFF71BBF30BCFFF726BFF1
:10311000022030BC704700BF0000003470B52DEDB8
:10312000048B9FED2B0A9FED2B8A8CB004462A4816
:1031300022F026FC21EE081A2848267CBDEEC11A92
:1031400060EE888A11EE103A20EE089A1DB275F0F2
:10315000C3FD07EE900AF8EEE77A204867EE887A1A
:10316000FDEEE77A17EE903A1CB275F0A1FDDFEDA7
:103170001C7A1C4B8DED059A20EE080AB722B4EE9E
:10318000E70AF1EE10FA58BFB0EE670ABCEEC00ACB
:10319000D3ED007ACDED068A00230893099310EE53
:1031A000103A27EE888AADF82C301A23CDE9003288
:1031B0003E2105AA30468DED078AADF82850ADF8BE
:1031C0002A404FF03BFA0CB0BDEC048B70BD00BF41
:1031D0009F0CB3450AD7233C945F002084670020EE
:1031E00000FF7F47AC63002008B591ED007AF6EE52
:1031F000007AB4EEE77AF1EE10FA06DD0448012217
:103200000521FEF7A1FA002008BD0420FCE700BF5D
:10321000C85D0020002070470020704700207047E4
:103220000120704790F89C308B4286BF283150F8BF
:10323000210000207047000090F89C308B4286BF30
:10324000283150F82100002070470000FA20704714
:10325000014B93F8320170475047002038B50446BF
:10326000D0E90B30616B40F4E052226341F4E0524C
:10327000626343F4F842E2622B4A92F8845D023DB5
:103280000E2D0FD8DFE805F00808080E0E080E080E
:103290000E0E0E0E0E0E080040F4F84041F4F841F8
:1032A0002063616392F8811DC80708D543F4F84391
:1032B00043F00803E362236B43F008032363636B6B
:1032C00023F00803636392F8A81DC90744BF43F0C5
:1032D00008036363154B93F85033013B012B0BD864
:1032E000E36A43F48003E362236B43F480032363C4
:1032F000636B43F48003636392F89839DB0712D55C
:103300000B4B1868E36A43F48073E362236B43F466
:103310008073236338B1192142F05AFB18B1636BF3
:1033200043F48073636338BD50470020507700201A
:10333000787F002013B54FF44470CDE900210FF0E1
:1033400071FA044628B1DDE9002155F02BFA024B51
:103350002360204602B010BD540B0C0870470000DB
:103360000020704700207047002070470020704701
:103370000020704700207047002070477047000011
:103380000120704700F50550243070470048704711
:10339000FC2F0C0800F5005090F8840D70470000D9
:1033A0009C207047F0B52DED028B8FB00023009369
:1033B00000F580439FED4F8A93F9B83A044600F533
:1033C0000056002B00F08C8000F5954001226946E4
:1033D000383048F04BFB3322002101A8A8F09EFDB5
:1033E000A3238DF8043095238DF805307AF07EFE06
:1033F00004F5405505F5FB63CDF8070004F537509B
:10340000D3F8DC20D3F8E030CDF80B103030CDF815
:103410000F20CDF813304DF08BFC0346DFED360A5C
:1034200093ED000A9F20B7EE001A1FF0EDFE10EE9C
:10343000103ACDF8173006F6CC63B6EE061AF4EE65
:10344000000A05F5426793ED000A30201FF0DCFE0C
:1034500097EDD87ADFED297AC7EE277A04F55C502C
:1034600010EE103ACDF81B3017EE903ACDF81F3021
:1034700076F0CCFD20EE080A242210EE103ACDF8AA
:10348000233094F8813202FB034301A9D3F89C3224
:10349000CDF8273004F5AB43D3ED2C7AFDEEE77A77
:1034A000332217EE903AD7EDDE7AADF82B30FDEEF1
:1034B000E77AB6F89A39ADF82D30009BCDF82F3069
:1034C00017EE903A04F6A860ADF83330B5F8B03690
:1034D000ADF8353049F07AFF0FB0BDEC028BF0BD8E
:1034E00006F6A813D3ED007A67EE887ACDED007A60
:1034F00071E700BF0AD7233C000000000000C8426B
:103500001FB5044600F561509FED0B0A043022F010
:1035100037FA04F5885001A908308DED010ACDED88
:10352000020A8DED031A08F099F809F075FF04B04E
:10353000BDE8104009F0FEBCE02E65427FB50E46A6
:103540004FF6FF710446154607F0A0F9E0B11022CE
:1035500000216846A8F0E2FCA3238DF800309523F3
:103560008DF8013004238DF802307AF0BFFD10226F
:10357000CDF80300CDF8071004F6A86069468DF871
:103580000B60039549F0A2FF04B070BDF0B58BB09D
:10359000154606460F462422002101A81C46A8F025
:1035A000BDFCA3238DF8043095238DF80530062348
:1035B0008DF806307AF09AFD2B6804936B680593BA
:1035C000AB680693236807936368CDF80700CDF8CE
:1035D0000B1008932422A3688DF80F7001A906F63A
:1035E000A860099349F0F2FE0BB0F0BD10B500F5EC
:1035F0000053044693F8EC2093F8841D00F6A8606D
:103600004AF0A4F804F5885008300AF0E5F804F50B
:103610009070BDE8104016F06FBF000070470000CA
:1036200070B504460B4E56F0F5F90B4B2360502550
:10363000601956F07DFB66513035B5F5547FF7D1F2
:1036400004F5547057F07EFF2046044940F0DCFE3C
:10365000204670BDF0430C087C4F0C0804450C0854
:1036600030B50A4D0FCD8DB06C460FC40FCD0FC4D1
:1036700095E80F0084E80F0000220321684640F01F
:10368000A5FA57F0E1FC0DB030BD00BF58010C08A1
:1036900037B500F5045101223031044648F0CAFB29
:1036A00005212948002240F091FA41F0B3F8274A59
:1036B0001388204643F008031380FFF7D1FF17213A
:1036C000234841F087FAB6EE000A224841F098FA02
:1036D000012504F5FE510023183139201E4A0095BA
:1036E00040F078FA1D490B68D8070CD41C4B0D60CC
:1036F00004F5F05208321A6004F5FB520832DA6021
:1037000004F6BC729A6104F50750154903222C3067
:10371000012540F0B1FA134A0095002304F6A86190
:10372000162040F057FA104B1A68D20705D40F4AFA
:103730001D6004F58154103414600C48012103B05D
:10374000BDE8304040F0B4BAB4440C085C7F0020BF
:10375000FC430C08D8430C086C760D083C2700206D
:1037600000220020F0EF0C08402700202422002037
:1037700000207047002070470069C0F34010704778
:103780000F299DBF302303FB0100503000207047FC
:10379000002070470120704700F0CEBF01F016B93D
:1037A00000F052BC01F07ABB70B5234B036000F50A
:1037B00000530446D3F8140D204AC3F8582B08B11F
:1037C0000FF03CF81E4B236004F5805393F8A42DB2
:1037D00042B9D3F8A05D2DB128461BF06DFF2846F5
:1037E0000FF028F804F5805014306EF021FD04F637
:1037F000D87058F0D9FC04F6AC3504F64C36B54216
:1038000004D0183D28461BF0ADFBF8E70D4BC4F87B
:10381000903504F5DE604CF067FF04F2C4604CF0B4
:1038200063FF04F224604CF05FFF04F5BF604CF0CE
:103830005BFF204670BD00BF083E0C08F80A0D086B
:10384000CCE80C086CAA0C0838B54C4B044640F880
:10385000043B5BF051FC04F110000CF0F5FF04F1A7
:10386000680046F023FB04F5907016F04BFA04F55F
:103870001C700BF0E7FD04F565700EF0E1FF04F538
:10388000B2601CF0D1FF04F628305BF0BDFB04F6FB
:10389000F83041F075FF04F6A86049F0CBFC04F65F
:1038A000BC7061F0C3F804F6D87058F065FC04F5FC
:1038B000805014306EF0A8FC04F58150103046F0B2
:1038C000B7FE04F5845004305CF0F4FD04F5805339
:1038D00000252B4A83F8A85004F5855004F585533C
:1038E0000833183013603CF095FD04F588502946E4
:1038F000083008F0C9F804F5BB50103068F030FE0D
:1039000004F5E15014306BF0B9FC04F5EA500C30CA
:103910006DF0D4FD04F5ED5010306EF009FA04F5A9
:10392000F050083007F040F804F5FB50083069F01B
:1039300075FA144904F5FE5040F066FD04F5FE509A
:10394000183061F0E5FB04F5025014306EF074FF9E
:1039500004F5005304F5045083F8EC500A4D04308C
:103960006FF0B8F82B6813B108487AF085FB204651
:10397000074940F049FD2C60204638BDCCE80C08D2
:1039800080880020887B0D08B07F0020984F0C08AD
:10399000E4E70C0810B504465A3076F043FB04F116
:1039A0005C0076F03FFB04F15E0076F03BFB04F137
:1039B000600076F037FB04F1620076F033FB04F12F
:1039C000640076F02FFB04F1660076F02BFB04F127
:1039D000680076F027FB04F16A0076F023FB04F11F
:1039E0006C0076F01FFB04F16E0076F01BFB04F117
:1039F000700076F017FB04F1720076F013FB04F10F
:103A0000740076F00FFB04F1760076F00BFB04F106
:103A1000780076F007FB04F17A0076F003FB04F1FE
:103A20007C0076F0FFFA04F17E0076F0FBFA04F1F8
:103A3000800076F0F7FA04F1820076F0F3FA04F1F0
:103A4000840076F0EFFA04F1860076F0EBFA04F1E8
:103A5000880076F0E7FA04F18A0076F0E3FA04F1E0
:103A60008C0076F0DFFA04F18E0076F0DBFA04F1D8
:103A7000900076F0D7FA04F1920076F0D3FA04F1D0
:103A8000940076F0CFFA04F1960076F0CBFA04F1C8
:103A9000980076F0C7FA204610BD00002DE9F04FDF
:103AA000044685B0FFF7D0FEBE4B236004F50450FA
:103AB0003030FFF76FFF04F507502C3004F5005548
:103AC000FFF7AEFD04F52550343076F0CDFA95F8C9
:103AD000983923F0030385F8983905F6A4134FF0BD
:103AE00000080026A5F89A89C5F89C89C5F8A08920
:103AF0001E6005F6A81304F526501E602C304DF00C
:103B000013F904F52650383057F048FFA64BC5F896
:103B10003C3AA64BC5F8443A04F52950A44BC5F8E5
:103B20004C3AC5F8384AC5F8404AC5F8484A2030EA
:103B30000EF02AFB04F529503C300EF025FB04F56D
:103B40002A5018300EF020FB4FF6FF79994BC5F83C
:103B5000AC3A04F52857A5F8B09A07F1B4000EF076
:103B600013FB1C37944B95491F604FF0FF3B3846C1
:103B7000C5F810BB40F048FC04F52C50A5F8749A29
:103B8000A5F858BA14303EF00BF8C5F8548B04F57C
:103B90002D588B4BC5F8583B08F1180808F1140054
:103BA00079F0CEF904F5045A04F52E5704F52F598F
:103BB0000AF12C0A103709F134093846143751F04C
:103BC00003FF4F45F9D10723C5F8183D0023A5F899
:103BD0001C3D4FF4CB700EF02BFEC5F8140D04F510
:103BE0003450203079F0ACF904F53550243079F0B8
:103BF000A7F9744B1A680AB9C3F80080724BC5F86C
:103C0000583B04F53659132309F12C0985F8843DF6
:103C10004FF4C871484678F067FB6C4BC5F8AC3D73
:103C20006B4B04F5405BCBE91B336A4B1F6817B144
:103C300069487AF021FAC3F80090684BC5F8AC3DAA
:103C400005F6AC534FF07E52C3F83823C3F83C63FB
:103C50006349484640F0D8FB624B0393624B0093A4
:103C6000029404AB04F5445013E90C004FF40071C6
:103C700004300CF009F904F5595038306EF0D8FFD3
:103C80005A4BCBF8783604F55B508BF8C17604308C
:103C90000EF07AFA01238BF8D4360BF5DB6304F5CA
:103CA0005C581E605E609E600BF20C73C8F800608A
:103CB000C8F80460C8F8086004F588511E605E60AA
:103CC0009E6046461C3608319FED490ACBF818170E
:103CD0003A46304604F55F5B07F062FE0BF1180BC5
:103CE000524604F5705A0AF1200A31464B465846AE
:103CF00070F0E6FC31464B464246CDF800B05046E7
:103D000072F03EFF04F58040324653464146CDF8FE
:103D100000B0343075F004F804F591403246534653
:103D20004146CDF800B0783075F07EFE04F5924043
:103D3000534632464146483074F08AFC04F59340BD
:103D40004FF4004120300CF081FE04F59440203007
:103D500058F02AFB04F59540243041F0DDFA04F5D3
:103D60009540383004F5A04647F032FD2C22394604
:103D700006F55570A8F0D2F81E4B1F4A1A6004F5DC
:103D8000A7414FF0140CB8B20CFB002301371B7C89
:103D9000002BF8D1194B1880194B1F68A7B319488D
:103DA00047E700BF083E0C08993701089D37010816
:103DB000A13701080000FFFFA07E0020C8B70C0853
:103DC000F80A0D08F4820020300C0C0848A00D08F9
:103DD000B4220D0838900020AC4F0C08E09E0D086E
:103DE000E89D0D08A537010830090C0808040C08E7
:103DF000000000006C7F002064450C086A7F0020F2
:103E0000287F0020CE4F0C0804F5A7401C30C6E9DF
:103E1000E477C6F89803196002F0E8FA304BC6F868
:103E20009C3304F5A740583002F0E0FA2D4BC6F859
:103E3000D83304F5A840143002F0D8FA2A4BC6F85B
:103E4000143404F5A840503002F0D0FA274BC6F8DD
:103E5000503404F5A9400C3002F0C8FA244BC6F8DF
:103E60008C3404F5A940483002F0C0FA214BC6F862
:103E7000C83404F5AA40043002F0B8FA1E4BC6F864
:103E8000043504F5AA40403002F0B0FA1B4BC6F8E6
:103E9000403504F5AA407C3002F0A8FA184BC6F869
:103EA0007C3504F5AB40383002F0A0FA154BC6F86B
:103EB000B83504F5AB40743005F096FCA6F83C76B6
:103EC00095F8A43D43F0010385F8A43D0E4B1A6814
:103ED0000AB10E48ADE620461C6005B0BDE8F08F83
:103EE000A8550C0864570C0850530C08A4530C0830
:103EF000B8540C0858550C0810570C0808550C08F5
:103F0000B4570C08C0560C0844270020E94F0C0891
:103F100010B579F0F5FB064C064B18602046FFF70C
:103F2000BDFD2046044A0549BDE81040A5F0B4BADD
:103F3000502700204827002080DD0020A9370108F5
:103F400030B5044689B0684604F588550EF01CF972
:103F5000083504A80EF018F96946284609F00AF851
:103F600060B104A9284609F049F838B1059B0193CE
:103F700023680022DB6C69462046984709B030BDB3
:103F800000F5805292F88423D20709D400F500523C
:103F900092F8771E09B1FFF7D3BF03689B6C1847EF
:103FA0007047000010B586B0044602A801910EF0DB
:103FB000EBF804F5885002A9083008F0DBFFC0B127
:103FC00094F88132DDED037A9FED0B7A019A24217A
:103FD00001FB0343D3EDA76A2368F8EEE77ADB6CB5
:103FE000E6EEC77A02A92046FDEEE77ACDED037A28
:103FF000984706B010BD00BF0000C842F0B50446A7
:1040000085B004F58856684608360F4615460EF00A
:10401000BBF86946304608F0F1FF10B9002005B042
:10402000F0BD3946304608F089FE0028F6D0002D54
:10403000F5D004F58054284694F8843343F0020305
:1040400084F88433EBE7000010B50A4A137804467D
:1040500000F5A94043F080030C30137003F074FAAC
:1040600030B920460822BDE81040022102F058BABB
:1040700010BD00BFEC7E00202DE9F04101F10803E6
:1040800005460F460FCB88B004AC84E80F0005F559
:104090004056134301BFD6F8CC360693D6F8D03637
:1040A0000793059BB3B920460EF09EF805F55B58C3
:1040B00008F10408014603AA40460EF0A1F8C0B179
:1040C0000399019120460EF08FF80199024620468F
:1040D0000EF060F80023C6F8F830BB88A6F8F6307A
:1040E00005F5A94021460C3002F00AFF08B0BDE8F2
:1040F000F081D6F8C81601914046E4E770B58CB05F
:104100000D4604AC064620460EF03EF82B691F49CA
:104110000BB96B693BB300230B7005F108010FC9A4
:1041200084E80F0006F55B5003AA032104300EF06B
:1041300067F890B108AA032120460EF061F860B13B
:104140000399032220460EF025F806F5A9402146E2
:104150000C3002F0D5FE0CB070BD06F540530122C4
:10416000D3F8C816EEE701220A7006F54051009216
:1041700008ADD1F8D026D1F8CC1628460EF024F898
:1041800095E80F0084E80F00DFE700BF907D002076
:1041900000F59B5100F5A94014310C3002F0B0BE7F
:1041A00070B5083105460FC98EB006AC84E80F0023
:1041B000134312D105F58040002303A93430039343
:1041C0000493059374F026FE022203A90AA80EF0B8
:1041D000CFFA0C9B08930D9B0993079BABB9204624
:1041E0000EF002F805F55B56043601460AAA304681
:1041F0000EF006F888B10A99019120460DF0F4FFFF
:104200000199024620460DF0C5FF05F5A94021465B
:104210000C3002F075FE0EB070BD05F5405330460F
:10422000D3F8C8160191E9E7F0B501F10803054696
:104230000E460FCB89B004AC84E80F00134307D1BE
:1042400005F54053D3F8CC26D3F8D0360692079321
:10425000059BABB920460DF0C7FF05F55B5704374A
:10426000014603AA38460DF0CBFF08B3039901912C
:1042700020460DF0B9FF0199024620460DF08AFF55
:10428000327EB388D2074FEA132344BF03EB830384
:104290005B00327A07EE903A05F5A940B8EE670A5E
:1042A000C2F3400221460C3002F06EFE09B0F0BDB0
:1042B00005F540533846D3F8C81601910DF094FF28
:1042C0000199024620460DF065FF4AF077F8022278
:1042D000152149F02BFED3E738B504460D46FFF70C
:1042E0005FFF04F540500023C0F8F830AB88A0F819
:1042F000F63038BD10B58B8853B100F5A9440C34A5
:10430000204604F089FA2046BDE8104003F08ABA3E
:1043100010BD000073B505460C4679F0DFFE05F5CB
:104320004056C6F80001D4ED027AF5EEC07AF1EEFF
:1043300010FA17DD9FED137A67EE877AFCEEE77AC5
:10434000C6ED3F7AD6F8FC2005F52D504FF47A7370
:10435000B2FBF3F30C4A0621183002B0BDE87040FE
:104360004DF038B960F07EFE0023009394F90D20E3
:1043700094F90E3094F90C1060F010FEC6F8FC00B1
:10438000E0E700BF00007A448C500C08DFED0B7AA8
:1043900091ED041AD1ED030A91ED020A8B8800F524
:1043A000A9404FF47A7121EE271A60EEA70A20EE99
:1043B000270A5943483004F023BA00BF0000C8421E
:1043C000F8B500F58043054693F8384014F0010431
:1043D0000F4602D100242046F8BD124A537800F55A
:1043E000405643F001035370D6F8F8301BB979F00A
:1043F00075FEC6F8F80079F071FED6F8F830C01AEC
:104400004FF47A73B0FBF3F0B6F8F6309842E1D38C
:1044100005F52D503B88044A062118304DF0DAF896
:10442000D9E700BFEC7E00209C500C08F0B5144E7C
:10443000357887B0044625B1012D1AD0012007B088
:10444000F0BD00F5804393F8382012F00100F6D05B
:1044500001270097D1E904122B4602A80DF0B4FE03
:1044600004F5A9400C3002A902F04AFD3770284635
:10447000E5E700F5804494F8380000F00100DEE73D
:10448000907D002010B500F58043044693F8383045
:1044900013F0010017D004F54054D4F8F8301BB9DC
:1044A00079F01CFEC4F8F80079F018FED4F8F83062
:1044B000C01A4FF47A73B0FBF3F0B4F8F6309842B8
:1044C00034BF0020012010BD7FB500F5A043054694
:1044D00093F83C36012B0C4634D100F5804393F819
:1044E000380010F001002BD001AE0023314604F15A
:1044F00008000193029303930EF008F8DDED037AB0
:104500009FED1F7AF0EEE77AF4EEC77AF1EE10FA3B
:1045100005D505F55C5075F079FD8DED030A23692D
:1045200043B9636933B905F55C5075F06DFD03C897
:1045300086E8030005F5A9400C3002F00FFD0020CD
:1045400004B070BD0B79DFED0F6A07EE903A0B7E79
:104550009B070D4B48BF9FED0D7A93ED006AF8EE77
:10456000677A48BF67EE877A86EE267AB0EEC77A1A
:10457000B4EEE77AF1EE10FAACBF01200020DFE7DD
:1045800000000034DB0FC940D07000200000803BE9
:104590008B8823B100F5A9400C3004F04FB90120FD
:1045A0007047000010B5044679F098FD04F54053BB
:1045B000D3F80021801AD3F8FC2090424FF000007D
:1045C00084BFC3F8FC00012010BD000038B50446CC
:1045D0000D4679F083FD04F540539FED077AC3F84B
:1045E000FC06D5ED027A67EE877AFDEEE77A17EEE4
:1045F000902AC3F8F82638BD00007A440B464A7C5E
:10460000D3ED030A91F9101093ED020A014802F06C
:104610009BBD00BFDC7B002010B5044679F05EFD39
:1046200004F54053D3F8FC26801AD3F8F82622EA82
:10463000E27290424FF0000084BFC3F8F8060120F8
:1046400010BD000038B500F54055044695F8D43645
:10465000032B03D00A48032103F068FB04F58054C0
:10466000D5F8EC36D4F80803C01A1EF097FD0028E0
:10467000B8BF4042C828CCBF0020012038BD00BFD1
:10468000DC7B002008B500F5005393F8843D042B33
:1046900007D0032B0AD100F5A04393F83C36032B37
:1046A00004D14B88102B03D0732B07D0002008E0D7
:1046B000BDE808400348083104F074B9FFF79EFFD5
:1046C000012008BD187C0020D1F8093007EE903A8F
:1046D000F5EEC07AF1EE10FA08DD9FED050A00F55F
:1046E000804027EE800A343074F028BC704700BF49
:1046F0000000C8428B88012B036805D00A6932B9D3
:104700004A6922B9CA6812B99B6C00211847DB6C50
:10471000002208311847000000F5804300F594405E
:1047200091ED041AD1ED020A91ED030A93F8991A5A
:104730000022203057F0A4BE37B501F10805044629
:10474000284601910DF050FD012801990BD1CB684D
:10475000002B11DD514A04F52D50042118304CF086
:1047600039FF00206BE0032804D1CB68002B03DA6B
:104770004B4AF0E74B4AEEE74B88702B74D01CD8BD
:10478000152B12D80F2B07D804F52D50464A0421BB
:1047900018304CF01FFFE4E7113B2046042B4BD8A8
:1047A000DFE803F055585B524F005C2B58D05D2B6F
:1047B000EAD12046FFF7AEFD40E0B32B60D014D81D
:1047C000732B55D0B22B57D0722BDDD1D1ED027A9D
:1047D0009FED367A67EE877A04F54054FDEEE77A6E
:1047E00017EE903AC4F8F83628E0CD2B1ED8C22B2D
:1047F000CAD9A3F1C3020A2AC6D801A050F822F0F0
:104800008948010889470108894801088947010842
:104810008947010889470108894801088947010833
:10482000894701088947010893480108DE2BABD16D
:104830002046FFF7ABFD01E0FFF71EFC012003B0AF
:1048400030BDFFF75BFCF9E7FFF7A2FCF6E7FFF7E7
:10485000A7FCF3E7FFF7E8FCF0E7FFF73DFDEDE726
:104860002046FFF747FDE9E72046FFF7AFFEE5E703
:104870002046FFF7C3FEE1E72046FFF725FFDDE70F
:104880002046FFF737FFD9E70948294602F0D0FC58
:10489000D4E72046FFF740FFD0E700BFB0500C0838
:1048A000D0500C08F3500C0801510C080000C8420D
:1048B000DC7B002010B5044604F5405400F5804030
:1048C000343074F0F5F9D4F8F83623EAE37307EEE0
:1048D000903AF8EEE77A0020B4EEE70AF1EE10FA2B
:1048E00044BFC4F8F806012010BD000010B54B8885
:1048F000152B04460A4615D80F2B1AD9113B042B49
:1049000035D8DFE803F05E454A3E3900A3F1C30223
:104910000B2A0ED8DFE802F0260D260D0D0D260D10
:104920000D0D2626702B44D00BD85C2B39D05D2B77
:104930003BD004F52D50244A042118304CF04AFE97
:1049400010E0732B39D005D8722BF2D1BDE810409E
:10495000FFF7B0BFCE2B07D8C22BD7D8A3F1B20236
:10496000012AE6D8012012E0DE2BFBD0E1E7BDE80A
:1049700010401146FFF724BDBDE810401146FFF777
:1049800055BD00F5804494F8380000F0010010BDDA
:10499000BDE810401146FFF797BDBDE81040FFF796
:1049A00071BDBDE81040FFF7F3BDBDE81040FFF753
:1049B000F9BDBDE81040FFF72FBEBDE81040FFF77E
:1049C00041BE0020E3E700BF18510C0870B500F5A8
:1049D0000053054693F8843D032B0E4602D0002475
:1049E000204670BDFFF782FF04460028F7D005F58A
:1049F0002D503188183050F0C9FFF1E708B5044B4D
:104A000001221A7079F05EFB024B186008BD00BFEE
:104A1000927D0020987D0020014B00221A70704783
:104A2000927D002038B500F50054054694F94631D2
:104A3000B3B179F053FBD4ED527A95EDA57A194BC9
:104A4000F8EEE77AF4EEC77AF1EE10FA09DD1860B5
:104A5000154B186094F8A43D6FF3451384F8A43DFA
:104A600038BD1B6803F5FA6383423EBF94F8A43D4A
:104A700043F0200384F8A43D94F8A43D9B06EFD5B1
:104A8000094A136803F5EA4330338342E8D21060E1
:104A900005F52D50054ABDE83840042118304CF08A
:104AA00099BD00BFA47D0020A87D002034510C08D2
:104AB00038B500F50054054694F94731C3B179F093
:104AC0000DFB94F94C3195EDA67A07EE903AF8EE8D
:104AD000E77A184BF4EEC77AF1EE10FA09DD1860A8
:104AE000154B186094F8A43D6FF3861384F8A43D29
:104AF00038BD1B6803F5FA6383423EBF94F8A43DBA
:104B000043F0400384F8A43D94F8A43D5B06EFD540
:104B1000094A136803F5EA4330338342E8D2106050
:104B200005F52D50054ABDE83840042118304CF0F9
:104B300051BD00BFAC7D0020B07D002050510C085D
:104B400070B500F50054284E94F88639054613B127
:104B500094F9443193B994F8A43DD90605D549F0A8
:104B60002DFC00221B2149F0E1F994F8A43D00221C
:104B700062F30413F27484F8A43D70BD0123F3744E
:104B800079F0ACFAD4F8883D03F59C432033834296
:104B900008D2C4F8880D05F52D50144A02211830AA
:104BA0004CF018FD94F8A43DDA06E6D443F0100367
:104BB00084F8A43D49F002FC01221B2149F0B6F91A
:104BC00094F8A43DDB06D8D594F94431022BD4D116
:104BD00094F8773E002BD0D028461D22BDE87040C7
:104BE000092101F09DBC00BFCD7E002070510C0852
:104BF00038B504460D4679F071FA04F500533DB915
:104C0000D3F8942DC3F8980D0AB9C3F8940D38BDA4
:104C1000D3F8982D801A642882BF0022C3F8982DFB
:104C2000C3F8942DF3E70000F8B5044679F04AFA8A
:104C3000294BB4F8BE201988284E914205460ED063
:104C40001A80274B18603378A3B10024347049F0E0
:104C5000B5FB22461321BDE8F84049F067B9337827
:104C6000204FD3B93B782BB11D4B1F4A1B68C31A89
:104C7000934200D8F8BD0123337004F5005393F834
:104C8000773E23B104F536502C3075F0F9FA49F02F
:104C900095FB0122132149F049F93B78002BE9D01B
:104CA0003378002BE6D00E4A10491368EB1A8B427A
:104CB000E0D904F50053156093F8773E002BD9D066
:104CC00004F536542C342046002176F039FA20467B
:104CD000BDE8F84077F00ABE947D0020917D002069
:104CE000987D0020927D002080841E0040420F00AD
:104CF00038B500F50054054694F8813DD80714D521
:104D000094F8A81D94F8A53DC90703F001020DD53C
:104D10005AB149F053FB00221A2149F007F994F8DF
:104D2000A53D6FF3000384F8A53D38BD002AFCD1F2
:104D300043F0010305F52D5084F8A53D144A0221E6
:104D400018304CF047FC49F039FB03221A2149F096
:104D5000EDF894F8843D022B0FD11C221321284634
:104D600001F0DEFB0028E0D105F559500122BDE835
:104D7000384017213830FCF7E7BC092BEDD0054B44
:104D8000D3F8980303689B6898470028E5D1CCE7DF
:104D900080510C0850770020F0B500F500543C4ECF
:104DA00094F968718BB0054667B979F097F994F872
:104DB000A43D306067F3820384F8A43D354BDF7374
:104DC0000BB0F0BD002307930893099307AF05AB21
:104DD00000F58850019303AA04AB06A90097083098
:104DE00008F032F8384621F0C9F9D4ED5B7AF4EED8
:104DF000C07AF1EE10FA13DD9DED067AF4EEC77A73
:104E0000F1EE10FA0CDD79F069F994F8A43D306008
:104E10006FF3820384F8A43D1E4B0022DA73CFE7C0
:104E200079F05CF9336803F5FA63984294F8A43D8D
:104E3000EED35A07C4D443F0040384F8A43D154BC1
:104E40000122DA7349F0BAFA0222102149F06EF811
:104E500079F044F9D4F8A03D03F59C4320339842FF
:104E60000AD979F03BF9C4F8A00D05F52D500A4A8E
:104E7000042118304CF0AEFB94F96831022B9FD11D
:104E800005F55950012218213830FCF75DFC97E7F1
:104E90009C7D0020CD7E002094510C0838B515462D
:104EA000044649F08BFA0122062149F03FF8022D11
:104EB00008D0032D0FD120460422BDE83840092137
:104EC00001F02EBB04F559500122BDE838400721FE
:104ED0003830FCF739BC38BD38B500F5005405460C
:104EE00094F94E3133B994F8A43D6FF3000384F87C
:104EF000A43D38BD79F0F2F8D4F8903D9FED1B7ACF
:104F0000D4ED546A07EE903AF8EE677AE6EE877AC7
:104F100007EE100AB8EE477AB4EEE77AF1EE10FA2F
:104F2000E1D494F8A43DDA07E3D443F0010384F814
:104F3000A43D49F043FA01221C2148F0F7FF05F592
:104F40002D500B4A022118304CF044FB284600F04B
:104F50005FFB94F94E31022BCBD105F5595001225C
:104F6000BDE838401D213830FCF7EEBB00007A4424
:104F70009C510C08F8B500F50054054694F94531EC
:104F800053B3D4F8107D3FB379F0A8F894ED550AE7
:104F9000DFED3A7A9FED3A1ADFED3A0A064620EE47
:104FA000270A4FF4A2701EF02FF9BCEEC00AF71BBF
:104FB00010EE103A9F4210D294F8A43D990705D5FF
:104FC00049F0FCF90022082148F0B0FF94F8A43D14
:104FD0006FF3410384F8A43DF8BDD4F88C3D47F24B
:104FE0003052F31A93420AD905F52D50B4F93431F1
:104FF000254AC4F88C6D042118304CF0EBFA94F873
:10500000A43D9A07E8D494F8772E002AE4D043F020
:10501000020384F8A43D49F0D1F90122082148F0A7
:1050200085FF94F94531022B08D10122122105F5A3
:1050300059503830BDE8F840FCF786BB032B0DD142
:1050400094F8773E002BC7D005220221284601F0B4
:1050500067FA0028C0D101221A21E8E7042BBBD14E
:1050600094F8773E002BB7D005220921284601F09D
:1050700057FA0028B0D101221921D8E700007A445C
:105080000000804F00000000B0510C0838B5054604
:1050900005F5005479F022F894F8772E294B12B1D7
:1050A00094F969213AB9186094F8A43D6FF3C713D5
:1050B00084F8A43D38BD94F8842D012AF3D0132A36
:1050C000F1D005F55F529FED207AD2ED3C7A67EE84
:1050D000877AB3EE0E7AF4EEC77AF1EE10FAE2D9DF
:1050E0001B6803F5FA638342E4D8D4F89C3D03F5CA
:1050F0009C432033834208D2C4F89C0D05F52D5003
:10510000124A042118304CF065FA94F9A43D002BA2
:10511000D0DB94F8A43D43F0800384F8A43D49F02B
:105120004DF901220C2148F001FF94F96931022B5D
:10513000C0D105F559500122BDE838400C21383066
:10514000FCF702BBA07D0020E02E6542CC510C088C
:1051500010B500F50053044693F94D31012B0AD0E8
:10516000022B18D000F55950BDE81040012215213E
:105170003830FCF7E9BA0B22102101F0D1F920B93F
:105180000B220221204601F0CBF9044A137843F0A8
:105190000803137010BD0B220921F4E7EC7E0020F8
:1051A00038B500F50055044695F8A43D43F00803D2
:1051B00085F8A43D49F002F90122172148F0B6FE16
:1051C00095F89839DB0704D42046BDE83840FFF74E
:1051D000BFBF034802F062F80028F5D038BD00BF19
:1051E000DC7B002070B500F50055064695F8843D3F
:1051F000D5F8984DD5F8942D033B012B18D8A41A57
:10520000B4F57A7F94BF0024012495F8A43DC3F33C
:10521000C003A3421AD06CB106F52D5018300C4AC9
:1052200002214CF0D7F93046BDE87040FFF7B8BF17
:105230000024EAE749F0C2F82246172148F076FE3A
:1052400095F8A43D64F3C30385F8A43D70BD00BF89
:10525000DC510C0813B500F5005393F8773EA3B169
:1052600000F500500021047D094860F0C5FB0246AE
:1052700048B1019249F0A2F8019A092102B0BDE8B3
:10528000104048F053BE002CF3D102B010BD00BF57
:105290002847002030B500F55C5587B00446002152
:1052A000284674F053FE02A80CF06EFF04F58850F7
:1052B00002A904F54054083007F05CFE049BC4F8D2
:1052C000CC36059BC4F8D036284674F091FE830690
:1052D00011D5284674F09AFEBDEEC00A284610EE9D
:1052E000103AC4F8C83674F099FEBDEEC00A10EE4C
:1052F000103AA4F8B03607B030BD0000024B0146AA
:105300001868026812681047FC82002001225BF0D6
:1053100097BA000000225BF093BA00001F2900F248
:105320008D80DFE801F08B1014181C2024282C300D
:1053300034383C4044484C5054585C6064686C704D
:1053400074787B7F838700F506500C30704700F53A
:1053500006500E30704700F506501030704700F5CB
:1053600006501230704700F506501430704700F5B3
:1053700006501630704700F506501830704700F59B
:1053800006501A30704700F506501C30704700F583
:1053900006501E30704700F506502030704700F56B
:1053A00006502230704700F506502430704700F553
:1053B00006502630704700F506502830704700F53B
:1053C00006502A30704700F506502C30704700F523
:1053D00006502E30704700F506503030704700F50B
:1053E00006503230704700F506503430704700F5F3
:1053F00006503630704700F506503830704700F5DB
:1054000006503A30704700F506503C30704700F5C2
:1054100006503E30704700F50750704700F50750C2
:105420000230704700F507500430704700F5075010
:105430000630704700F507500830704700F50650F9
:105440000A30704710B50446FFF768FF114674F044
:10545000F3FD6B280AD8672809D8512812D84F289D
:1054600031D8A0F14C03DBB2012B20D910BDA0F143
:10547000690304F584500430022B0ED8DFE803F0F2
:1054800011131500A0F15403DBB2012BEED8114B20
:105490001B680B21B3F8CC200EE00021FFF73AFF88
:1054A000E4E70121FAE70221F8E70321F6E7094BD7
:1054B0001B68B3F8A420092104F585500830BDE825
:1054C00010405BF02DBA034B1B680A21B3F8B820DB
:1054D000F2E700BF58830020F0B50F4B89B06A4651
:1054E000064603F12007144618685968154603C597
:1054F0000833BB422A46F7D10025E9B23046FFF710
:105500000DFF0135627814F8021B74F09BFD102D1D
:10551000F3D109B0F0BD00BF88010C0837B50446CF
:10552000FFF7DAFF0820FFF7E9FE354B42891A80C2
:105530000920FFF7E3FE334B42891A8004F500553A
:1055400001221321204600F0EBFF95F98031002B5A
:1055500008DC01230DF1070104F506508DF8073032
:105560003FF0E4FD95F9802195ED5D0A95ED5E1A19
:10557000D5ED5F0A012A04F540540FD0DFED227A01
:1055800031EE277AB4EEC07AF1EE10FA1CDD70EE3F
:10559000E77AF4EEC07AF1EE10FA15D52D201DF061
:1055A00033FE04F2BC6383ED000A04F2BC64DFED59
:1055B000170A94ED000A3320B7EE001A1DF024FEFE
:1055C00084ED000A03B030BD02EBD2735B10013BE7
:1055D0005BB207EE903A013A31EE601AF8EEE77AE4
:1055E00007EE102A67EE817AB8EEC77A04F2BC6142
:1055F000C7EE876A76EEA00AC1ED000AD5E700BFC4
:10560000382200203A2200200AD7233CCDCCCC3DC2
:1056100038B578F063FD00240546E0B22A4640F232
:10562000DC51013454F09AFA062CF6D1024A0023D8
:105630001380024A138038BDC67D0020C47D00203F
:10564000054A00231380054A00F540501380044AA0
:1056500080F8C03613807047B87D0020BA7D0020E6
:10566000BC7D0020F0B585B01D460446FFF756FE10
:10567000114674F0E1FC0238692800F2CB80DFE8C3
:1056800010F06A0079008300890091009400A30063
:1056900097009D009A00A000A600C900C900C9009B
:1056A000C900C900C900C900A900C300C600C900DB
:1056B000CB00E600E800C900C900C900EA002601E5
:1056C0004F017901A501BE01C900C900C900C90087
:1056D000D70121029502EA02F7020003090312032F
:1056E000A904C90078036203690389037F03810366
:1056F00095038B038D03C900A303BA03C503E0031D
:10570000ED03F2032D0438044F045C0461047504B6
:1057100080049704A404C503E003CA03E503380426
:105720004F043D0454048004970485049C04C9007C
:10573000C900C900C900C900C900C900C900C90021
:10574000C900C900C900C900A103970399037503E3
:10575000860392039E0304F5595004F50054012278
:1057600094F8773E383011464BB105B0BDE8F040B3
:10577000FBF7EABF012204F559501146383005B055
:10578000BDE8F040FBF758BF012204F5595011461F
:105790003830EAE701221321204605B0BDE8F04089
:1057A00000F0BEBE01220021F6E701220221F3E74C
:1057B00001220321F0E701220421EDE70122072164
:1057C000EAE701221146E7E701221021E4E701227E
:1057D0001521E1E79FEDA91A04F5944504F58044ED
:1057E000203594F8991A28460022F0EE410AB0EECE
:1057F000410A56F045FE94F8991A0322284605B04E
:10580000BDE8F04056F028BE9D4B9E4A01E09C4BFF
:105810009D4A1A6005B0F0BD002DFBD19B4A13785C
:1058200004F52D5083F0010313701830984A4BB1E2
:1058300040F26C731380974A062105B0BDE8F04032
:105840004BF0C8BE40F24C431380934AF4E7934BAD
:10585000DBE7924BDCE7002DDCD10820FFF74EFDA3
:10586000C78946898E4D07EE907A04F50050B8EE50
:10587000671AB0F988218B4C07EE906ABB1B93FB2B
:10588000F2F32A78F8EE670A9BB2CAB1B4F90020A5
:10589000D31800EE103AF120B8EEC00A1DF0B4FCA7
:1058A000BDEEC00A10EE103A2380B4F900309F42DA
:1058B00001DD9E42AEDB2B7883F001032B70A9E75C
:1058C000B4F90020D31A00EE103AF320E4E7002DDB
:1058D000A0D10820FFF712FD4289C18904F50050CC
:1058E000704CB0F988018B1A93FBF0F3B4F9000007
:1058F00010FA83F300EE103A4FF4807007EE901A1E
:10590000B8EE671A07EE902AF8EE670AB8EEC00AFA
:105910001DF07AFCBDEEC00A10EE103A238079E744
:10592000002D7FF477AF0820FFF7E8FC5D4D41893B
:10593000C689B5F9002004F50050731AB0F9880142
:1059400093FBF0F39BB2D31A00EE103A40F2091029
:1059500007EE906AB8EE671A07EE901AB8EEC00A22
:10596000F8EE670A1DF050FCBDEEC00A10EE103ACA
:105970002B804FE7002D7FF44DAF0920FFF7BEFCD1
:10598000C7894689484D07EE907A04F50050B8EE75
:10599000671AB0F98821454C07EE906ABB1B93FB50
:1059A000F2F32A78F8EE670A9BB23AB1B4F9002014
:1059B000D31800EE103A4FF48A706DE7B4F9002066
:1059C000D31A00EE103A4FF48B7065E7002D7FF488
:1059D00021AF0920FFF792FC4289C18904F50050EC
:1059E000324CB0F988018B1A93FBF0F3B4F9000044
:1059F00010FA83F300EE103A40F223107EE7002DF8
:105A00007FF408AF0920FFF779FC284D4189C6894A
:105A1000B5F9002004F50050731AB0F9880193FB22
:105A2000F0F39BB2D31A00EE103A4FF496708FE762
:105A3000002D7FF4EFAE1E4A137883F00103002B94
:105A4000F6EE007AB7EE007A0CBF17EE100A17EEEA
:105A5000900A137004F55A5304F52D54D863FAF7DD
:105A600053FD0022134BFAF7A7FDCDE90001124ABE
:105A70001834062120464BF0ADFDCBE600000000B7
:105A80003C2200200080ED4400808944C87D002035
:105A900030220020F8510C080F520C08342200204C
:105AA0004022002038220020412200203A220020FB
:105AB000C97D00200000594026520C08CDCC4C3F37
:105AC000CDCCCC3D002D7FF4A5AE04F500551FEDE7
:105AD000051A5FED050A95ED5F0A4FF49F701DF002
:105AE00093FB04F5055003A93C308DED030A3FF00C
:105AF000B3FAD5ED5F0A95ED5E0AB7EE001A40F2F3
:105B00003F101DF081FB04F5055003A938308DEDE1
:105B1000030A3FF0A1FA0A22012195F980011DF044
:105B2000B1FB03A98DF80C0004F506503FF0FEFA16
:105B300095F98031012B04F540560ED140F2431007
:105B400095ED5E1AD5ED5F0A95ED5D0A1DF05CFBE3
:105B500006F2BC6383ED000A18E0013B95ED5E1A86
:105B6000D5ED5F0A07EE903A31EE607AF8EEE77A0B
:105B700006F2BC6587EE270A40F24510D5ED007AA3
:105B800030EE270A1DF040FB85ED000A06F2BC66E8
:105B900004F52D543068FAF7B7FC0022BC4BFAF735
:105BA0000BFD1834CDE90001BA4A62E7002D7FF4FD
:105BB00031AE04F500559FEDB81ADFEDB80A95ED4A
:105BC0005F0A4FF4A7701DF01FFB04F5055003A9F1
:105BD0003C308DED030A3FF03FFAD5ED5F0A95EDBD
:105BE0005E0AB7EE001A40F24F101DF00DFB04F5EF
:105BF000055003A938308DED030A3FF02DFA0A2233
:105C0000012195F980011DF03DFB03A98DF80C00E1
:105C100004F506503FF08AFA95F98031012B04F51E
:105C2000405602D140F253108AE7013B95ED5E1ACF
:105C3000D5ED5F0A07EE903A71EE606AF8EEE77A0A
:105C400006F2BC6586EEA77A40F2551095ED000A83
:105C500030EE470A96E7924CB4F900300A3300EE72
:105C6000103A4FF4AE709FED8F1ADFED8F0A4DE6BC
:105C70008B4CB4F900300A3B00EE103A40F25F1052
:105C8000F1E78A4CB4F900300A3300EE103A4FF4D1
:105C9000B170E8E7854CB4F900300A3B00EE103AE9
:105CA00040F26510DFE704F5005393F8773E002BD0
:105CB0003FF4B0AD002D7FF4ADAD7D4BB3F90030B6
:105CC000A3F5FA7383EAE372A2EBE372322AC8BF48
:105CD0001DB2784B1D80784BB3F9002082EAE27345
:105CE000A3EBE2739BB2322B744B98BF00221A8055
:105CF000734BB3F9003083EAE371A1EBE37189B22E
:105D0000322998BF00236F4915431D430B8004F5CA
:105D1000405610D001236C4A86F8C03604F52D5049
:105D2000062118304BF056FC96F8C036674A83F0CF
:105D3000010313706EE596F8C03686F8C056002B46
:105D4000F2D0634AEAE7002104F584500430FFF7FB
:105D5000E1FA5FE5002D7FF45DAD294604F584503E
:105D6000043005B0BDE8F0405AF078BD002D7FF456
:105D700051AD002104F584500430FFF7C7FA49E51E
:105D80000121E1E7002D7FF445AD0121E6E7002D7B
:105D90007FF440AD0121EDE70221D5E7002D7FF42E
:105DA00039AD0221DAE7002D7FF434AD0221E1E7BD
:105DB0000321C9E7002D7FF42DAD0321CEE7002D8F
:105DC0007FF428AD0321D5E7424B1D68424B1B6889
:105DD000586A036808219B6B98473230B5F9A220B6
:105DE000B5F9A01000B21DF04DFA82B2092104F5F8
:105DF0008550083020E0374B1D68374B1B68586AC8
:105E0000036808219B6B98473238E7E7314B1B68E2
:105E1000B3F8A020EAE7002D7FF4FCAC2D4B1B6803
:105E2000B3F8A020B3F8AA10914204F5855008BF3A
:105E3000B3F8A4200830092105B0BDE8F0405AF0BD
:105E40006FBD244B1B68B3F8A220CFE7002D7FF471
:105E5000E1AC204B1B68B3F8A220E3E71D4B1B68A5
:105E6000B3F8A420C2E71B4B1D681B4B1B68586A84
:105E7000036809219B6B98473230B5F9B620B5F914
:105E8000B41000B21DF0FEF982B20A21AFE700BFE4
:105E90000000594035520C08CDCC4C3FCDCCCC3D08
:105EA000C47D002000004843000048C3C67D002098
:105EB000C27D0020BC7D0020BE7D0020B87D00207A
:105EC000C07D0020BA7D002046520C0832220020FE
:105ED00056520C085883002048270020474B1D6865
:105EE000474B1B68586A036809219B6B98473238F7
:105EF000C3E7424B1B68B3F8B420C6E7002D7FF41C
:105F000089AC3E4B1B68B3F8B420B3F8BE1004F55F
:105F10008550914208BFB3F8B82008300A218BE7BA
:105F2000364B1B68B3F8B620AFE7002D7FF472AC98
:105F3000324B1B68B3F8B620E7E7304B1B68B3F869
:105F4000B820A2E72D4B1D682D4B1B68586A0368CB
:105F50000A219B6B98473230B5F9CA20B5F9C810B1
:105F600000B21DF08FF982B20B2140E7234B1D6870
:105F7000234B1B68586A03680A219B6B9847323889
:105F8000EAE71E4B1B68B3F8C820EDE7002D7FF44D
:105F900041AC1A4B1B68B3F8C820B3F8D21004F513
:105FA0008550914208BFB3F8CC2008300B2143E75D
:105FB000124B1B68B3F8CA20D6E7002D7FF42AAC39
:105FC0000E4B1B68B3F8CA20E7E70C4B1B68B3F80D
:105FD000CC20C9E7002D7FF41DAC04F5405204F538
:105FE0002D5092F8C13683F0010382F8C136183083
:105FF0000BB1044A20E4044A1EE400BF5883002089
:10600000482700206B520C087D520C082DE9F84FF0
:106010002DED068B994600F55A53D3ED0FAADFED0F
:10602000D67A9FEDD69A9FEDD68ABDF8447000F5DA
:1060300000532AEE899A6AEEA7AAD3ED617A6AEE36
:10604000A7AADFEDD07AF0EE488AEAEEE78A4FF0B1
:10605000000804460E46FDEEE88A154618EE903A12
:106060001BB208EE903AC84B83ED008AC74B83ED14
:10607000008ABDF84830C34647EA03474FF0010A9B
:106080000AFA08F33B425FFA88F109D02046FFF78D
:1060900045F9002173F0D0FF012808BF4FF0010B34
:1060A00008F10108B8F1200FEAD1DFF80CA34FF096
:1060B0000008012303FA08F0DAF8003038425FFAEA
:1060C00088F103EA000300F01E81003B18BF0123A2
:1060D0005A462046FFF7C6FA08F10108B8F1200F2A
:1060E000E7D104F54053CAF8007093F8C126A84BD5
:1060F000BAB1724207EE902AF8EEE77A67EE897A33
:10610000FDEEE77A17EE902A07EE905AF8EEE77A5E
:106110001A8067EE897A9F4AFDEEE77A17EE901AA9
:10612000118077F0DBFF9C4ADFF890821278DFF86D
:1061300090A2974B07461FFA89F19848002A40F031
:10614000EA800088B8F900B000F5FA7000B20AEEF3
:10615000100ABAF9000009EE900A6FF4E1700144E8
:1061600062290FD885EAE570A0EBE57080B231288E
:1061700008D886EAE672A2EBE67292B2312A8CBFA8
:1061800000220122844802701888BDF9503000F2C4
:10619000DC50184440F26C7240F24C4100B21DF0E9
:1061A00071F83A460146002053F0D8FC794B188824
:1061B000BDF9543000F2DC50184440F26C7240F2E9
:1061C0004C4100B21DF05EF83A460146012053F002
:1061D000C5FCB8EECAAAF8EEE88A40F26C72EAEEA4
:1061E0002A8A40F24C4104F54054FDEEE88A18EE4C
:1061F000903A18B21DF046F83A460146022053F094
:10620000ADFCBDF9403007EE103AB8EEC77AF0EEBB
:10621000487AE7EE097A40F26C7240F24C41FDEEAA
:10622000E77A17EE903A18B21DF02CF83A4601467C
:10623000032053F093FC94F8C136002B7CD1F8EE88
:10624000E99AF0EE487AE9EE897A40F26C7240F20F
:106250004C41FDEEE77A17EE903A18B21DF012F8B5
:106260003A460146042053F079FC07EE90BAF8EE66
:10627000E77A40F26C72A7EE898A40F24C41BDEE9B
:10628000C88A18EE103A18B21CF0FCFF3A460146D4
:10629000052053F063FC3D4BD3ED007AFDEEE77A29
:1062A0003A4617EE903A062019B253F057FC364B97
:1062B000D3ED007AFDEEE77A3A4617EE903A0720E2
:1062C00019B253F04BFC364B3A46B3F90010082094
:1062D00053F044FC334B3A46B3F90010092053F015
:1062E0003DFC314B3A46B3F900100A2053F036FC1E
:1062F0002E4B1E802E4B1D802E4BA3F80090BDEC24
:10630000068BBDE8F88F002B3FF4E6AE5A462046D8
:10631000FFF798F8E0E60288B8F800B011440AB236
:106320000AEE102ABAF800203244AB4412B209EE49
:10633000902A0FFA8BFB27E7BAF9003007EE103AE4
:10634000B8EEC77AF0EE487AE7EE097A40F26C725E
:1063500040F24C41FDEEE77A17EE903A18B21CF08D
:1063600091FF3A460146042053F0F8FBB8F900309B
:1063700007EE903A7BE700BFCDCC4C3FCDCCCC3E76
:106380000080BB440000FA433C220020342200205D
:10639000C67D0020C47D002032220020BC7D00206C
:1063A000382200203A22002030220020BE7D00202A
:1063B000C07D0020C27D0020B47D0020BA7D002079
:1063C000B87D0020012070470020704700207047F2
:1063D0000020704700207047002070479FED010AA1
:1063E000704700BF0000000070470000144A0260C0
:1063F000144A426002F1BC0181601349C160134933
:10640000016102F67C41416102F62C01816102F5D5
:106410000361C16102F63401016202F63801416292
:1064200002F63C0102F50462C262094A0263A2F567
:1064300089624263A2F55B5281628263704700BF4A
:1064400008530C0880480020505E00205838002077
:1064500070630020152938D8DFE801F00F131723E7
:106460002737372B372F3737373737371F37370B24
:10647000331B00F5A7401C30704700F5A74058308B
:10648000704700F5A8401430704700F5A840503020
:10649000704700F5AB407430704700F5AA400430F7
:1064A000704700F5A9400C30704700F5A94048300E
:1064B000704700F5AA404030704700F5AA407C3094
:1064C000704700F5AB40383070470020704700003F
:1064D00000F5A040D0F8980303685B6818470000F7
:1064E00038B500F5A0450446D5F8980303685B6904
:1064F00098470A4B04F50052187492F8842DD5F889
:106500009803DA7003681B6A9847014604F58550C2
:106510001830BDE838403AF03BB900BFCD7E0020CE
:106520002DE9F04700F50059064699F8843D8B4265
:106530000F46924605D189F8EC2001252846BDE892
:10654000F087FFF787FF044620B9304645F000FF8B
:106550002546F3E703689B68984706F52D5808F130
:106560001808A8B1314804F07FF9054680B92368BE
:106570002046DB6998472E4A0346042140464BF0EB
:1065800029F847F01BFF3A460A2147F0CFFCD5E730
:106590002648FBF737FA50B3236800211B682046D2
:1065A00098470546002839D006F5804306F5944003
:1065B00093F8991A203055F041FF99F8843D89F8F5
:1065C000853D06F5A0435246C3F89843394606F682
:1065D000A86089F8847D89F8ECA047F0B7F84046B8
:1065E000002152F0BBFC3046FFF77AFFA6E706F524
:1065F000A043D3F898030368DB6898470028CBD002
:1066000023682046DB68984705460028C4D12368E4
:106610002046DB699847074A0346AEE723682046D1
:10662000DB699847044A0346A7E700BF50270020CC
:1066300090520C08B9520C08E2520C080148FFF7BE
:106640006FBF00BF502700202DE9F04F07EE902AC2
:106650002DED048BF8EEE78A07EE901AB8EEE78A84
:1066600095B028EE080A4FF0000BA8EEA80A0646DF
:10667000884615461F46CDF808B0CDF80CB0CDF8C9
:1066800010B0CDF814B0CDF818B0CDF81CB0A3F010
:1066900095FBDFEDBB9AB4EEE90AF1EE10FA10DDDE
:1066A000C9EE807A27EE888A67EEA87ABDEEC88A9E
:1066B000FDEEE77A18EE103A0FFA83F817EE903AEB
:1066C0001DB2736807EE908A93ED2C7AB8EEE79AC4
:1066D000B5EEC07A07EE905AF1EE10FAF8EEE75AEE
:1066E00000F29A8093ED278A28EE099A28EE258AEF
:1066F000736807EE907A93ED280A93F9AC30F8EEC0
:10670000E78A68EE808A002B78D03369D3F8F801E5
:106710001CF044FD9B4940F6B83281461CF0A2FDB6
:10672000434207EE903A7368F8EEE77A93ED297AE0
:10673000336967EE877AD3F8FC01CDED027A1CF05D
:106740002DFD40F6B8328F4982461CF08BFD424247
:106750007368CDF810B007EE102AD3ED2A6A93F9CA
:10676000AC20B8EEC77A022A27EE267A8DED037A9E
:106770001ED1854AB2F92C414C457ADAA9EB0409BD
:1067800007EE909AD3ED295AB8EEE76ADDED027A6A
:10679000E5EEC67ACDED027A54457BDAAAEB040425
:1067A00007EE904AF8EEE77AA6EEE77A8DED037AE7
:1067B000D6F834C00CF184030FCB10AC84E80F0082
:1067C0000DF1300908AC89E80F0084E80F0005AB33
:1067D00002AA214660466EF04DFF736893F9AC3013
:1067E000022B5CD1DDED057A39EE279ADDED067AD4
:1067F00038EE278ADDED077A78EEA78A229B83EDB3
:10680000009A239B83ED008A249BC3ED008A15B078
:10681000BDEC048BBDE8F08FF7EE007AB4EEE77ABA
:1068200089EE297A85EEA98AF1EE10FAC8BFC3ED88
:106830002C7A7368D3ED2C6A93ED270A77EEE67A0B
:1068400027EE076A27EE879A26EE076A28EE087A6F
:1068500067EE887A27EE087AA6EE869AE6EE877AC1
:1068600029EE299A27EEA98A29EE009A28EE008AB5
:106870003EE762424A458FDDA14407EE909A9DEDC6
:10688000026AD3ED295AF8EEE77AA5EEE76A8DEDB4
:10689000026A81E7634253458ADD544480E7002D54
:1068A00088EAE871B8BF6D42A1EBE87189B2ADB278
:1068B000A9420191D4BF214601A90895002FB8BF74
:1068C0007F420B68DFED310ABFB29F42A8BF494645
:1068D0000C97D1ED007AF8EEE77AB7EE001A87EE62
:1068E000A90A4FF4827031EE400A1CF08DFC336926
:1068F000D3ED937A05A820EE270A1FF041F8F0EEB9
:10690000C07A8DED071AB0EEC91A31EE671A8DED17
:10691000050AB0EEC11A30EE090ACDED060A4FF4B1
:106920008670F1EE410A1CF06FFCB0EE409A9DEDCE
:10693000060AB0EEC81AF0EEC07A31EE671A30EEF1
:10694000080AB0EEC11AF1EE410A40F211101CF033
:106950005BFCB0EE408A9DED070AB0EEE81AF0EE5F
:10696000C07A31EE671A38EE800AB0EEC11A4FF4E1
:106970008B70F1EE410A1CF047FCF0EE408A3DE7D7
:1069800000A08C4548F4FFFF5047002000000000A5
:106990000148FFF7C5BD00BF5027002000487047E1
:1069A000A852002000207047012070470120704746
:1069B000002070470048704740530C08004870475B
:1069C00040530C0808B5036B03480022C3F8542356
:1069D000FEF71EFE012008BD5027002070B50446BA
:1069E000406990F8CB3088B093B9012174F0B8FBBE
:1069F000606B62680368D2ED020A5B6E9FED240A49
:106A000001219847606B08B0BDE870406FF000BA94
:106A1000022174F0A5FB636AE269A1691B68126830
:106A20000968B2F90820B1F90810B3F9083007A8CD
:106A3000029006A8019005A800902046FFF704FEEA
:106A4000606B9DED071A0368DDED060A9DED050AF2
:106A50009B6B9847656B2B685E6E236A186853F0D2
:106A600011FA63680021D3ED020A2846B047A36AF1
:106A70006569186853F006FA85ED0E0AE36A6569E0
:106A8000186853F0FFF985ED0F0A08B070BD00BF1C
:106A90000000000000207047002070470120704770
:106AA000002070470048704788530C080048704722
:106AB00094530C0870B504462148FAF7A3FF054625
:106AC00000283AD01E48266BFBF71AFB6368B3F91F
:106AD0003020B3F92C3000EE903A434201EE102AF8
:106AE00000EE103AB8EEC11AF8EEE00AB8EEC00AAD
:106AF000304670F0B7FA1248266BFBF701FB63686B
:106B0000B3F93020B3F92C3000EE903A434201EE55
:106B1000102A00EE103AB8EEC11AF8EEE00AB8EE0C
:106B2000C00A304670F018FB206B71F093FB2369AC
:106B3000D3F80022034BC3F88423284670BD00BF5E
:106B4000502700205077002070B52DED028B8AB0C1
:106B5000044677F0C3FA06467348256BFBF7D0FA74
:106B60006368B3F93020B3F92C3000EE903A434219
:106B700000EE103A01EE102A2846B8EEC11AF8EEDF
:106B8000E00AB8EEC00A70F06DFA6069674D90F8DF
:106B9000CB30EBB9012174F0E3FA606B62680368F3
:106BA000D2ED020A5B6E0121B6EE000A9847606BD7
:106BB0006FF02EF96069266B03681B6998473046B1
:106BC00071F0C4FB2369D3F80032C5F8843390E038
:106BD000022174F0C5FAD5F8543341F28732F31A22
:106BE000934233D8D5F85C330693D5F860330793D6
:106BF000D5F864330893D5F86833099303A905AB36
:106C000006A804AA1EF0D4F89FED497ADDED037AB8
:106C1000DDED040A9DED051A606B9FED460A67EEF7
:106C2000877A60EE870A21EE071ACDED040A8DED12
:106C3000051ACDED037A036821EE001A60EE800A92
:106C40001B6B27EE800A0121984752E0A369606B15
:106C50001B68B3F9083008EE103AE3691B68B3F912
:106C6000083000EE903A0368F8EEE00A9B6ECDED36
:106C7000010A9847B8EEC88AB0EE401ADDED010A65
:106C8000B0EE480A04AA03A9A5F5A040FBF736F91F
:106C9000636A1868438A828907EE903A264BF8EEB9
:106CA000E77A93ED007A67EE877AFCEEE77A17EEE3
:106CB000903A99B253F07CF80146A5F5A040FBF755
:106CC00087F9DFED1E7A606BB0EEC07AB4EEE77A3A
:106CD000F1EE10FAB0EE401A0FD40368DDED040AAD
:106CE000DB6A9DED030A98472369D3F80032C5E9B2
:106CF000E1360AB0BDEC028B70BDD5F8883302686E
:106D00009DED030ADDED040AFA33B34204D9D36AD8
:106D10009FED0B1A984755E795EDE11A136BB8EE06
:106D2000411A012190E700BF502700205077002032
:106D3000E02E65420000C8420C5E002000000034D6
:106D40000000000038B5836A45690446186853F0AE
:106D500099F885ED0E0AE36A6569186853F092F8B0
:106D600085ED0F0A38BD000030B52DED028B036AAA
:106D70001B68B3F9083000EE103A83B00446B8EE51
:106D8000C00A2F48FBF7CEF92D488DED010AFBF71D
:106D9000B7F963689DED010AB3F92C3001EE103AA2
:106DA000434200EE903AB8EEC11AF8EEE00A6C20C9
:106DB0001CF02AFADFED237AB0EEC07AB4EEE77A5F
:106DC000F1EE10FAB0EE408A19D51F4B256B93F8FF
:106DD000802D93F9803D002B1EDA636895EDD57AFE
:106DE000D3ED2D7AF1EE046A77EEE67AF4EE477A87
:106DF000F1EE10FAC8BFF0EE477AC5EDD57A206BF8
:106E0000B0EE480A70F0B4F9206B03B0BDEC028B11
:106E1000BDE8304071F00CBB5306F0D5E06873F06C
:106E2000F5F8236BF2EE047A30EE270AD3EDD57A2B
:106E3000B4EE670AF1EE10FAC8BFF0EE407ADCE774
:106E400050270020CDCC4C3D5047002010B50446C3
:106E5000FFF77AFE2046FFF787FF2046BDE8104087
:106E6000FFF770BF01207047012070470020704776
:106E7000012070470120704700487047DC530C0820
:106E800000487047DC530C0830B5054685B01748FC
:106E900003F0EAFC044620B3154BB3F8502A012A4C
:106EA00022D903F5405203F58053042193F8D436D8
:106EB00082F83C16022B03D10021284600F036FF51
:106EC000DFED0C0A0C48B0EE601AF0EE601AB0EE7E
:106ED000600A72F0E3FB284600F01EFF074821F02D
:106EE000B9FD204605B030BD0024FAE75027002048
:106EF0005047002000000000846700206C510020F3
:106F000070B5144C05460026A4F6CC7084F83C6697
:106F100072F02AFB60B92846FFF740FD0E4A0421B3
:106F20004AF058FBA4F5A040BDE87040FEF738B920
:106F3000A4F5005494F8D436022B09D031462846E3
:106F400000F040FE01462846BDE8704000F0EEBE6D
:106F500070BD00BF50770020E4530C08094B03F5C7
:106F6000A042022103F5804382F83C1603F6741216
:106F700003F6641192ED000A93F89829A1F11C0020
:106F800071F0FABC50270020F0B52DED028B0446BD
:106F9000B0EE408A4648DFED478A8FB00E4617466E
:106FA00071F06CFBF0EEC87AF4EEE87AF1EE10FACC
:106FB00006D49FED410A3E4828EE000A71F0C4FB5A
:106FC0003E4D95ED000AA5F67415B0EEC00A0FB15E
:106FD000B1EE400A364871F0A7FB0023344807930E
:106FE00002AA07A90893099371F0BEFBDFED347A7A
:106FF0009DED027AB4EEE77AF1EE10FA54DD314FEE
:107000000123022207A90AA887F83C360BF0B0FB3F
:107010007168019130460BF0E7F8019902460AA821
:107020000BF0B8F80AA9A7F6CC7072F09DFA18B95F
:10703000A7F5A040FEF7B4F8E06872F0E5FF03A9F9
:10704000026843682048049303921EF017F905A8CC
:107050008DED050ACDED060A1EF0DEF905F5176384
:10706000D3ED007AF4EEE87AF1EE10FABCBF05F643
:107070005815D5ED007AF4EEC07AF1EE10FA4FF023
:10708000000120460AD5DFED117AB4EEE70AF1EEF1
:1070900010FA03DD00F096FD0146204600F046FEA2
:1070A0000FB0BDEC028BF0BD2046FFF757FFF7E7AE
:1070B00098700020000000340000C842C470002016
:1070C0000000964350770020B47000200000FA437F
:1070D00037B59FED1A0A1A4D04461A4871F0E6FCBE
:1070E00001462846FDF784FD694601AA284602F0BC
:1070F000C3FD6369009ADA636369019A9A63206B3E
:1071000071F096F9E369606B1B68B3F9083000EE23
:10711000903AA3691B68B3F9083000EE103A03688F
:1071200005F592451B6B95ED1E1AF8EEE00AB8EED8
:10713000C00A0121984703B030BD00BF0000000025
:107140005027002098700020F0B52DED028B0446EA
:10715000406B264D85B0F0EE408A6C309FED240ADE
:10716000B0EE608A0E4617461EF00AFCDFED217A6B
:107170008DED031AF7B928EEA70A1BF0DBFF9FED90
:107180001E7ABDEEC00AF0EEC87A10EE103AF4EEA8
:10719000C77AF1EE10FAC5F8EC3618D53C23032176
:1071A0002046A5F8F03605B0BDEC028BBDE8F040F6
:1071B00000F0BCBD9DED030ABDEEC00A002EB8EE86
:1071C000C00AB8BFF1EE688AA8EEA70AD5E7DFEDDE
:1071D0000B7AB4EEE78AF1EE10FA58BFB0EE678A88
:1071E000BDEEC88A18EE103AD9E700BF505700200C
:1071F0009F0CB3450000C8420000003400007042FC
:10720000DFED097A094BB4EEE70AF1EE10FA58BF48
:10721000B0EE670ABDEEC00A072110EE102AA3F8EF
:10722000F02600F083BD00BF0000704250570020E0
:1072300070B54B68164D06460C468BB98B687BB90A
:10724000C96869B900F0BEFC0146304600F06EFD29
:1072500095F8991A05F52260BDE8704055F038BAE6
:1072600095F8991A0B4855F0DDF840B90A492046BF
:107270000BF04CF918B10221304600F057FD95F89B
:10728000991A04482246BDE8704055F015BA00BF6F
:107290005067002070710020285E002070B5192111
:1072A000054624483EF03CFB023802283FD8224CD9
:1072B000052384F83C3676F011FFC4F88C031F4890
:1072C0001EF0C6FFDFED1E0AA4F5E160B0EE600A15
:1072D00072F0C2FBA4F5E16072F09CFC68692E6B51
:1072E00003681B699847A4F58054304671F02EF866
:1072F00094ED150A94ED191AD4ED140A286BB0EE2A
:10730000C00A6FF0AFFE94ED150A94ED191AD4ED92
:10731000140A286BB0EEC00A6FF01EFF2846FFF774
:107320003DFB084A04214AF055F9012070BD0020B8
:10733000FCE700BF48330020507700206C5100204C
:107340000000000010540C0870B52DED028B0446AF
:10735000406990F8CB3084B0FBB9012173F000FF95
:10736000606B62680368D2ED020A5B6E9FED6C0A87
:1073700001219847606B6EF04BFD6A4872F04AFC41
:107380006069256B03681B699847284604B0BDEC0B
:10739000028BBDE8704070F0D9BF6348634D19217E
:1073A0003EF0BEFA032865D004286DD00228604E56
:1073B00040F0A58005F58045002395ED148A3360E3
:1073C0005C4D76F08BFED5F88C3303F51C531033EF
:1073D00098420AD92046FFF7E1FA574A02214AF0BB
:1073E000F9F8A5F5A040FDF7B3FE4E48012172F073
:1073F000A3FD694601AA4D4802F0F8FB6369009AB3
:10740000DA636369019A9A63B0EE480A206B9FEDD4
:10741000448A6FF0ADFE206B71F00AF847488DED9D
:10742000028AB0F92C318DED038A01EE103AE3693E
:107430001B68B3F9083000EE903AA3691B68B3F9F2
:10744000083000EE103AB8EEC11AF8EEE00AB8EED5
:10745000C00A03AA02A9A0F50050FAF74FFD606B1D
:10746000DDED030A03689DED020ADB6AB0EE481AFF
:10747000984750E005F5804595ED158A2C4B002284
:10748000B0EEC88A1A609BE705F5005595F8983963
:107490009B0731D5264D2B6853B976F01FFE286027
:1074A0006069266B03681B699847304670F04EFF91
:1074B00076F014FE2B6803F2DC5398421CD9204668
:1074C000FFF76CFA1E4A06214AF084F8174801219A
:1074D000FDF78EFB194890F8A43D6FF3C30380F8C5
:1074E000A43D00F54053042200F61C2083F83C26FE
:1074F00021F042FA00232B609FED098A60E72046C5
:10750000FFF74CFA0F4A02214AF064F82846FDF7CB
:107510001FFE0023336004B0BDEC028B70BD00BFC2
:107520000000000048700020483300205027002051
:10753000CC7D0020507700208D540C08504700204F
:1075400034540C085A540C087FB505460F4803F014
:107550008BF90446B0B10E4E042386F83C3601A9DF
:107560000023A6F6CC7001930293039371F062FCA2
:1075700001A90022A6F6CC7072F070F9002128460D
:1075800000F0D4FB204604B070BD00BF502700209F
:107590005077002070B52DED028B0446406990F8BD
:1075A000CB3088B03BBB012173F0DAFD606B9FEDFF
:1075B000508A62680368D2ED020A5B6EB0EE480A38
:1075C00001219847606B6EF023FC4A488DED058AD7
:1075D000F0EE480AB0EE481AF0EE481AB0EE480A4B
:1075E0008DED068A8DED078A08B0BDEC028BBDE8F3
:1075F000704072F053B8404E96F8A41D11F001058A
:107600005DD1636A1B68A6F50050B3F90810FAF75C
:10761000DFFCDFED3A7AB0EEC07AB4EEE77AF1EE55
:1076200010FAB0EE408A03D42946204600F07EFBD3
:107630000221606973F094FD2E4871F015FF014638
:107640002F48FDF7D5FA02A92D4803AA02F0CEFA79
:107650006369029ADA636369039A9A63206B70F034
:10766000E7FEB6F92C31264801EE103AE3691B68B3
:10767000B3F9083000EE903AA3691B68B3F90830FB
:1076800000EE103AB8EEC11AF8EEE00AB8EEC00A01
:1076900005AA04A9FAF732FC1A4B656B93F8D436A5
:1076A00083B92B68DDED050ADB6A9DED040AB0EEB7
:1076B000481A2846984708B0BDEC028B70BD9FED74
:1076C0000C8AB5E72B68DDED050A9DED048ACDED4A
:1076D000010A20461E6B00F0E9FDDDED010AB0EE67
:1076E000401A0121B0EE480A2846B047E3E700BF40
:1076F0000000000084670020504700200000003494
:10770000502700205057002030B52DED028B044645
:10771000406990F8CB3087B03BBB012173F020FD6E
:10772000606B9FED3C8A62680368D2ED020A5B6E73
:10773000B0EE480A01219847606B6EF069FB36484D
:107740008DED038AF0EE480AB0EE481AF0EE481AC2
:10775000B0EE480A8DED048A8DED058A07B0BDECC8
:10776000028BBDE8304071F099BF2C4D95F8A43DD7
:10777000DB074BD4636A1B68A5F50050B3F908100A
:10778000FAF726FCB0EE408A6069022173F0E8FC4B
:10779000214871F069FE01462148FDF729FA694642
:1077A00001AA1F4802F022FA6369009ADA6363694A
:1077B000019A9A63206B70F03BFEB5F92C311848A2
:1077C00001EE103AE3691B68B3F9083000EE903A15
:1077D000A3691B68B3F9083000EE103A03AA02A9A6
:1077E000B8EEC11AF8EEE00AB8EEC00AFAF786FB66
:1077F000606BDDED030A03689DED020ADB6AB0EE03
:10780000481A984707B0BDEC028B30BD9FED018A46
:10781000BAE700BF00000000846700205047002046
:107820005027002008B50748012101F0ABF8064BAE
:10783000032283F83C2603F28C40BDE8084000F0A8
:10784000EBBF00BF187C00205077002010B5044625
:10785000134820F09BFF134B93F83C36052B1DD8A3
:10786000DFE803F00303080D12172046BDE81040BF
:10787000FFF790BE2046BDE81040FFF729BCBDE8E9
:107880001040094801F052BA2046BDE81040FFF709
:107890003BBF2046BDE81040FFF756BD10BD00BFFE
:1078A0006C51002050770020187C00200120704788
:1078B0000020704701207047012070470048704742
:1078C000F0540C0800487047F8540C0870B52DEDC2
:1078D000028B614DDFED618AD5ED177ADFED600A2D
:1078E00095ED130AF4EEE87AF1EE10FA0446A8BF1B
:1078F000F0EE670A82B0006B6FF06CFAA5F580407D
:10790000266BFAF7FDFB6368B3F93020B3F92C302E
:1079100000EE903A434200EE103A01EE102A304653
:10792000B8EEC11AF8EEE00AB8EEC00A6FF09AFBA2
:10793000606990F8CB30C3B9012173F011FC606B22
:1079400062680368D2ED020A5B6E9FED460A012170
:107950009847606B6EF05CFA05F6481002B0BDEC1B
:10796000028BBDE8704071F023B8636A1B68A5F50F
:107970008040B3F90810FAF72BFBF0EEC07AF4EE72
:10798000E87AF1EE10FAA5F580565CBF012386F87F
:10799000EC30236A34481B68B3F90830B0EE408AF3
:1079A00000EE103AB8EEC00AFAF7BCFB022160699B
:1079B000F0EE408A73F0D4FB9FED2A0A2B4871F059
:1079C00075F801462848FDF713F9274801AA6946CA
:1079D00002F052F96369009ADA636369019A9A6363
:1079E00096F8EC10606BD4E90632F1B112681B68AE
:1079F000B2F90820B3F9083000EE902A00EE103AF0
:107A00000368F8EEE00ADB6AB8EEC00AB0EE481A86
:107A10009847206BB0EE680A6FF0AAFB206B70F0FD
:107A200007FD02B0BDEC028B70BD12681B68B2F995
:107A30000820B3F9083000EE902A00EE103A0368EF
:107A400005F678151B6B95ED001AF8EEE00AB8EE16
:107A5000C00A01219847DCE750670020000000348D
:107A600000007A430000000050270020987000209A
:107A7000F8B504462DED028B334802F0F5FE0546BD
:107A800000285CD0314EDFED328A9FED328A06F558
:107A90008057D7ED170A97ED130A0023F4EEE80A92
:107AA00086F8EC30F1EE10FAB8BFF0EE480A206B21
:107AB0006FF090F9D7ED170A97ED130A206BF4EEEB
:107AC000E80AF1EE10FAB8BFF0EE480A6FF0FAF9E2
:107AD000A6F54050276BFAF713FB6368B3F9302023
:107AE000B3F92C3000EE903A434201EE102A00EE3A
:107AF000103AB8EEC11AF8EEE00AB8EEC00A3846FD
:107B00006FF0B0FAA6F54050276BFAF7F9FA636800
:107B1000B3F93020B3F92C3000EE903A434201EE35
:107B2000102A00EE103A3846B8EEC11AF8EEE00A14
:107B3000B8EEC00A6FF010FB074870F039FFBDECDB
:107B4000028B2846F8BD00BF502700205057002068
:107B50000000003400007A43987000200120704734
:107B6000002070470120704701207047004870478F
:107B700040550C080048704748550C0890ED007AB5
:107B8000DFED0F7AB0EEC77AB4EEE77AF1EE10FAD5
:107B900014D590ED017AB0EEC77AB4EEE77AF1EE43
:107BA00010FA0BD590ED027AB0EEC77AB4EEE77A10
:107BB000F1EE10FA4CBF0120002070470020704702
:107BC00000000034436893F92930042B0BD8DFE818
:107BD00003F00C0A050308000420704781F001003F
:107BE0007047062070470120704700207047000052
:107BF00038B52DED048B0446406990F8CB30B3B90D
:107C0000012173F0ADFA606B62680368D2ED020A7D
:107C10005B6E9FED3D0A01219847606B6EF0F8F8AE
:107C2000BDEC048B206BBDE8384070F013BB374DC2
:107C300095ED028AD5ED018A28EE080AA8EEA80A79
:107C4000A2F0BCF8606B03689B6EB0EE409A984758
:107C50002F4BB3F92C3107EE903AF8EEE77AB4EEF9
:107C6000E70AF1EE10FA58BFB0EE670AB4EEC90A9F
:107C7000F1EE10FA48BFC0EE097A95ED030A44BF51
:107C800028EE278A68EEA78A1BF06AFA214BD3ED0B
:107C9000150A93ED141AF0EEE00AF1EE600AF0EE28
:107CA000409A4FF4307095ED040A1BF0ADFAB0EE37
:107CB000409A76F013FA2B68C01AB0F57A7F88BF25
:107CC0009FED118A60694FF0020184BFB0EE489ABF
:107CD000F0EE488A73F044FA606B0368B0EE691AFC
:107CE0001B6BF0EE480AB0EE680A01219847206B42
:107CF000B0EE490A6FF03CFABDEC048B206BBDE896
:107D0000384070F095BB00BF00000000D47D00201B
:107D10005047002050670020034B00221A600022C9
:107D20005A609A60DA607047007E00200C4B93F82E
:107D3000D4268A420FD0022983F8D41602D004290F
:107D40000AD0704703F2E4630269D2ED807AF8EE5C
:107D5000E77AC3ED007A704703F2F463F4E700BFFB
:107D6000505700202DE9F0412DED048B82B088465C
:107D70001446F0EE608A0193B0EE408A074605F0A3
:107D80004BFB9FED279A90ED830A264D1BF012FACC
:107D900028EE098AF0EE409AB0EE480A1BF00AFA83
:107DA00030EE690A1BF01CFAB5EEC00AF1EE10FACB
:107DB0004CBF4FF0FF360126B8F1000F16D0019AE4
:107DC00071B26CB9DFED180A85F8D5461748B0EEE8
:107DD000480A02B0BDEC048BBDE8F041FFF7B4B92E
:107DE000002368EE890A85F8D536EFE764B128EEFE
:107DF000890A0E48012385F8D53602B0BDEC048B04
:107E0000BDE8F041FFF7FCB92146384685F8D54674
:107E100002B0BDEC048BBDE8F041FFF787BF00BFA7
:107E20000AD7233C5057002000000000DC7B0020D4
:107E300070B5244D05F5A0430122044683F83D2684
:107E4000066B2846FAF75CF96368B3F93020B3F99A
:107E50002C3000EE903A434201EE102A00EE103A28
:107E6000B8EEC11AF8EEE00AB8EEC00A30466FF07C
:107E7000F9F82846266BFAF743F96368B3F930201E
:107E8000B3F92C3000EE903A434201EE102A00EE96
:107E9000103AB8EEC11AF8EEE00AB8EEC00A304661
:107EA0006FF05AF9206B70F0D5F905F54055206B4D
:107EB0006FF06AFF002185F8D5162046BDE87040B6
:107EC000FFF734BF5027002038B50A4B93F83D36F2
:107ED000012B05460C4601D0FFF7AAFF76F0FEF80D
:107EE000054B186094E807002B6B03F5597383E882
:107EF000070038BD50770020D07D002030B50C46FB
:107F000011461A46134B93F83D36012B85B00546B2
:107F10000DD0CDED030A02928DED010A0091FFF71D
:107F200087FFDDED030A029A9DED010A00999DF895
:107F300020302846FFF716FF76F0D0F8064B186081
:107F400094E807002B6B03F5597383E8070005B02D
:107F500030BD00BF50770020D07D002070B5174E97
:107F600006F5804506F5A043022295ED150A83F833
:107F70003D26044695ED191AD5ED140A006BB0EEB6
:107F8000C00A6FF06FF895ED150A95ED191AD5ED49
:107F9000140A206BB0EEC00A6FF0DEF8206B70F0B0
:107FA00059F906F54056206B6FF0EEFE002186F879
:107FB000D5162046BDE87040FFF7B8BE5027002018
:107FC0002DE9F04F2DED028B89B00746154604A828
:107FD00002220C460AF0CCFB284804A95DF06AFB9B
:107FE000814658B946F0EAF90522162145F09EFF70
:107FF000484609B0BDEC028BBDE8F08FDFF890A0D9
:108000009AF83D36022B02D03846FFF7A7FF76F0EC
:1080100065F81B4B1B4E216862681860A368B3604B
:108020003160726095E80700DFF868809FED168A7E
:108030004FF0010B88E8070002AB386BCDF800B0B9
:10804000424631468DED028A8DED038A6EF042FF85
:10805000B368386B029308F108025B4602A9B0EEE0
:10806000480A6FF005FE029BB3609AF83D16074878
:108070002B462246FBF78AFABAE700BF28470020C2
:10808000D07D0020E87D0020000000005027002067
:1080900050770020F47D00202DE9F04F2DED028B6C
:1080A00089B00746154604A802220C461E46B0EECB
:1080B000408AF0EE608A0AF05BFB2E4804A95DF06E
:1080C000F9FA814658B946F079F90522162145F0AA
:1080D0002DFF484609B0BDEC028BBDE8F08FDFF8FC
:1080E000A8A09AF83D36022B02D03846FFF736FF9B
:1080F000F0EE680AB0EE480A9DF854309DF8502022
:10810000DFF888809FED1C8A31463846FFF72AFE4B
:1081100075F0E4FF194B1A4E216862681860A36875
:10812000B3603160726095E807004FF0010B88E89A
:10813000070002AB386BCDF800B0424631468DEDFA
:10814000028A8DED038A6EF0C5FEB368386B029328
:1081500008F108025B4602A9B0EE480A6FF088FDFC
:10816000029BB3609AF83D1606482B462246FBF761
:108170000DFAAEE72847002000000000D07D002067
:10818000E87D00205027002050770020F47D00205B
:1081900070B5224E06F5804506F5A043032295ED05
:1081A000150A83F83D26044695ED191AD5ED140AF3
:1081B000006BB0EEC00A6EF055FF95ED150A95ED17
:1081C000191AD5ED140A206BB0EEC00A6EF0C4FF88
:1081D000206B70F03FF875F081FF2269104BD2EDF3
:1081E0007E7A1860F8EEE77A06F54056C3ED017A1C
:1081F000D2ED7F7AF8EEE77A0021C3ED027AD2ED74
:10820000807A86F8D516F8EEE77A0022C3ED037A75
:108210001A612046BDE87040FFF788BD5027002056
:10822000D47D002038B52DED028B1C4B93F83D36E4
:10823000032B0D46B0EE408A01D0FFF7A9FF184C82
:10824000284604F10C0304F10802211D1CF0B0FDC6
:10825000DFED146AD4ED017A9FED137A94ED030AF1
:1082600067EEA67A20EE260A67EE877A20EE070AE6
:10827000C4ED017AD4ED027A67EEA67A67EE877ACA
:10828000C4ED027A1AF06CFF84ED048A84ED030ACF
:1082900075F024FFBDEC028B206038BD50770020C4
:1082A000D47D0020E02E65420000C84230B52DED9F
:1082B000028B3C4A92F8D436023B83B00446042B2E
:1082C0006AD8DFE803F0030B151D2000364803B021
:1082D000BDEC028BBDE83040F9F79EBE02F2EC63C4
:1082E00093ED000AB8EEC00A03B0BDEC028B30BDBE
:1082F0002D4803B0BDEC028BBDE83040F9F7AEBEAF
:1083000092ED3C0AEEE72949DFED298AA1F10C0044
:108310001BF05EF9236BD3E9DC016D4685E80300B1
:108320002846B0EE408A1DF077F8236B9FED217A46
:10833000D3EDC27A67EE877AB4EEE70AF1EE10FA6F
:1083400027DB28461DF01EF8DFED1B7A20EE270AFA
:10835000F0EE487AD0EE287AB0EE670A1AF000FF05
:10836000636893F9283007EE903A5B4200EE903A4A
:10837000B8EEE71AF8EEE00A21EE281A60EEA80A35
:108380004FF44D701AF040FF38EE000A1AF0D2FE9A
:10839000AAE79FED0A0AE3E7094B5B6C93EDD10A6C
:1083A000A2E700BF5057002050270020187000207F
:1083B0000000C842CDCCCC3DE02E6542000000005C
:1083C0005067002070B52DED028B0446406990F88F
:1083D000CB3084B0D3B9012172F0C2FE606B626809
:1083E0000368D2ED020A5B6E9FED6C0A012198478B
:1083F000606B6DF00DFD206B6FF02CFF206B04B0F7
:10840000BDEC028BBDE870406FF0BEBC644890F8D4
:10841000A41D11F0010500F580566BD1636A1B683D
:10842000A0F50050B3F90810F9F7D2FDDFED5D7A41
:10843000B0EEC07AB4EEE77AF1EE10FAB0EE408A10
:1084400051D429462046FFF771FC6069022172F081
:1084500087FE75F043FE544B1B68C01A40F6B833D4
:1084600098420CD9256B05F55970FFF787FB30B999
:108470000023C5F86433C5F86833C5F86C33206B46
:108480006EF0CCFD206B6FF095FD206B90EDDB0A5C
:108490006EF06EFE206B6FF0CBFF03AA02A943487B
:1084A00001F030FC6369029ADA636369039A9A63A4
:1084B00096F8D436656BD4E90612F3B91368B3F9AC
:1084C000083000EE903A0B68B3F9083000EE103A2D
:1084D0002B68F8EEE00ADB6AB8EEC00AB0EE481A84
:1084E0002846984735E096F8D5360BB10721A9E71D
:1084F0000321A7E79FED298AA7E709681268B1F968
:108500000810B2F9082008EE101A00EE902A032B8A
:10851000B8EEC88AF8EEE00A1FD1B6F9F036DFED02
:10852000247ACDED010A01EE903AF8EEE11A2046E8
:1085300061EEA71ACDED001AFFF7B8FEDDED001AC7
:10854000DDED010AB0EE401A2846B0EE480A6CF0A4
:10855000BDFA04B0BDEC028B70BD072B2A680DD1AB
:10856000B6F9F0369FED121A07EE903AF8EEE77A78
:10857000D36A27EE811AB0EE480AB1E72046CDED66
:10858000000A166BFFF792FEDDED000AB0EE401A0E
:108590000121B0EE480A2846B047DAE700000000A3
:1085A0005047002000000034D07D002050270020DC
:1085B0000000C842F0B52DED028B0446406990F8EA
:1085C000CB308DB0D3B9012172F0CAFD606B626807
:1085D0000368D2ED020A5B6E9FED800A0121984785
:1085E000606B6DF015FC206B6FF034FE206B0DB0EE
:1085F000BDEC028BBDE8F0406FF0C6BB78489FED44
:10860000778A90F8A41D11F0010500F5805640F01E
:108610009180636A1B68A0F50050B3F90810F9F760
:10862000D7FCDFED707AB0EEC07AB4EEE77AF1EE07
:1086300010FAF0EE408A76D429462046FFF776FB02
:108640006069022172F08CFD75F048FD664B1B6875
:10865000C01A40F6B83398420AD9644D2846FFF74D
:108660008DFA28B985ED028A85ED018A85ED008AAB
:10867000236B5E4893EDBF0A5D4D1DF081F9012724
:1086800009A92846CDED070A8DED081ACDED0A0A95
:108690008DED0B1A8DED060A8DED090A1DF090F98E
:1086A0002946524A206B009709AB8DED098A8DED62
:1086B0000A8A6EF00FFCAB689FED480A4D4A206BAA
:1086C000059305A93B466FF0D3FA059B206BAB6081
:1086D0006FF070FC206B6FF0ABFE09AA06A946484C
:1086E00001F010FB6369069ADA636369099A9A6379
:1086F00096F8D436656BD4E90612F3B91368B3F96A
:10870000083000EE903A0B68B3F9083000EE103AEA
:108710002B68F8EEE00ADB6AB8EEC00AB0EE681A21
:108720002846984735E096F8D5360BB1072184E7FF
:10873000032182E7F0EE488A82E709681268B1F9FE
:108740000810B2F9082008EE101A00EE902A032B48
:10875000B8EEC88AF8EEE00A1FD1B6F9F036DFEDC0
:10876000277ACDED030A01EE903AF8EEE11A2046A1
:1087700061EEA71ACDED021AFFF798FDDDED021AA2
:10878000DDED030AB0EE401A2846B0EE480A6CF060
:108790009DF90DB0BDEC028BF0BD072B2A680DD101
:1087A000B6F9F0369FED151A07EE903AF8EEE77A33
:1087B000D36A27EE811AB0EE480AB1E72046CDED24
:1087C000020A166BFFF772FDDDED020AB0EE401AE9
:1087D0003946B0EE480A2846B047DAE70000000004
:1087E0005047002000000034D07D0020F47D0020A0
:1087F000E87D0020FC7D0020502700200000C842BA
:10880000044B196083ED010AC3ED020A83ED031ADC
:10881000704700BF007E002038B5054675F05EFC4D
:10882000054C2061E86871F0EDFB07C804F1140302
:1088300083E8070038BD00BF007E002037B5284C14
:1088400023680546002B3FD1E86871F0DBFBD4EDCF
:10885000017A9FED247AF0EEE76AF4EEC76AF1EE52
:1088600010FA06D4D0ED026AF4EEE67AF1EE10FAD0
:1088700031DCD4ED027AF0EEE76AF4EEC76AF1EE8D
:1088800010FA06D490ED027AF4EEC77AF1EE10FAFF
:1088900021D4D4ED037AF5EEC07AF1EE10FA1DDDA5
:1088A00011491CF0EBFC68468DED000ACDED010A84
:1088B0001CF0B2FDD4ED037AF4EEC07AF1EE10FABA
:1088C0004CBF0120002007E075F008FC23692268F6
:1088D000C31A9342B8D3012003B030BD0020FBE798
:1088E000007E002000000034147E0020024B002295
:1088F0005A619A61DA617047007E002070B51E4EA1
:108900002DED028B9FED1D8A06F5A04384B0002556
:108910000446F0EE480AA3F6CC70B0EE481AF0EE2A
:10892000481AB0EE480A83F83D568DED018A8DED68
:10893000028A8DED038A70F0B1FE01A910488DED19
:10894000018A8DED028A8DED038A06F5405670F09E
:1089500071FA2A4601A90A4870F080FF294620468C
:1089600086F8D556FFF72EF901462046FFF7DEF9C7
:1089700004B0BDEC028B70BD502700200000000049
:108980008467002038B5054605480C4601F06CFFA9
:1089900000B91CB12846FFF7B1FF0124204638BDBD
:1089A00050270020F0B5064687B01F480D465CF002
:1089B00081FE044640B945F001FD0522162145F02F
:1089C000B5FA204607B0F0BD184F97F83D3613B101
:1089D0003046FFF793FF1648294670F0C5FD044660
:1089E00018B945F0EBFC0222E8E7D5ED027A97F8DA
:1089F0003D161048F8EEE76AD5ED037ACDED006A32
:108A0000B8EEE77AD5ED017A8DED017A0023F8EE24
:108A1000E77A0393049305936A4603ABCDED027A9C
:108A2000FAF7B4FDCDE700BF2847002050770020BB
:108A30008467002050270020F0B589B00222064646
:108A400004A80D4609F094FE134804A95CF032FE18
:108A5000044640B945F0B2FC0522162145F066FAFD
:108A6000204609B0F0BD0D4F97F83D3613B13046A2
:108A7000FFF744FF29460022094870F0EFFE00236B
:108A800001930293039397F83D16064801AB2A46DB
:108A9000FAF77CFDE4E700BF28470020507700206C
:108AA00084670020502700202DE9F0432DED028B34
:108AB00089B00646174604A802220D46B0EE408A49
:108AC0009846F0EE608A09F053FE1D4804A95CF058
:108AD000F1FD044658B945F071FC0522162145F018
:108AE00025FA204609B0BDEC028BBDE8F083DFF823
:108AF000609099F83D3613B13046FFF7FFFE9DF8C0
:108B00004830F0EE680A4246B0EE480A3946304630
:108B1000FFF728F975F0E2FA0A4B2946186000229F
:108B2000094870F09BFE002301930293039399F888
:108B30003D16064801AB2A46FAF728FDD1E700BFEB
:108B400028470020D07D0020846700205027002087
:108B50005077002070B52DED028B0446406990F8E7
:108B6000CB3086B03BBB012172F0FAFA606B9FED0F
:108B7000698A62680368D2ED020A5B6EB0EE480A49
:108B800001219847606B6DF043F963488DED038ACE
:108B9000F0EE480AB0EE481AF0EE481AB0EE480A75
:108BA0008DED048A8DED058A06B0BDEC028BBDE823
:108BB000704070F073BD594890F8A41D11F0010584
:108BC00000F5805651D1636A1B68A0F50050B3F9D7
:108BD0000810F9F7FDF9DFED527AB0EEC07AB4EE85
:108BE000E77AF1EE10FAB0EE408A37D429462046F3
:108BF000FFF79CF80221606972F0B2FA464870F003
:108C000033FC01464748FBF7F3FF02A9454803AA96
:108C100000F0ECFF6369029ADA636369039A9A636E
:108C2000206B6FF005FC96F8D436656BD4E906121C
:108C3000F3B91368B3F9083000EE903A0B68B3F952
:108C4000083000EE103A2B68F8EEE00ADB6AB8EE66
:108C5000C00AB0EE481A2846984735E096F8D5364F
:108C60000BB10721C3E70321C1E79FED2A8AC1E7C2
:108C700009681268B1F90810B2F9082008EE101A54
:108C800000EE902A032BB8EEC88AF8EEE00A1FD156
:108C9000B6F9F036DFED247ACDED010A01EE903A17
:108CA000F8EEE11A204661EEA71ACDED001AFFF7A3
:108CB000FDFADDED001ADDED010AB0EE401A28469E
:108CC000B0EE480A6BF002FF06B0BDEC028B70BD3F
:108CD000072B2A680DD1B6F9F0369FED131A07EE6F
:108CE000903AF8EEE77AD36A27EE811AB0EE480A96
:108CF000B1E72046CDED000A166BFFF7D7FADDEDA0
:108D0000000AB0EE401A0121B0EE480A2846B047EA
:108D1000DAE700BF00000000846700205047002011
:108D200000000034502700200000C842084B93F890
:108D30003D36032B0BD8DFE803F002040608FFF7EB
:108D400009BFFFF73FBBFFF735BCFEF751BF7047C8
:108D500050770020002070470120704701207047A5
:108D6000002070470048704790550C080048704735
:108D700098550C0808B5036B03480022C3F8542328
:108D8000FCF746FC012008BD5027002038B52C4DCB
:108D900095F8773E04469BB905F6AC50012172F078
:108DA000DFF9606B62680368D2ED020A5B6E9FEDCB
:108DB000250A01219847606BBDE838406DF028B85E
:108DC000022105F6AC5072F0CBF9A369186851F096
:108DD00059F805F55C6383ED000AE369186851F002
:108DE00051F805F6C85383ED000A636A186851F01C
:108DF00049F86268D2ED287A20EE270AB0EE0B7AA5
:108E0000C0EE077A05F55D63C3ED007A236A186842
:108E100051F038F805F6D85383ED000AA36A1868B4
:108E200051F030F805F6E45383ED000AE36A186860
:108E300051F028F805F6E85585ED000A38BD00BF69
:108E400050470020000000000020704700207047BD
:108E5000012070470120704700487047E0550C081A
:108E600000487047EC550C08044A00231370044A6C
:108E70001370044B01201880704700BF207E002033
:108E80002E7E00202C7E0020F0B50446406990F82C
:108E9000CB508BB0B5B9012172F062F960692946F7
:108EA000EEB272F079F828B1606940F2DC523146D6
:108EB00072F070FD01350C2DF0D19E4B00221A701E
:108EC0000BB0F0BD9B4D2B78042BF9D8DFE813F0E5
:108ED0000500110040005E002201974B01241C8018
:108EE000964B00221A7075F0F9F8954B2C701860AB
:108EF000E6E7002660693146F7B272F04DF828B116
:108F0000606940F2DC52394672F044FD01360C2EA5
:108F1000F0D121698A4C01F5457108461CF0ACFD81
:108F2000DFED887AB4EEE70AF1EE10FA02DD75F0B3
:108F3000D5F8206075F0D2F8236803F5FA739842EB
:108F4000BED902232B7075F0C9F87F4B1860B7E7C4
:108F500075F0C4F87C4B1B6803F5FA73984212D283
:108F6000754B60691A88754B02EB8202C2EB0212E4
:108F7000920002F2DC52197812B272F00BFD002856
:108F80009ED1042300E003232B7099E72369DFEDD2
:108F90006F5AD3EDC57ADFED6E6A674F93EDC66AFF
:108FA00093EDC77AB7F90010644EF4EEE57AF1EE6E
:108FB00010FAF4EEE67ACCBF01220022F1EE10FAAC
:108FC0004CBF01230023D21AB4EEE56A4A43F1EE06
:108FD00010FAB4EEE66A07EE902ACCBF0122002216
:108FE000F1EE10FA4CBF01230023D21AF8EEE77A13
:108FF0004A43CDED017A07EE902AF8EEE77ACDEDFF
:10900000027AF6EE007AB4EEE77AFEEE007AF1EE3E
:1090100010FAB4EEE77ACCBF01230023F1EE10FA88
:109020004CBF012200229B1A4B4307EE903AF8EE08
:10903000E77A3178CDED037A71F094FF07A901A8A2
:109040008DED070ACDED080A8DED091A1CF022FC02
:10905000F8B12046FDF7A2FC33783E4A01330621E1
:1090600048F0B8FA3178606901231944C9B22B700D
:1090700031703B8071F090FF00287FF421AF04260F
:1090800020462E70FDF78AFC334A314648F0A2FA9A
:1090900016E701A81CF038FC317860698DED040AF0
:1090A000CDED050A8DED061A71F05CFF07A904A845
:1090B0008DED070ACDED080A8DED091A1CF0EAFBCB
:1090C00070B12046FDF76AFC3378244A013306214B
:1090D00048F080FA31786069012271F065FFC1E7DC
:1090E0002046FDF75BFC1E4A062148F073FAB7F9EB
:1090F0000030013309D12046FDF750FC3378194A7E
:109100000133042148F066FA3BE74FF6FF733B80DA
:10911000012339E7144B082293F8851D2046FDF7FB
:1091200037FC1248012216210BB0BDE8F040F8F7D9
:109130000BBB00BF2E7E00202C7E0020207E002056
:10914000247E00200AD7233C287E0020CDCCCC3EB4
:10915000CDCCCCBEF4550C088E560C0807560C0826
:109160002B560C085C560C0850470020C85D0020A8
:109170000020704700207047012070470120704791
:1091800000487047F8560C080048704700570C0814
:1091900070B52DED028B84B0044674F09FFF064637
:1091A00060696C4D90F8CB3003BB012171F0D8FFA2
:1091B000606B62680368D2ED020A5B6E0121B6EE55
:1091C000000A9847606B6CF023FE206B6EF074FE13
:1091D000206BB6EE000A6FF0B9F82369D3F80032BD
:1091E000C5F8843304B0BDEC028B70BD022171F070
:1091F000B7FFE36A186850F045FEA36A1868B0EE3E
:10920000408A50F03FFE0023A5F5A040F0EE408AD2
:109210000093019301F028FB00287AD09FED4E7A4D
:10922000F0EEC87AF4EEC77AF1EE10FA06DCF0EE52
:10923000E87AF4EEC77AF1EE10FA02DD206B6EF0F8
:109240003BFE464801AA694600F05CFD206B6EF0CB
:10925000B1FE9DED010A636970EE288A9DED000A5A
:10926000C3ED0E8A30EE088A636983ED0F8A636A64
:109270001868438A828907EE903A394BF8EEE77A0C
:1092800093ED007A67EE877AFCEEE77A17EE903A74
:1092900099B250F08DFD01463048F8F799FE314BF8
:1092A0002E48B3F92C3101EE103AE3691B68B3F98B
:1092B000083000EE903AA3691B68B3F90830B0EEAD
:1092C000408A00EE103AB8EEC11AF8EEE00AB8EEA5
:1092D000C00A03AA02A9F8F711FEDFED237A606B3A
:1092E000B0EEC87AB4EEE77AF1EE10FA15D403685E
:1092F000DDED030ADB6A9DED020AB0EE481A9847DD
:109300002369D3F80032C5E9E1362046FDF72CFD8C
:1093100068E7206B6EF0D0FD9BE7D5F888330268D4
:109320009DED020ADDED030AFA33B34209D9D36A8F
:109330009FED0E1A98472369D3F80032C5F884339D
:10934000E3E795EDE11A136BB8EE411A0121984756
:10935000DBE700BF50770020CDCCCC3D502700206C
:109360000C5E002050470020000000340000000088
:10937000F8B504462DED028B3E4801F075FA06461D
:10938000002873D03C4DDFED3D8AD5ED170A9FEDE7
:109390003C8A95ED130A206BF4EEE80AF1EE10FA20
:1093A000B8BFF0EE480A6DF015FDD5ED170A95ED42
:1093B000130A206BF4EEE80AF1EE10FAB8BFF0EEF3
:1093C000480A6DF07FFDA5F58040276BF8F798FE01
:1093D0006368B3F93020B3F92C3000EE903A434281
:1093E00001EE102A00EE103AB8EEC11AF8EEE00ACB
:1093F000B8EEC00A38466DF035FEA5F58040276B03
:10940000F8F77EFE6368B3F93020B3F92C3000EE34
:10941000903A434201EE102A00EE103AB8EEC11A1B
:10942000F8EEE00AB8EEC00A38466DF095FE206B03
:109430006EF042FD206B6EF00DFF606B626803689A
:10944000D2ED020A5B6E0121B6EE000A9847606B0E
:109450006CF0DEFC206BB6EE000A6EF077FF23693D
:1094600005F58055D3F80032C5F88433BDEC028B86
:109470003046F8BD5027002050670020000000341F
:1094800000007A4300207047012070470120704798
:10949000002070470048704748570C080048704744
:1094A00054570C08036B0022C3F854230369D3F804
:1094B0000022024B0120C3F884237047507700201C
:1094C00073B5044674F00AFE06466069524D90F882
:1094D000CB30B3B9012171F043FE606B6268036861
:1094E000D2ED020A5B6E9FED4D0A01219847606B39
:1094F0006CF08EFC2369D3F80032C5F8843302B0D7
:1095000070BD022171F02CFEA5F5405301AAB3F9FC
:109510002C3101EE103AE3691B68B3F9083000EE14
:10952000903AA3691B68B3F9083000EE103AB8EE20
:10953000C11AF8EEE00AB8EEC00A6946A5F5A040E7
:10954000F8F7DCFC636A1868438A828907EE903A70
:10955000A5F5CA5313ED017AF8EEE77A67EE877A3C
:10956000FCEEE77A17EE903A99B250F021FC0146F2
:10957000A5F5A040F8F72CFDDFED297A606BB0EE81
:10958000C07AB4EEE77AF1EE10FAB0EE401A27D4C2
:109590000368DDED010ADB6A9DED000A9847236947
:1095A000D3F80032C5E9E136656B2B685E6E236A3D
:1095B000186850F067FC63680021D3ED020A284662
:1095C000B047A36A6569186850F05CFC85ED0E0A27
:1095D000E36A6569186850F055FC85ED0F0A8EE75F
:1095E000D5F8883302689DED000ADDED010AFA33F3
:1095F000B34209D9D36A9FED091A98472369D3F872
:109600000032C5F88433CFE795EDE11A136BB8EE5D
:10961000411A01219847C7E7507700200000000059
:10962000000000340120704700207047012070477F
:1096300001207047004870479C570C08004870474D
:10964000A4570C0837B5436993F8CB200446D2B928
:109650001A681846926A90476069012171F080FD8E
:10966000606B62680368D2ED020A5B6E9FED360A9A
:1096700001219847606B6CF0CBFB206B03B0BDE819
:1096800030406EF0E7BD314D95F9803D002B03DA97
:109690001B220221FDF77CF9B5F92C312C482D4D08
:1096A00001EE103AE3691B68B3F9083000EE903A16
:1096B000A3691B68B3F9083000EE103A01AAB8EEAE
:1096C000C11AF8EEE00A6946B8EEC00AF8F716FCCF
:1096D000636A1F481B68B3F90810F8F779FC606BE0
:1096E000DDED010A0368B0EE401ADB6A9DED000A69
:1096F0009847236B95ED140A93EDC31AF7EE000A11
:109700003320B0EEC00A19F07FFDFDEEC07AA5F55A
:10971000805517EE903AA5F8F430206B6DF028FDD7
:10972000206B6EF085FEA36A6569186850F0AAFB8D
:1097300085ED0E0AE36A6569186850F0A3FB85EDB4
:109740000F0A03B030BD00BF0000000050470020EA
:10975000502700205067002070B504461D48F8F7D8
:1097600051F90546A0B31B48266BF8F7C9FC63689E
:10977000B3F93020B3F92C3000EE903A434201EEB9
:10978000102A00EE103AB8EEC11AF8EEE00AB8EE70
:10979000C00A30466DF066FC0E48266BF8F7B0FC48
:1097A0006368B3F93020B3F92C3000EE903A4342AD
:1097B00001EE102A00EE103A3046B8EEC11AF8EE6B
:1097C000E00AB8EEC00A6DF0C7FC206B6EF042FDF7
:1097D000284670BD5027002000487047EC570C0801
:1097E00000487047F8570C0810B50446FCF7FEFD1A
:1097F000054B2360054BE363002384F840300023CE
:109800006364204610BD00BF20590C08000080BFD3
:10981000034BC3639FED030A03486DF0CFBD00BF48
:10982000000080BF000000007063002037B50546CF
:10983000FDF740F9044660B12846FFF7E9FF1548F7
:1098400000F082FD054638B9134A1448062147F056
:10985000C1FE204603B030BD1148124C70F0D6FB5B
:10986000D4ED507AB4EEE70AF1EE10FA0FDB9FED7B
:109870000E7A67EE877A17EE900AF6F745FE0B4AE6
:10988000CDE90001042104F6583047F0A3FE2C4630
:10989000DFE700BF5027002000580C08A852002026
:1098A000505E0020504700200AD7233C22580C0865
:1098B00030B5374C2DED028B94F8843D152B83B0D9
:1098C0000546B0EE408A06D0324A042104F65830EC
:1098D00047F080FE1AE004F5B85070F097FBD4ED25
:1098E000507AB4EEE70AF1EE10FA14DB9FED2A7A13
:1098F00067EE877A17EE900AF6F706FE274ACDE95B
:109900000001042104F6583047F064FE2846FFF7B2
:109910007FFF002036E0B4F99C3907EE903AF8EE6C
:10992000E77AF4EEC87AF1EE10FA01DD1C4ACCE7D2
:10993000B4F99E3907EE903AF8EEE77AF4EEC87A79
:10994000F1EE10FA22D4DFED147A85ED0F8A68EE7D
:10995000277A17EE900AF6F7D7FD124ACDE90001F3
:10996000062104F6583047F035FE04F5B85070F083
:109970004DFBD5ED0F7A04F5E15030EE670A6DF03E
:109980001DFD012003B0BDEC028B30BD064A9CE7F3
:109990005047002048580C080AD7233C6F580C0841
:1099A000A1580C08CB580C08ED580C0838B50446E3
:1099B0002DED028B1C4800F0C7FC90B3D4ED0F7A5C
:1099C0001A4DF5EEC07A05F6A813F1EE10FA93EDF4
:1099D000008A0FDC05F6A41393ED000AD5ED507A4A
:1099E000B4EEE70AF1EE10FA04D530EE480A20464C
:1099F000FFF75EFFD4ED0F7AF5EEC07AF1EE10FAC4
:109A00000FDD78EE277A95ED507A094BF4EEC77AA0
:109A1000F1EE10FAA4BF77EE677A38EE278A83ED6D
:109A2000008ABDEC028B38BD502700205047002033
:109A30001467002030B52DED028B036A1B68B3F963
:109A4000083000EE103A83B00446B8EEC00A484829
:109A5000F8F768FB46488DED010AF8F751FB63689B
:109A60009DED010AB3F92C3001EE103A434200EEAD
:109A7000903AB8EEC11AF8EEE00A6B2019F0C4FB78
:109A8000DFED3C7AB0EEC07AB4EEE77AF1EE10FA90
:109A9000B0EE408A58D594F8403083B1E068D4EDF8
:109AA0000F8A70F0B3FAD4ED117A38EE800A2046AE
:109AB00030EE670AFFF7FCFE002384F840302E4B9F
:109AC00093F8802D93F9803D002B22DA6268236B96
:109AD000D2ED2D7A93EDD57AF1EE046A77EEE67A3F
:109AE000F4EE477AF1EE10FAC8BFF0EE477AC3ED14
:109AF000D57A2046FFF78CFE206BB0EE480A6DF059
:109B000037FB206B03B0BDEC028BBDE830406EF03C
:109B10008FBC530614D5E068256B70F077FA236B81
:109B2000F2EE047A30EE270AD3EDD57AB4EE670A66
:109B3000F1EE10FAC8BFF0EE407AC5EDD57AD8E75D
:109B40002046FFF733FFD7E7D4ED0F7AF5EEC07A62
:109B5000F1EE10FAD0DD94F84030002BCCD1E06863
:109B600070F054FA012384ED110A84F84030C3E701
:109B700050270020CDCC4C3D5047002010B5044666
:109B8000FCF7E2FF2046FFF755FF2046BDE81040F6
:109B9000FDF7D8B838B5044604F5A04574F09EFA30
:109BA000D5F8943303F5FA7398421BD904F52D5078
:109BB00004F500540C4A0621183047F00BFD94F8C8
:109BC000803D6FF3C30384F8803D6AF0CFFA0368E9
:109BD00001229B680321984774F080FAC5F890032E
:109BE000002038BD0120FCE758590C0870B52DED58
:109BF000028B00F5804300F500545B6CD3EDCF7A07
:109C0000D3EDD08AFDEEE77A1546B4F92C2117EE94
:109C1000903A0E46F1EE688A5142FDEEE88A09B2AA
:109C200018B219F02FFBB4F92C2118EE903A5142DA
:109C300008EE100A09B218B219F024FBB4F92C315D
:109C400007EE903AB8EEC88AF8EEE77A88EE277AFF
:109C5000BDEC028B07EE900A86ED007AB4F92C3148
:109C6000B8EEE77A07EE903AF8EEE77AC7EE276AA1
:109C7000C5ED006A70BD000070B52DED028B00F5DA
:109C8000804300F50054D3F85439D3EDCF7AD3EDA7
:109C9000D08AFDEEE77A1546B4F92C2117EE903AFA
:109CA0000E46F1EE688A5142FDEEE88A09B218B21A
:109CB00019F0E8FAB4F92C2118EE903A514208EE66
:109CC000100A09B218B219F0DDFAB4F92C3107EE16
:109CD000903AB8EEC88AF8EEE77A88EE277ABDECBB
:109CE000028B07EE900A86ED007AB4F92C31B8EEBB
:109CF000E77A07EE903AF8EEE77AC7EE276AC5ED05
:109D0000006A70BD70B52DED028B00F57053D3ED78
:109D1000D77AD3EDD88A00F50054FDEEE77A1546E0
:109D2000B4F92C2117EE903A0E46F1EE688A5142B2
:109D3000FDEEE88A09B218B219F0A4FAB4F92C21A0
:109D400018EE903A514208EE100A09B218B219F012
:109D500099FAB4F92C3107EE903AB8EEC88AF8EEC9
:109D6000E77A88EE277ABDEC028B07EE900A86ED43
:109D7000007AB4F92C31B8EEE77A07EE903AF8EEB3
:109D8000E77AC7EE276AC5ED006A70BD00F5365068
:109D90002C3070F075BA000070B5044674F09EF96E
:109DA00004F5A043D3F8902302F51C5310338342EB
:109DB0000AD94AB1164A04F52D500221183047F04D
:109DC00009FC0025284670BD124B1B68D86A036841
:109DD000DB699847012801D10F4AECE704F50056EA
:109DE00096F8775E3DB904F52D500C4A04211830E1
:109DF00047F0F0FBE6E704F536502C3070F040FAFF
:109E000096F8803D43F0080386F8803DDAE700BF0E
:109E100070590C08482700209D590C08D2590C088D
:109E200084B070B52DED048B84B004460DA880E895
:109E30000E0074F053F904F5A04304F50055C3F87F
:109E4000940395F8803D1B071DD44A4E74F046F9E3
:109E5000336803F5FA6398420DD92046FFF79CFF5B
:109E600088B904F52D50444A0421183047F0B2FB5C
:109E700074F034F93060002004B0BDEC048BBDE810
:109E8000704004B07047129802280CD0F6F71AFB05
:109E9000CDE9000104F52D54384A18340421204638
:109EA00047F098FBE7E79DED0E0A9DED0D8A8DEDDD
:109EB000030AF0EE000ADDED0F8A19F0A3F89DED1C
:109EC000030A50B110EE100AF6F71EFB04F52D54EC
:109ED000CDE900012A4A1834E0E7F7EE000A8DEDDB
:109EE000030A19F08FF89DED030AA8B1FDEEE88A88
:109EF000FCEEC87A18EE903ACDED037A04F53650B0
:109F00009DF80C101AB22C3004B0BDEC048BBDE8E7
:109F1000704004B071F03EBDDFED1A0A19F072F81E
:109F20000028A8D09FED189ADFED160A8120B0EE28
:109F3000491AB0EE680A19F067F9C0EE096AD5F857
:109F40006429B2F90A30B2F90E20D21A07EE902A2B
:109F5000B8EEE77A07EE903AF8EEE77AE6EE877A1F
:109F6000BCEEC87AFDEEE77A8DED037A17EE903AF3
:109F7000C4E700BF307E0020F4590C08165A0C08C4
:109F80002A5A0C08000000000000C84238B500F54D
:109F90000053044693F8842D142A1DD093F8802D85
:109FA000120703D5BDE83840FFF7F4BD012283F85E
:109FB000782E51F0EFFB054651F082FB51F016FB75
:109FC00050F00CFF04F536502C3072F08FFC284610
:109FD000BDE8384051F07CBB38BD000010B50446E8
:109FE0000020FBF78BF904F50054C4F86009012048
:109FF000FBF784F9C4F85C090220FBF77FF9C4F889
:10A0000064090320FBF77AF9C4F868090420FBF718
:10A0100075F9C4F86C090520FBF770F941F2941149
:10A02000C4F87009D4F85C094FF096FED4F86009C2
:10A0300041F294114FF090FED4F8680941F2941166
:10A040004FF08AFED4F864094FF47A714FF080FE25
:10A05000D4F86C0941F294114FF07EFED4F87009E7
:10A0600041F294114FF078FED4F85C091E214FF0B4
:10A0700077FED4F860091E214FF072FED4F864090F
:10A080001E214FF06DFED4F8680928214FF068FEBC
:10A09000D4F86C091E214FF063FED4F870091E211C
:10A0A0004FF05EFE0024E0B2002240F2DC510134A9
:10A0B0004FF054FD062CF6D12046002240F2DC5130
:10A0C0004FF04CFD002240F2DC5107204FF046FDDE
:10A0D0000820FBF713F90022B0F90A1008204FF00E
:10A0E0003DFD0920FBF70AF90022B0F90A1009200A
:10A0F0004FF034FDBDE81040002240F24C410A20F0
:10A100004FF02CBD37B5044604F5005500F5365028
:10A110002C30B5F87211019071F010F995F8E81132
:10A120000198002271F0F6F8D5F864390198B3F976
:10A130000A10B3F90E2072F0FFFB019872F0FEF9DD
:10A1400004F5595001213830F7F7EEF910B12046E7
:10A15000FFF71CFE03B0BDE8304050F0A1BF000087
:10A1600013B5044600F51C70019005F07BFA94F8D5
:10A1700081320198242202FB0343D3EDA77AF5EE46
:10A18000C07AF1EE10FA02DD05F030FA019804F51C
:10A19000005494F8813DDB0709D594F8A91D05F01A
:10A1A00015FA94F8A83D60F3000384F8A83D02B0C6
:10A1B00010BD000037B5102300F6F8350446C0F88E
:10A1C000A43E192128463BF0F7FF04F526504FF036
:10A1D0007A5301A92C30019304F5005446F03AFE5D
:10A1E000192128463BF0A6FB94F8983960F3000348
:10A1F00084F8983903B030BDF0B52DED028B00F630
:10A20000F83683B0054630463BF04EFC1921304607
:10A210003BF0B6FB1921074630463BF081FB042892
:10A2200005F5005472D0002094F8983960F341038A
:10A2300084F89839192130463BF092FBA4F89A092A
:10A2400005F55C506FF0E2FE04F6A41383ED000AFE
:10A25000192130463BF0AAFB1921A4F89C0930468D
:10A260003BF09AFB94F89839A4F89E099B0728D5EF
:10A2700073F034FFD4F8A0390646F31AB3F57A7FA9
:10A28000B4F99A3907EE903A05F52650F8EEE77AD8
:10A2900000F12C004BD901A9CDED017A46F04AFD21
:10A2A0002748C4F8A0690346083093ED008A46F0B9
:10A2B0003FFDD0ED007A78EE677A04F6A813C3ED7F
:10A2C000007A94F8983904F6A81405F580402268BD
:10A2D00000F6F404C3F30006C3F3400113F00103D6
:10A2E00080F8EE6880F8F018226004D090F9EF381A
:10A2F000003B18BF012380F8993980F89A1900F6BD
:10A300004810426503B0BDEC028BF0BD1921304608
:10A310003BF068FB022886D97A1C06D094F93C31C0
:10A32000BB42CCBF002001207EE701207CE7054B2B
:10A33000CDED007A01AA6946019346F08FFDAFE7A3
:10A34000F4500020CDCC4C3D10B5044673F0C6FE51
:10A3500004F5005393F8982912F001010BD0C2F3D1
:10A360004001920707D5D3F8A039C01AB0F57A7F1B
:10A370002CBF00210121084610BD000008B500F5E2
:10A38000005090F8803DB1EBD31F13D061F3C71399
:10A39000094A80F8803D00211B06116006D544F073
:10A3A0000DF8A321BDE8084043F0A0BD44F006F835
:10A3B000A421F7E708BD00BF387E002008B500F5EE
:10A3C000005090F8803DC3F380128A4213D061F3AD
:10A3D0008613094A80F8803D00215B06116006D58E
:10A3E00043F0ECFFA521BDE8084043F07FBD43F0FA
:10A3F000E5FFA621F7E708BD347E002070B500F523
:10A40000005586B095F8771E044649B90191FFF7CB
:10A41000B5FF0199204606B0BDE87040FFF7CEBFFA
:10A4200000F58850002303A9083003930493059393
:10A4300002F0F0FDDDED057A9FED3E7AF4EEC77A8D
:10A44000F1EE10FA47DD9FED3C7AF4EEC77AF1EEBB
:10A4500010FA4CBF0126002695F8813DDA0744D555
:10A4600095F8A83DDB0740D594F8813295ED796ADF
:10A47000DFED326A242202FB034393EDA77A95F9BC
:10A48000803D002BC6EE267A27DADFED2B6A77EEC9
:10A49000E67AF4EEC77AF1EE10FA4CBF0121002102
:10A4A0002046FFF76BFF95F8B33D002B3FD0002E01
:10A4B0003DD0234A136807EE903AB8EE677ADFED95
:10A4C000217AB4EEE77AF1EE10FA1FD4012120468A
:10A4D000FFF774FF21E00026BEE7B4EEE77AF1EE65
:10A4E00010FACCBF01210021DAE7E6B195F8B43DBE
:10A4F000ABB1154A136807EE903AB8EE677ADFED14
:10A50000117AB4EEE77AF1EE10FA02D50133136056
:10A5100003E001212046FFF731FF06B070BD95F83A
:10A52000B33D002BC5D100212046FFF727FF0021B6
:10A53000CDE700BFCDCC4CBDCDCC4C3D0000C842DA
:10A54000347E00200000C843387E0020F9F74EB862
:10A550000148FAF769BB00BF5027002038B500F565
:10A56000885508350446284601F00CFC04F5805354
:10A57000042283F81C23002283F81124B4F9A430A8
:10A5800004F5B2601BB9B4F8A230A4F8A430B4F852
:10A59000A41018F097F92846BDE8384001F0ECBC4B
:10A5A0002DE9FF41044600F58550183036F0BCF81F
:10A5B00004F5445004F51C76043005F011FD3046D6
:10A5C00005F092FBB7EE000A7B483AF0C5FA94F822
:10A5D0000D337A4800EE103AB8EE400A3AF0BCFA71
:10A5E00004F52D5018304BF035FA4FF06DFB9922E1
:10A5F000292150F033FB4FF067FB4FF00DFB204655
:10A60000FFF7ECFC2046FFF77DFD2046FAF786FFBA
:10A6100004F58450043056F033F9694B69491B68DE
:10A62000986A03684FF47A72DB6A98470423C4F887
:10A630005C3104F590700FF0DFFB08F0C1FB4FF4C4
:10A640000053436208F0BCFB04F5805709F000FC9E
:10A65000802504F52C504FF400611430C7F8585F82
:10A6600037F0B6FA04F594402030019004F58048A4
:10A6700052F062FB9FED541A98F8991A0198F0EE87
:10A68000410AB0EE410A002251F0FAFE032298F886
:10A69000991A019851F0E0FE04F59340203006F03D
:10A6A00003FF00213046C4F8845205F0E7F8304635
:10A6B00004F0D8FF94F880C2002304F5217024220E
:10A6C0005FFA83F8C44520D903FB02215D1C415C7D
:10A6D00001296CD104F5005502A904F543708DF8E9
:10A6E00008303AF023FD95F8813D85F8A98D43F0B7
:10A6F000010385F8813D4146304604F067FF95F837
:10A70000A83D60F3000385F8A83D04F5005504F565
:10A71000885695F8813D13F0010306F108060DF106
:10A72000080846D1414604F543708DF808303AF0E8
:10A73000FDFCB2EE040A304602F008FC04F5255098
:10A7400034306FF0A3FC04F5A043D7F80823C3F816
:10A7500084232046FFF72EFD04F52650383051F0B3
:10A76000B3F904F528501C301DF0B6F94FF480738E
:10A77000C5F8103B154B0293154B039398E8060060
:10A7800004F6A86042F0FAFD2046FFF7E7FE2046F7
:10A79000FAF734F94FF40023C4F8803A95F8803D75
:10A7A00043F0100385F8803D04B0BDE8F0812B46EE
:10A7B00086E79FED080ABEE7445A0C08515A0C0878
:10A7C0004827002051A50108000000005027002064
:10A7D0004DA50108CDCCCC3D13B5044600F58850FD
:10A7E000083001F0E1FC88B104F55C5004F5005438
:10A7F0006FF0FEFB94F8772E0190C3B2C0F3001007
:10A8000032B918B99DF80500C0F3400002B010BD80
:10A810000028FBD083F08000C009F7E737B5044675
:10A8200000F58850083001F0BFFC80B104F50055F8
:10A8300095F9190B58B104F55C506FF0D9FB95F8F8
:10A84000773E01902BB99DF8050000F0010003B0A0
:10A8500030BD9DF804301A07C3F3C00044BF83F035
:10A860008000C009F3E7000010B500F5005304466E
:10A8700093F8A43D5B0707D4FFF7AEFF28B9204645
:10A88000BDE81040FFF7CABF002010BD37B500F685
:10A89000A865044604F500542846019142F0B6FE2E
:10A8A00094F8803D019960F34103284684F8803D87
:10A8B00003B0BDE8304043F0A7BB00000020704764
:10A8C0000020704737B500F59545383504462846D1
:10A8D00041F04CF9012201A9284641F0C7F820B106
:10A8E00004F6F834019BC4F89C3203B030BD00007C
:10A8F00010B504210446FFF7C9FF30B104F59540B7
:10A900003830BDE8104041F07FB910BD00F58053EC
:10A91000D3EDC57A9FED227AF5EEC07AF1EE10FA0A
:10A9200004DBF4EEC77AF1EE10FA17D4F4EEC77A2E
:10A93000F1EE10FA14DC9FED1B7AF4EEC77AF1EE1B
:10A9400010FA4CBF0223032300F5405090F8B826BC
:10A95000032A0ED8DFE802F006161B1F0023F3E7D8
:10A960000123F1E7012B07D1D0F8B4260132C0F85A
:10A97000B42680F8B8367047032BFAD1D0F8B42645
:10A98000013AF4E7022BEFD0002BF7D0F1E7032BCD
:10A99000EAD0012BF1E7002BE6D0022BEDE700BF58
:10A9A000DB0FC93FDB0FC9BF13B50446143000F0FD
:10A9B000C1FD04F12C0000F0BDFD04F1740075F040
:10A9C000BFF904F1F40075F0BBF94FF0FF331549FE
:10A9D000C4F85031204639F017FD00230DF107016E
:10A9E00004F128008DF807303AF072FB01230DF1D5
:10A9F000070104F129008DF807303AF069FB0F23B5
:10AA00000DF1070104F125008DF807303AF060FBE5
:10AA1000054B1A6812B1054873F02EFB20461C60E6
:10AA200002B010BD0C5C0C083C7E00205C5A0C0887
:10AA30002DE9F0478CB003A938F018FE60B300216F
:10AA40000D2208A807AF1C4CDFF87080DFF870906B
:10AA500007910B26A1F062FA0697237ADFF864A02B
:10AA60008DF81430002554F825300493D8F80000F0
:10AA7000E368B5B90093C06A53461122394614F011
:10AA8000B5FD0021B7EE000A03A838F0F3FF35B199
:10AA9000013E04F11004E0D10CB0BDE8F0870125BF
:10AAA000E1E701930223009311224B463946C06A25
:10AAB00014F09CFDE5E700BFAC5C0C0848270020C3
:10AAC000B95A0C08B05A0C082DE9F04F2DED028B45
:10AAD000D0F8543183B0044693BB9FED7E8ADFF8F3
:10AAE00000A2074600F1740800F5AA750126721E3F
:10AAF000D2B297ED070A0192404675F041F9FB6921
:10AB0000C8F83C304FF07E53C8F8483097F92830E9
:10AB1000019A013B5FFA86FB0E2B22D8DFE803F097
:10AB200015414D5A636C7D218B959FAA21C5B500B7
:10AB3000D4F8543103B96361D4F8583103B9E362EE
:10AB400003B0BDEC028BBDE8F08F4820019207F006
:10AB500069FE814618B1019A214673F0EDFFC5F8F0
:10AB60000090286898B103689B689847002840F0D7
:10AB7000AA804DF0D5FB584A3346032146F02AFD02
:10AB8000286810B103685B68984700232B60022E89
:10AB900007F1180708F1800805F10405C8D002265E
:10ABA000A5E72820019207F03DFE81460028D6D077
:10ABB000019A214675F0ACF8D1E76820019207F0C0
:10ABC00031FE81460028CAD0FF23019A214674F045
:10ABD00055FAC4E76820019207F024FE8146002858
:10ABE000BDD00023F1E76820019207F01BFE8146EB
:10ABF0000028B4D00123E8E74420019207F012FEB8
:10AC000081460028ABD0019A214673F0E5FBC9F8D4
:10AC100000A00023C9F84030A1E74820019207F0C6
:10AC200001FE814600289AD0B1EE040A019A21461D
:10AC300073F070FC93E74820019207F0F3FD814622
:10AC400000288CD0B2EE040AF0E74820019207F009
:10AC5000E9FD8146002882D0B3EE040AE6E74820E9
:10AC6000019207F0DFFD814600283FF478AFB3EE94
:10AC70000E0ADBE74820019207F0D4FD8146002848
:10AC80003FF46DAFB0EE480AD0E74420019207F0E0
:10AC9000C9FD814600283FF462AF019A214673F056
:10ACA0009BFB0E4BC9F80030B3E73420019207F04C
:10ACB000B9FD814600283FF452AF019A0023214696
:10ACC00074F0B6FC4BE72B68002B3FF460AF84F8C0
:10ACD0004FB15CE700007042965A0C0898A90D0825
:10ACE0001CAC0D0813B50446FFF7A2FE204638F051
:10ACF00013FE68B994F9283013B994F940303BB188
:10AD000001230DF1070120468DF807303AF00EFAC5
:10AD100094F90030002B08DD94F928302BB120463F
:10AD200002B0BDE81040FFF7CFBE02B010BD00007A
:10AD30000346406C012807D0032805D0986C0128F1
:10AD400002D0032818BF02207047000070B590F9A8
:10AD50000030002B04460D4611DD0B78012B0ED878
:10AD6000D0F8540110B10368DB699847D4F8580152
:10AD700028B103682946DB69BDE87040184770BDFB
:10AD800090F90030002B0ADD012908D8182303FBB5
:10AD9000010090F92800003818BF012070470020FA
:10ADA0007047000037B50446FFF7EAFF9FED0B0A36
:10ADB0000D4680B104EB81038DED010AD3F85401F7
:10ADC00038B1036801A9DB68984704EBC51484F81F
:10ADD00065009DED010A03B030BD00BF000000001A
:10ADE00070B50446FFF7CCFF50B104EB8104D4F8F2
:10ADF000540128B10368BDE870401B69114618472B
:10AE0000002070BD2DE9F04F2DED028B90F9003040
:10AE1000002B83B00646894653DD2C4B1B68D86A4D
:10AE200003685B689847044650B14DF079FA284AA8
:10AE3000062103B0BDEC028BBDE8F04F46F0CABB63
:10AE40009FED248ADFF890A0DFF890B0354606F138
:10AE50004407B04621463046FFF792FF20B195F8EF
:10AE6000643043B188ED068A8035043708F118084C
:10AE70003CBB0124EEE7B9F1000F03D098F926306E
:10AE8000002BF1D1D7F81021631C01933AB94DF092
:10AE900047FA019B5A46032146F09CFBE4E773F016
:10AEA0001DF90022A5F87020A5F872200122A866DD
:10AEB00085ED1B8A3A604DF033FA019B524606211C
:10AEC000EAE703B0BDEC028BBDE8F08F4827002015
:10AED000C45A0C0800000000025B0C08DB5A0C0886
:10AEE0002DE9F0432DED028B85B004460D46B0EE02
:10AEF000408AFFF745FF98B304EBC119CF01D9F899
:10AF000068306BB373F0EAF8D9F86830C01AB0F55E
:10AF10007A7F03D3B9F872300F2B0CD8E31993F86A
:10AF20006520002A40F08C803C44B4F87230013334
:10AF3000A4F8723014E0B9F8703005F1010805F199
:10AF4000100693B94DF0ECF904EB86064346454AEA
:10AF5000042146F03FFB032373603C440023A366B7
:10AF600005B0BDEC028BBDE8F08307EE903AD9ED59
:10AF70001B6AD4F85C21F8EEE77A86EEA77A8DEDAD
:10AF8000037ACAB394F90230002B35DD07EE903A0C
:10AF9000B2F90C209FED345AF8EEE75AF7EE007A3A
:10AFA000E5EE857A182101FB054506EE902AF8EEBC
:10AFB000E66A95ED066A67EEA67A37EE467A67EEA0
:10AFC000A77AB0EEC77AE6EEE67AF6EE006A67EEAA
:10AFD000A67AF4EEC77AF1EE10FA0DD5B0EEC66A95
:10AFE000B5EEC06AF1EE10FA06DD4DF099F91F4A90
:10AFF0004346042146F0EEFA182003A900FB08405E
:10B0000004EB86063AF028F8022373606368DB06D7
:10B010000ED54DF085F905460398F5F775FA144AF3
:10B02000CDE9000143460621284646F0D3FA94E7CD
:10B030004DF076F90F4A4346062146F0CBFA8CE7ED
:10B04000B3F87220052A7FF66FAFD3ED1B7AB3F801
:10B05000702037EE880A013283ED1B0AA3F87020B6
:10B0600062E700BF245B0C080AD7233C3A5B0C085C
:10B07000675B0C088E5B0C0810B590F90030002B54
:10B0800002460C461CDD90F84D31CBB9FFF778FE37
:10B09000A8B1182101FB042292F9243093B1022BAC
:10B0A0000DD146204FF094FFDFED077AB0EEC00AD5
:10B0B000B4EEE70AF1EE10FA4CBF0120002010BDFB
:10B0C0000020FCE71846FAE7000000342DE9F843B9
:10B0D0002DED028B04460E46FFF752FEE8B104EB5D
:10B0E00081090DB2D9F85431BBB172F0F7FF04EB0E
:10B0F000C6174FEAC6183866D9F8540103685B6969
:10B10000984770B1D9F85401036839469B695031AA
:10B1100098473B6D87F86500FB64BDEC028BBDE88A
:10B12000F8833146204697F86590FFF73BFE1823D9
:10B1300003FB064393ED068ABB6E30EE488A87ED2B
:10B14000178A1BB131462046FFF7CAFEB9F1000F3E
:10B1500043D0DFED447A9FED447A04EB080368EEB8
:10B16000277AD3ED166AE6EE877A182104EB0807F2
:10B1700001FB0646C7ED167A96F9273083B3012BFB
:10B1800053D1DFED3A8AF1EE487A05EB4505B4EE8E
:10B19000E88AC7ED157A04EBC505F1EE10FA95EDD6
:10B1A000070A58BFF0EE687A27EE800A9EF006FE86
:10B1B00087ED130A97ED160AB4EEE80AF1EE10FADD
:10B1C00048BFF1EE408A95ED070A28EE800A9EF00E
:10B1D000F5FD444484ED140A9FE7F0EE487AC4E795
:10B1E000B5EEC08A05EB4505F1EE10FA87ED158A3C
:10B1F00004EBC505D8BF9FED1D8A95ED070A28EE23
:10B20000000A9EF0DBFD04EB0803D3ED167A83ED14
:10B21000130AF5EEC07AF1EE10FAD8BFDFED137A1B
:10B2200095ED070A27EE800AD1E7B0EEC88A05EB54
:10B23000450587ED158A04EBC50494ED070A28EE51
:10B24000000A9EF0BBFDD7ED167A87ED130A94ED48
:10B25000070AF0EEE77A27EE800A9EF0AFFD87ED51
:10B26000140A5AE79A99993E3333333F000000009D
:10B2700038B50A460446FFF783FD10B304EBC1134B
:10B28000CD0193F8653033B104EB8103D3F8543129
:10B29000003B18BF0123182101FB0242D2ED067AC0
:10B2A000F0EEE77AF5EEC07AF1EE10FA08DC2C4405
:10B2B00094F8640020B992F92600003818BF0120E4
:10B2C000184038BD10B500210446FFF759FD18B1EC
:10B2D0002046FFF7CDFF50B101212046FFF750FD7A
:10B2E00030B12046FFF7C4FF003818BF012010BD61
:10B2F0000846FCE710B50246FFF742FD20B102EB1D
:10B30000C11292ED140A10BDBFEE000AFBE7000067
:10B3100010B50246FFF734FD20B102EBC11292EDE9
:10B32000130A10BDBFEE000AFBE7000010B502468D
:10B33000FFF726FD20B102EBC11292ED150A10BDF8
:10B340009FED010AFBE700BF0000000010B50246B8
:10B35000FFF716FD20B102EBC11292ED170A10BDE6
:10B360009FED010AFBE700BF000000002DE9F04F50
:10B370002DED028B8DB0044672F0B8FE9FED3C8A35
:10B38000DFED3C8A80468946274625464FF0000B74
:10B3900004F5AA7A5FFA8BF631462046FFF7F0FCF7
:10B3A000002858D05AF82B30002B54D06A4620463B
:10B3B000FFF716FD08B9CDED008A1D22002104A873
:10B3C000A0F0ACFDA3238DF80430952331468DF811
:10B3D0000530204672238DF80630CDF80780CDF871
:10B3E0000B908DF80F60FFF793FF20468DED040A58
:10B3F000FFF79CFFDDED007A8DED050A67EE887A98
:10B400002046FDEEE77A17EE903AADF81830FFF7D8
:10B410009DFF10EE103A2046CDF81A30BB69CDF8EA
:10B420001E30FFF729FE31468DF822002046FFF737
:10B430001FFFD5F8BC300993D5F8C0300A9394F8B3
:10B440004E318DF823008DF82C3042F0B7FF2922C1
:10B4500001A941F0BBFF18378035BBF1000F04D0C4
:10B460000DB0BDEC028BBDE8F08F4FF0010B91E702
:10B470000000C84200000000F8B590F90030002B31
:10B4800004464DDD0021FFF721FE01212046FFF794
:10B490001DFE94F90030002B0DDD94F9403053B1BE
:10B4A0004CF03EFF012105462046FFF723FF1D49D2
:10B4B000284646F01BFB667894F84E7131462046CC
:10B4C000FFF7D6FE054668B901462046FFF7D0FED5
:10B4D00028B901212046FFF7CBFE28B1012584F8C9
:10B4E0004E5101E084F84E61204673F0C5FA94F89D
:10B4F0004E31BB4204D042F061FF5A2142F0F6FCCB
:10B50000D4F8503101330BD042F058FFD4F8501129
:10B5100042F07AFD20B12046BDE8F840FFF726BF93
:10B52000F8BD00BFA85B0C08014B1868704700BF4E
:10B530003C7E002010B50349044638F065FF2046E4
:10B5400010BD00BF5C5D0C08F0B52DED048B91B013
:10B5500004466D46284606F017FE94F8BC33002BCF
:10B5600072D004F57A730FCB85E80F0094F8F833A6
:10B57000D4EDEC8A94EDED8A94EDEE9A002B63D035
:10B5800094F8D033002B5FD02D22002104A8D4F8EA
:10B59000C073D4F8C463D4F8C853D4F8CC43A0F033
:10B5A000BDFCA3238DF8103095238DF81130462370
:10B5B0008DF8123072F09AFD9FED250A9FED257AE5
:10B5C000CDF8171068EE807ACDF8130067EE877A11
:10B5D000FDEEE77A17EE903A68EE007A29EE000A5F
:10B5E00067EE877AADF81B30FDEEE77A20EE070AAA
:10B5F00017EE903AADF81D3017F09CFDDDED017AA5
:10B600009FED157ACDF82D70BCEEC00AF8EEE77A02
:10B6100010EE103A67EE877AADF81F3017EE903AC9
:10B62000CDF82130029BCDF82530039BCDF8293091
:10B63000CDF83160CDF83550CDF8394042F0BEFE3E
:10B640002D2204A941F0C2FE11B0BDEC048BF0BD67
:10B65000E02E65420000C8420AD7233C30B52DEDEC
:10B66000028B8BB0044624220D4601A80021A0F0D5
:10B6700055FCA3238DF8043095238DF8053048231D
:10B680009FED1F8A8DF8063072F030FDD4ED817A7F
:10B690002B68CDF80F3067EE887A95ED020ACDF869
:10B6A0000B1017EE903AD4ED827ACDF8133067EE96
:10B6B000887A6B68CDF8173017EE903ACDF807000E
:10B6C000CDF81B3017F00CFD10EE103A94ED830A04
:10B6D000CDF81F3020EE080A17F002FD10EE103AE8
:10B6E000CDF8233094F80C338DF8273042F066FE05
:10B6F000242201A941F06AFE0BB0BDEC028B30BDE3
:10B70000E02E654230B587B014460D461822002160
:10B710006846A0F003FCA3238DF8003095238DF834
:10B72000013049238DF8023072F0E0FCA3680393E6
:10B73000E36804936368CDF807100593CDF8030020
:10B740008DF80B5042F03AFE1822694641F03EFE59
:10B7500007B030BD10B58EB0044602A806F014FD47
:10B7600002A9204601F006FC002845D001F054FE55
:10B77000694601F08FFA1F22002106A8A0F0CEFB37
:10B78000A3238DF8183095238DF819304A238DF8AE
:10B790001A3072F0ABFCDDED037A9FED1B7A049B4F
:10B7A000CDF82330F8EEE77A059BCDF8273067EE29
:10B7B000877ACDF81B0017EE903ADDED007ACDF8D0
:10B7C0002B30F1EE677A17EE903ACDF81F10204635
:10B7D00001A9CDF82F3000F051FD78B1DDED017AEF
:10B7E000F1EE677A17EE903ACDF8333042F0E6FD8D
:10B7F0001F2206A941F0EAFD0EB010BD42F0DEFDA9
:10B80000DFED027AEEE700BF0AD7233C5241C07F4A
:10B810007047000010B5044607F00CF8204610BD34
:10B820000023036043608360C360036143618361FD
:10B83000C3610362704700002DE9F041076A07F514
:10B840004876044600F16C050FCE0FC50FCE0FC52C
:10B8500033682B6007F5457393E8070004F19008FF
:10B8600088E8070094ED2E7AD4ED2D7A77EE877A6A
:10B870009FED367AF0EEE77AF4EEC77AF1EE10FA41
:10B880008EB004F16C0718D404F14802394604A8BC
:10B8900004AD17F0C3FF0FCD3E460FC60FCD0FC648
:10B8A0002B683360414604F1240017F039FF84ED22
:10B8B000240AC4ED250A84ED261A04F10C0304F1D0
:10B8C0000802211D384618F057F99FED216AD4ED82
:10B8D000037A94ED017ADFED1F6A206A67EE867ABB
:10B8E00027EE067A67EEA67A27EE267AFDEEE77A4D
:10B8F000BDEEC77A17EE903A84ED047A94ED027AA1
:10B90000002BB8BF03F50C4327EE067AB8BFA0336F
:10B9100027EE267AA36104F1B003039304F1AC038C
:10B92000BDEEC77A029304F1A803019304F1A403C6
:10B93000009384ED057A04F1A00304F19C023946DA
:10B9400001F028FE0EB0BDE8F08100BF0000003419
:10B95000E02E65420000C84210B504468AB0006A75
:10B9600001F0A8FD04A904F124008DED040ACDED39
:10B97000050A8DED061A17F0D3FE0AB010BD0000BF
:10B9800030B58BB0014604466D46684617F0B6FFE9
:10B990000FCD0FC40FCD0FC42B6823600BB030BD8B
:10B9A000F8B50446244B036000F1240501620277D8
:10B9B00004F148072846FFF733FF3846FFF730FF0A
:10B9C00004F16C00FFF72CFF217F00231829C4F835
:10B9D0009030C4F89430C4F8983026D0192926D075
:10B9E00039BBC4F8B430D4ED2D7A84ED2E0A30EE94
:10B9F000270A17F075FB9FED111ADFED110A284693
:10BA000060EE200AB0EE410A18F056F80FCD3E461F
:10BA10000FC60FCD0FC62B6833603846FFF7B0FF57
:10BA20002046FFF709FF2046F8BD064BD9E7064B35
:10BA3000D7E7064872F020FB405E0C0800000000CB
:10BA400035FA8E3C0000B442000087431C5E0C08AF
:10BA50000023036043608360C360036143618361CB
:10BA6000C36103627047000090F82031B02202FBEE
:10BA7000030390F8482193F8693012B1012B28BFD5
:10BA800001231846704700002DE9F04F04468BB0A3
:10BA90004FF0000A0D461EF0E9F884F814A204F5F0
:10BAA00006704FF07E5771F04BFA4FF47A73A4F89A
:10BAB000623284F86852C4F84872C4F84C72C4F810
:10BAC000507204F51B70002506F05EFB04F52B791F
:10BAD0000323C4F8803204F53476C4F89452C4F8D1
:10BAE0009852C4F89C52C4F8A052C4F8A452C4F8A6
:10BAF000A8524846FFF7ACFF04F5487B3046FFF7F5
:10BB0000A7FFC4F81453C4F81853C4F81C5358467C
:10BB1000FFF79EFFC4F84453C4F84853C4F84C538D
:10BB2000C4F85053C4F85453C4F85853C4F85C5381
:10BB3000C4F86053C4F86453C4F86853C4F86C5331
:10BB4000C4F87053C4F88C53C4F89053C4F8945399
:10BB5000C4F8A853C4F8A453C4F8A053C4F8B0530D
:10BB6000C4F8B453C4F8B853C4F8CC53C4F8C85399
:10BB7000C4F8C453C4F89C73C4F8C07304F575705A
:10BB800006F002FB04F57A7006F0FEFA04F5806315
:10BB9000C4F8FC531D6004F5816304F583601D60E7
:10BBA0005D609D6006F0F0FA04F22C4304F26448F4
:10BBB0001D605D609D60704BC4F83C3404F50D73EE
:10BBC000C4F8403404F50E73C4F8443404F50F731C
:10BBD000C4F8483404F51073C4F84C3404F2452317
:10BBE000C4F8503404F51173C4F8543404F58B636D
:10BBF00040461D605D609D60FFF72AFF04F591607F
:10BC0000FFF726FF04F5976304F23C421D605D6078
:10BC10009D6004F2C44304F2BC501D605D609D60F1
:10BC200004F59A631D605D609D6004F2DC431D6055
:10BC30005D609D6004F2EC431D605D609D6004F2F8
:10BC4000FC431D605D609D6004F5A1631D605D6047
:10BC50009D6004F22C53C2F8E070C2F8E4701D60DD
:10BC60005D609D6004F5A7631D605D609D6004F2EA
:10BC700044531D605D609D6004F5AC631F605D60B2
:10BC800004F284531D605D609D6004F5B2631D6025
:10BC90005D609D6004F5B5631D605D609D6006F0AC
:10BCA00073FA04F2CC5324221D605D6004F2D45375
:10BCB00051461D605D6004F2DC5340461D605D60CE
:10BCC000A0F02CF904F2FC50C8F82070C8F81070ED
:10BCD000C8F80070FFF7BCFE04F5C46304F5CA6041
:10BCE0001D605D609D6004F22C631D605D609D6061
:10BCF00004F5C7631D605D609D6004F244631D60D0
:10BD00005D609D6006F040FA1C4B1D491C6020469A
:10BD100038F07AFB94F8683243F0010384F8683213
:10BD2000514624225846A0F0F9F8C4F84073C4F8EC
:10BD30003073C4F8207304F5257207CA04F528731C
:10BD400083E80700484694EDAA1AD4EDA90A94EDB9
:10BD5000A80A17F0B1FE3546494668466E4617F008
:10BD6000CDFD0FCE0FC50FCE0FC533682B6020461B
:10BD70000BB0BDE8F08F00BF94600C08407E00203F
:10BD8000505F0C0810B5044688B001F0E3FB94F94D
:10BD90003232012B02D1274804F046FE022B0AD191
:10BDA000032384F8323204A9012304F111008DF831
:10BDB000103039F07DF994F8323284F8903204F280
:10BDC0003C4001F069FB94F93132642B30D165239A
:10BDD00004A904F231208DF8103039F0A7F904A934
:10BDE000204637F07BFC18B304238DF8183000236D
:10BDF000CDE9013303930F230593694604A837F077
:10BE0000EDFD059B28B108AA02EB8302009942F8D8
:10BE1000581C0133112B0593EFD966F0EDFE9DED13
:10BE2000031ADDED020A9DED010A652166F0A2FE0E
:10BE300008B010BD485E0C0870B500F5257600F519
:10BE400028758CB004463146284619F023FDE0B928
:10BE500096E8070085E8070004F52B7194EDAA1A0F
:10BE6000D4EDA90A94EDA80A0191084617F024FE22
:10BE700002AD019902A817F041FD0FCD04F534740D
:10BE80000FC40FCD0FC42B6823600CB070BD000031
:10BE900013B540F2411200F50671044601A813F0F3
:10BEA000C7F904F23C4001F0F1FC20461EF036F9DF
:10BEB00001A813F0DFF902B010BD0000F8B50B685F
:10BEC000C0F804324B68C0F808328B68C0F80C32F6
:10BED00001F10C0607460C4600F548750FCE0FC55C
:10BEE0000FCE0FC533682B6004F1300207CA07F587
:10BEF000457383E8070004F13C0207CA07F5517354
:10BF000083E8070004F1480207CA07F5547383E881
:10BF10000700543494E8070007F5577383E80700D7
:10BF2000384601F029FC3846BDE8F84001F00CBC69
:10BF300013B5044600F23C40019003F0C3F804F549
:10BF4000BE610198009102F0D1FB0099204602B039
:10BF5000BDE81040FFF7B2BF4A78064BC2F340126B
:10BF60001A754A78C2F380125A750A78C2F3001221
:10BF70009A757047CD7E002013B540F2F522044635
:10BF800000F5067101A813F053F9002104F23C40BA
:10BF900001F0CAFE94F8603223B120461EF006FB81
:10BFA00084F8600201A813F065F902B010BD00002A
:10BFB00038B590F80C3305460C462BB1032B0BD04B
:10BFC00095F86832DB070CD405F5CA630FCB84E81B
:10BFD0000F0095F8600603E01EF016F90028EFD078
:10BFE00038BD0020FCE7000000F23C4090ED380A2C
:10BFF0007047000000F23C4090ED390A70470000A5
:10C0000010B490F80C230C462AB1032A0AD0002061
:10C010005DF8044B704700F5B56007C884E8070079
:10C020000120F5E75DF8044B1EF0ACB890F88403EE
:10C03000431E58425841704738B590F80C330D46AE
:10C040008BB900F23C4001F093FC044610B9002487
:10C05000204638BD01F0E0FBD5ED007A27EE800ADE
:10C0600085ED000AF4E7D0EDE07AC1ED007A90F8B2
:10C070007C43002CEBD090EDDE7ADFED086AB4EE65
:10C08000E67AF1EE10FAF7EE006AB8BFB0EE667A23
:10C0900067EE877AC1ED007ADAE700BF000000346E
:10C0A00090F80C33032B01D11DF0E6BF0020704740
:10C0B00010B490F80C43032C03D15DF8044B1DF031
:10C0C000E7BF00205DF8044B7047000090F80C2398
:10C0D000032A01D11EF04EB900F23C4002F086B8AE
:10C0E00030B590F80C3385B004460D468BB1032B68
:10C0F00018D004F5257019F007FC284601A98DED2C
:10C10000010ACDED020A8DED031A18F0BBFF0120E4
:10C1100006E000F23C4001F0D5FB0028E9D1002008
:10C1200005B030BD90F86032002BF8D01EF00AF94F
:10C13000DFE700007FB590F80C2332B1032A4FF0FF
:10C14000000309D0039304930CE000F23C4007B0D5
:10C150005DF804EB01F06CBC03A903930493059311
:10C160001DF080FF9DED030ADDED040A07B05DF8C8
:10C1700004FB000007B590F80C3333B100F57F7075
:10C1800003B05DF804EB19F047B900F23C4001F050
:10C190004FFC68468DED000ACDED010A19F03CF91F
:10C1A00003B05DF804FB000090F80C03003818BFE2
:10C1B0000120704708B590F80C23032A05D0BDE88C
:10C1C000084000F23C4001F01DBC1DF04BFF012077
:10C1D00008BD000010B590F80C230C461AB1032AD4
:10C1E00007D0002010BDBDE8104000F23C4001F037
:10C1F000D1BB1DF05DFF012084ED000AF2E70000D5
:10C2000090F80C33032B01D11EF05CB8002070476E
:10C2100030B590F80C3385B005460C4623B1032B9E
:10C2200009D0002005B030BD00F23C4005B0BDE8AB
:10C23000304002F08BBA002302A9029303931DF051
:10C24000F9FE0028EDD001A928461DF0FFFE0028C8
:10C25000E7D0029B2360039B6360019BA360E1E73F
:10C2600090F80C231AB1032A05D00020704700F281
:10C270003C4002F09FBA1DF0DDBE000090F80C2398
:10C280001AB1032A05D00020704700F23C4002F0AA
:10C2900083BA1DF0DBBE000090F932323BB990F852
:10C2A000683213F0010F14BF0320002070470320F1
:10C2B00070470000F7B50446FFF7EEFF054600287B
:10C2C00062D0032839D194F860326BB394F86832A5
:10C2D000D8072BD501A920461EF09AFABDF80430E4
:10C2E000002B18BF002594F8146206F0FD06012EFD
:10C2F0004AD10023032D019307D101A920461EF046
:10C3000093FA20461EF04EF8064604F23C4002F036
:10C31000CFFA08B994F809039DF80430D90703D57A
:10C320005A0701D59F0632D400252DE020461DF086
:10C33000F1FD002808BF0025D5E70025D3E713F05D
:10C34000020F2EE094F9443223B99DF80430DB0942
:10C350002FD0E9E7002EF8D00EF04CFEFFF784FB5B
:10C36000022807D99DF805309806DDD59DF80430E0
:10C37000D906D9D5FB6A93F89C30002BE5D118E09B
:10C38000DA0601D41B0718D5284603B0F0BD0028F3
:10C39000FAD094F80923B4F96436002ACFD013F008
:10C3A000010FF1D1154B1F68FB6A93F89C30002BED
:10C3B000C8D19DF804309C07E2D406F001FD06F0D8
:10C3C00025FC0028B0D10EF015FEFFF74DFB02282A
:10C3D000AAD90EF00FFE90F82031B02202FB030024
:10C3E00090ED217AF0EE007AB4EEE77AF1EE10FAF1
:10C3F0009AD59DF80530DB09C6D195E7482700207E
:10C400002DE9F04790F8603292B00446002B00F01E
:10C41000948020461EF0C8FB2046FFF74BFF032800
:10C420007BD104F5487800274146204600970197C4
:10C4300002971DF05DFF694620461DF04FFF009BEF
:10C44000C4F80432019BC4F80832029BC4F80C32D1
:10C45000204601F091F9204601F076F916F08CF9AA
:10C46000054620461DF0D8FD0028A8BFC6B203AA85
:10C470004FF0FF312046BCBF95F8EB9495F8EC6483
:10C480000397A8BFB146049705971DF01FFE03A8A8
:10C4900019F03AFA4FF00C0A0AFB095084EDD10A60
:10C4A000C4EDD20A84EDD31A04F5517100F55C7025
:10C4B00019F03AFA04F557770AFB065584EDC50AD8
:10C4C000C4EDC60A84EDC71A3A464FF0FF31204644
:10C4D00005F500751DF00EFE95E8070006AE86E82E
:10C4E00007003946304619F085FA04F52B724146AB
:10C4F00009A817F093F9314609A817F011F909A90D
:10C50000204684EDD40AC4EDD50A84EDD61A1EF077
:10C510008BF909A92046FFF71FFD94F86636002B1A
:10C520003AD109A805F030FE09A920461DF078FE91
:10C5300090B3012384F866362EE0D0F864321BB93C
:10C5400071F0CCFDC4F86402154B1B68D86A03680F
:10C550005B68984788B171F0C1FDD4F86432C01AA5
:10C56000B4F86232984204D920461EF01FF884F8CD
:10C57000600294F860327BB14BE771F0AFFDD4F804
:10C580006432C01A41F287339842E4D841F016FF72
:10C5900041F056FD0028DED112B0BDE8F08700BFA3
:10C5A0004827002090F80C3323B1032B4FF00000F4
:10C5B00007D0704790F93222032A04D10A70012073
:10C5C00070470870FBE718467047000073B50D46CA
:10C5D0000DF107010446FFF7E5FF064628B19DF877
:10C5E00007302BB1032B09D00026304602B070BDB6
:10C5F00004F5CA630FCB85E80F00F6E7294620460D
:10C600001DF002FE94F86062EFE700007FB50E4671
:10C610000DF103010446FFF7C5FF054618B90025D3
:10C62000284604B070BD9DF8033083B1032B16D0AB
:10C6300004F5257019F068F901A930468DED010A5D
:10C64000CDED020A8DED031A18F01CFDE8E7314626
:10C6500004F23C4001F036F90028E9D1DFE794F814
:10C660006032002BDBD0314620461DF06BFEDFE749
:10C6700037B50D460DF107010446FFF793FF28B1CA
:10C680009DF8073023B1032B0FD0002003B030BD3D
:10C6900004F5BE631B682B6004F2F45304F5BF6419
:10C6A0001B686B602368AB60F0E7204629461DF0ED
:10C6B00015FE94F86002E9E710B50446FFF7ECFDBB
:10C6C00018B1032807D0002010BD04F23C40BDE89B
:10C6D000104001F021B994F86032002BF3D02046CD
:10C6E0001DF018FC0028EED094F8143203F0FD037E
:10C6F000012BE9D194F80C03C31E58425841E3E7DB
:10C7000010B50446FFF7C8FD80B1032810D194F896
:10C71000600250B171F0E2FCD4F86432C01A44F601
:10C720002063984294BF0020012010BD0120FCE747
:10C730000020FAE708B50246FFF7AEFD032804D152
:10C7400010461EF071F8012008BD0020FCE7000033
:10C7500030B585B004460191FEF7E6FE0199054625
:10C7600010B9002005B030BD0191FEF785FC01999C
:10C770000028F6D02846FEF77BFD0028F1D0B4F85B
:10C7800064365907EED494F80933002BEAD00B4AEB
:10C790001268D26A92F89C506DB103A92046FFF747
:10C7A000C9FF30B19DF80E309A07DBD5C3F3800086
:10C7B000D8E72846D6E71846D4E700BF4827002028
:10C7C0001DF0FEBD1DF032BE10B490F80C4324B134
:10C7D000032C08D05DF8044B70475DF8044B00F261
:10C7E0003C4001F065B85DF8044B1DF0B1BC0000A1
:10C7F00090F80C33F5EE007A002BB7EE000A08BF74
:10C80000B0EE670A7047000010B50446FFF744FD1C
:10C81000032804D12046BDE810401DF0CBBC002009
:10C8200010BD00002DE9F04190F80C338CB00027CA
:10C83000032B06460C46154600970197029719D11F
:10C840001DF0EAFB6A4680464FF0FF3130461DF08E
:10C8500051FCB8F1FF3FA760676027600DD115F06C
:10C860008BFF2B4690F8EC14224614F0B5FE0CB06A
:10C87000BDE8F0814FF0FF38EBE715F07DFF2B4668
:10C8800022465FFA88F114F0A7FE95ED000A68468B
:10C8900019F076F803A920468DED051A8DED030AEF
:10C8A000CDED040A19F0A6F806F52B7206F54871CD
:10C8B00003A816F0B3FF214603A816F031FF84ED5C
:10C8C000021A84ED000AC4ED010A95ED007ADFED4D
:10C8D000037AA7EE271A84ED021AC8E70AE81C417A
:10C8E0001FB5DFED0B7A20EE270A0C461946094BDF
:10C8F000CDE90042BDEEC00A18688DED020A064B74
:10C900009DF81820C06A12F071FE04B010BD00BF7F
:10C91000E02E6542482700205C5E0C082DE9F047B8
:10C920002DED028B92B0002504460F464FF07E5A43
:10C9300000F5487106A89046CDF818A0099508950D
:10C94000079517F0A5FF06F03BFA06F05FF9814660
:10C950002046FFF7A1FC032803D094F80C33032BE7
:10C960004FD19FED558ADFED558A00262379F2B22B
:10C97000934247D90AAA71B22046CDF828A00D9556
:10C980000C950B951DF0BEFC0AA906A818F0ECFB4F
:10C99000B4EEC80AF1EE10FA0DDD494ACDF8008078
:10C9A0003B4648492046FFF79BFF002012B0BDECF4
:10C9B000028BBDE8F0870AA906A8039504950595A2
:10C9C00018F0BCFB03A90EA88DED0E0ACDED0F0AE1
:10C9D0008DED101ACDED111A18F0E0F8B9F1000F35
:10C9E0000DD09DED050AB0EEC00AB4EEE80AF1EEF6
:10C9F00010FA04DD344ACDF800803B46D1E7013619
:10CA0000B4E7002394F8686216F0010001D0012B0E
:10CA1000CCD104F2FC510AA8CDF828A00D950C95B4
:10CA20000B9517F035FF0AA906A818F09DFBDFED5E
:10CA3000227AB4EEE70AF1EE10FA05DD204ACDF8CD
:10CA400000803B462149ADE72046FFF725FC03283F
:10CA50002DD120461DF09AFC94F86832DB0728D4CB
:10CA600038BB0AA906A803950495059518F066FB3E
:10CA700003A90EA88DED0E0ACDED0F0A8DED101A4B
:10CA8000CDED111A18F08AF8B9F1000F11D09DED13
:10CA9000050ADFED0A7AB0EEC00AB4EEE70AF1EE5D
:10CAA00010FA06DD084ACDF800803B46CAE70020B0
:10CAB000D2E701207AE700BFC2B8323EC2B8B23E28
:10CAC000885E0C08935E0C08BF960D08985E0C08F3
:10CAD0002DE9F7431446054688460193FFF7ECFD20
:10CAE000019A074638B92448244B00682146C06A99
:10CAF00012F07CFD019A019221462846FFF70EFFB5
:10CB0000064630B32846FFF7C7FB95F80C33019A69
:10CB100083420DD006F054F906F078F8019A38B146
:10CB2000174B154800682146C06A12F05FFD10E0FF
:10CB30002846FFF7B1FB18B103280FD0114BF0E7DF
:10CB400013464146224605F23C4000F0F9FE00B192
:10CB500007B90026304603B0BDE8F08395F860922F
:10CB6000B9F1000F01D1084BDBE7134641462246DD
:10CB700028461DF0DFF9EAE7482700209C5E0C08F4
:10CB8000A85E0C08D85E0C08C75E0C0890F80C3341
:10CB9000032B01D11DF05EBE0020704790F80C33CE
:10CBA000032B01D11DF096BE0020704790F80C3386
:10CBB000032B01D11DF0D2BE0020704708B50246FC
:10CBC000FFF76AFB10B1032806D008BDBDE8084096
:10CBD00002F23C4000F06ABEBDE8084010461DF07D
:10CBE0002FBE00000B4610B411462BB1032B09D009
:10CBF00000205DF8044B70475DF8044B00F23C40A8
:10CC000000F06ABE5DF8044B1DF00ABB13B5044684
:10CC1000FFF742FB0A46014620460192FFF7E2FF7A
:10CC200070B9084B019A1B68DB6A93F89C0038B115
:10CC300094F80C13204602B0BDE81040FFF7D2BFB5
:10CC400002B010BD4827002037B504460D4640F21B
:10CC5000B25200F5067101A812F0EAFA2946204600
:10CC60001DF0FCFA94F80C33032B054610D148B1A3
:10CC700004F583612046FFF7C9FF84F828042046A5
:10CC800000F0AAFD01A812F0F5FA284603B030BD65
:10CC90000025F7E770B590F87C32DB0786B00446D4
:10CCA0000D460CD402F040FF437C242202FB03001B
:10CCB000D0ED0B7AF1EE677AC5ED007A3AE002A882
:10CCC00005F062FA01A92046FFF7D8FAE0B90EF0A4
:10CCD00091F994F94432022B0646E3D1FEF7C4FEE3
:10CCE0000228DFD996F820019FED137AB02303FBC9
:10CCF0000066D4F87032B26F9B1A07EE903AF8EEE5
:10CD0000E77A67EE877AD7E702A92046FFF77EFF2A
:10CD10000028DCD0D4F87022039BDFED076A9DED7C
:10CD2000017A9B1A07EE903AF8EEE77AA7EEE67AD8
:10CD300085ED007A06B070BD0AD7233CF0B50C46ED
:10CD400087B000F50671064640F6863201A812F05B
:10CD50006FFAA36853B9E36843B9636833B900272E
:10CD600001A812F087FA384607B0F0BD204605F05A
:10CD700013FB0028F3D094E80F0002AD85E80F0004
:10CD80000021284605F0CAFA07460028E7D096F8A1
:10CD90007C32DB0704D441F011FB192141F0A6F8E5
:10CDA00095E80F0006F51B7C8CE80F0096F87C32A6
:10CDB00043F0010386F87C32304600F00DFD4BF065
:10CDC000AFFA46214CF0CAF84BF0AAFA45214CF0D4
:10CDD000C5F8054BA2681B68DB6A1A61E2685A61F4
:10CDE00062689A61BCE700BF4827002038B5144B41
:10CDF0001B68DD6A2B6804465B6828469847F0B1DB
:10CE00002B690BB96A69D2B1C4F874326B69C4F882
:10CE10007832A969002204F51B7005F0BBF994F87B
:10CE20007C3223F0030343F0030384F87C324BF09D
:10CE300077FABDE83840034A062144F0CBBB38BD41
:10CE400048270020EC5E0C0810B588B00446059316
:10CE5000FFF722FA0328059B4FF000000AD1069045
:10CE6000079006A802900B9801900A98009020461F
:10CE70001DF072FA08B010BD38B50446FEF754FB39
:10CE80000546D0B194F80C33032B03D095F84E41EE
:10CE9000204638BD20461DF081F9FF280446F5D014
:10CEA00001462846FEF7E4F90028EFD0214628463F
:10CEB000FEF7E2F80028E9D0EAE70446E8E70000D8
:10CEC00008B590F80C33032B05D015F055FC90F9FC
:10CED000EB04C0B208BD1DF09FF8431CF9D1F4E784
:10CEE00008B590F80C3383B1032B03D1BDE808409B
:10CEF0001DF08AB83FF080FC40F6ED424FF48011FF
:10CF00003FF032FC4FF0FF3008BD1846FCE7000050
:10CF100090F80C33032B01D11DF092BF7047000035
:10CF200090F80C33032B01D11CF052BF7047000066
:10CF30001CF0D8BF10B5044620F010F82046FEF7CC
:10CF400003FB2046BDE81040FEF704BC07B52030C7
:10CF500001A98DED010A38F07FF803B05DF804FBFC
:10CF600090F80C330BB1032B01D11DF0E5BF00206D
:10CF70007047000030B500F5757304460D460FCBC1
:10CF800085E80F0094F8E40330BD00007FB5054646
:10CF900068460E4605F0F8F895F87C32DB0703D4B6
:10CFA0000024204604B070BD69462846FFF7E2FF22
:10CFB00004460028F4D0694605F51B7005F0FCFA1C
:10CFC00086ED000AC6ED010AEBE70000D0F88033D9
:10CFD0000B6090F87C037047D0F888330B6090F8B2
:10CFE0008503704730B500F5677304460D460FCBD7
:10CFF00085E80F0094F8AC0330BD000030B500F5B3
:10D00000836304460D460FCB85E80F0094F828048F
:10D0100030BD000010B500F22C4203460C4607CA92
:10D0200084E8070093F8380410BD00002DE9F043B0
:10D030002DED028B8BB005460E461746FFF71CFF01
:10D04000014680462846FFF783FB0446002848D067
:10D05000FEF76AFA4146FEF74DF986ED000A95F9AA
:10D060003032002B3ADD0DF0C5FFFEF7FDFC012844
:10D0700034D90DF0BFFF90F82031D5EDDE7ADFED29
:10D080005D8A96ED000AB02202FB030095F930326A
:10D09000D0ED210A07EE103AF4EEE87AB8EEC77A3E
:10D0A000F1EE10FAB7EE008AB8BFF0EE487A37EE2C
:10D0B000201A20EE270A70EEC70A40F2B63016F0AA
:10D0C000A3F8D5EDDE7AF4EEE87AF1EE10FAB8BF07
:10D0D000F0EE487A80EE277A86ED007A01233B70E5
:10D0E00003E095F8083333B9387020460BB0BDEC37
:10D0F000028BBDE8F08395F80C334FF00009CDF8B2
:10D100000490CDF80890CDF80C9043B1032B10D0CB
:10D11000CDF81090CDF81490CDF818907CB902237A
:10D120003B703246414605F23C4001F085FB044627
:10D13000DBE701A928461DF025F80446E8E795F845
:10D140000C33002BEBD004A92846FFF763FF0446FD
:10D150000028E4D001A904A818F0FCFB07A8CDED35
:10D16000080A8DED091A8DED070A19F007F804A8D1
:10D17000B0EE408A19F002F895F93032002B30DD1C
:10D1800007EE903AF8EEE77A4FF47F7070EE670A98
:10D1900037EE801AF5EEC00AF1EE10FA48BFDFED67
:10D1A000160AF4EE410AF1EE10FAB0EE480AC8BFD2
:10D1B000B0EE601A16F028F8B0EE408AD5EDDE7AAF
:10D1C0009FED0C7AF4EEC77AF1EE10FAB7EE007A22
:10D1D000B8BFF0EE477A88EE277A032386ED007A0F
:10D1E0007DE7B5EEC08AF1EE10FA48BF9FED028AE6
:10D1F000E4E700BF000000340000000010B5044662
:10D20000FFF75EFE84F80D032046FFF759FE84F811
:10D210000E032046FFF754FE84F80F032046FFF765
:10D220005FFE04F55A7184F810032046FEF7E8FE0D
:10D2300084F8740300F0F0FA04F5617284EDDE0AFC
:10D2400004F560712046FFF7F1FE04F5627184F881
:10D250007C032046FEF7F0FE04F5637184F8850335
:10D260002046FEF71DFF04F5677184F898032046F9
:10D27000FEF736FF04F56C7184F8AC032046FFF727
:10D28000F7F904F5707184F8BC032046FFF7BEF986
:10D2900004F5757184F8D0032046FEF789FE04F585
:10D2A0007A7184F8E4032046FFF790F984F8F803D4
:10D2B0002046FEF73FFF04F5806384EDFF0A204619
:10D2C000C3ED000AFEF756FF04F2044383ED000AA3
:10D2D00004F2144204F581612046FFF7A3FA04F535
:10D2E00083612046FFF792FC04F22C4184F8280465
:10D2F0002046FEF75FFF84F8380410BD37B50D46B1
:10D30000044600F027F91DB915F036FA14F038F884
:10D310004FF4BE7204F5067101A811F089FF94F86C
:10D3200069322BB92046FFF761FD012384F8693289
:10D33000224B1D68A86A03689B6998472046FEF740
:10D340007BFD2046FEF7F4FD204600F077FA2046EC
:10D35000FFF756F8286B30B10368D4EDD20ADB68CA
:10D3600094EDD10A9847D4F8100208B1FEF764FA98
:10D37000204600F091F82046FEF79CFF94F890328A
:10D3800084F80C0383420ED084F8900298B10C4DBF
:10D390000C4B032808BF1D464AF0C2FF0A4A2B4621
:10D3A000062144F017F92046FFF728FF01A811F0E5
:10D3B00061FF03B030BD054DEEE700BF48270020F8
:10D3C000E71C0C08935E0C08045F0C08985E0C08C0
:10D3D000D0EDDE7A9FED057AF4EEC77AF1EE10FA21
:10D3E000B7EE000AA8BFB0EE670A7047000000342D
:10D3F000D0EDDE7A9FED077AF4EEC77AB7EE000A39
:10D40000F1EE10FAB8BFF0EE407A67EEA77A80EE40
:10D41000270A704700000034014B1868704700BFAE
:10D42000407E00204FF0FF30704700000120704721
:10D4300070470000002070470020704770470000D0
:10D4400070470000002070470020704700207047A0
:10D450000020704700207047002070470020704770
:10D46000012070470368D3F89430184700207047B4
:10D470000020704700207047002070470020704750
:10D480000020704700207047002070470020704740
:10D4900000207047704700007047000008B515F085
:10D4A0006BF990F8EC0408BD08B515F065F990F833
:10D4B000EB0408BD30B585B090F80E53044615F066
:10D4C0005BF90C2303FB050004F5517100F55C705A
:10D4D00005B0BDE8304018F027BA000030B52DED9A
:10D4E000028B9FED1A1ADFED1A0A91ED000A87B040
:10D4F00005462D200C468DED011ACDED000A15F0E4
:10D5000083FE9DED011ADDED000AF0EE408A2E202B
:10D5100094ED010A15F078FE9DED011ADDED000A8B
:10D52000B0EE408A2F2094ED020A15F06DFE03A99B
:10D5300005F52570CDED038A8DED048A8DED050A84
:10D5400037F0D8FE07B0BDEC028B30BDC2B8323E1A
:10D55000C2B832BE10B5044670F0C0FDD4F8F43243
:10D560001BB1C21AB2F57A7F11D3094A1268D26A86
:10D5700092F89C2002B153B9C4F8F40294F83142F5
:10D5800015F0FAF880F8E24405F01AFC447610BD74
:10D59000482700202DE9F0432DED028B91ED007A14
:10D5A000D1ED037A87B08DED047AB0EEC77AB5EE8F
:10D5B000C07AF1EE10FADDE91087DDF84C90CDED80
:10D5C000057A0C4615461E4606DCF0EEE77AF5EEC7
:10D5D000C07AF1EE10FA02DD04A817F09BFF6B2071
:10D5E000B7EE001AFFEE000A9DED050A15F00CFEDD
:10D5F0006C2089ED000AB7EE001AFFEE000A9DEDDF
:10D60000040A15F001FE04A888ED000A17F0DEFEFA
:10D61000B7EE008A002852D00023C9F8003088ED08
:10D62000008AD4ED067A67EEA77AF4EEC87AF1EEB6
:10D6300010FA4ADB0023336085ED008ADFED3F0AF4
:10D6400096ED000A7C20B7EE001A15F0DDFD86EDA0
:10D65000000A95ED000A7D20B7EE001AFFEE000AE1
:10D6600015F0D2FD85ED000AD4ED067A129BDFEDB0
:10D67000346AF1EE677AC3ED007A96ED007AF0EE47
:10D68000C77AF4EEE67AF1EE10FA2BD503AB02AAD4
:10D6900001A9204616F070FA9DED018AB0EE480A05
:10D6A0009CF020F885ED000AB0EE480A9CF070F975
:10D6B00087ED000A07B0BDEC028BBDE8F08304A83B
:10D6C00017F070FE0028A7D1ABE738EE670A15F017
:10D6D000CDFC86ED000A94ED087AC7EE007AC5ED20
:10D6E000007AABE794ED076AC6EE077AC7ED007AD9
:10D6F00096ED007AB0EEC77AB4EEE67AF1EE10FA63
:10D70000C4D495ED007ADFED0F6AB0EEC76AB4EECF
:10D71000666AF1EE10FAB9DCB4EE477AF1EE10FA6F
:10D72000B4D6B0EEE77AB4EE667AF1EE10FAADDC7C
:10D73000F4EE677AF1EE10FABCD7A7E7000000001C
:10D7400000000034FFFF7F7F1FB500F517730393C0
:10D7500000F51673029300F51573019300F5147329
:10D76000009300F5127200F5137300F54871FFF78E
:10D7700011FF05B05DF804FB9FED156A90ED817A0D
:10D78000DFED146AD0ED837A27EE067A67EE867AAB
:10D7900027EE267A67EEA67ABDEEC77AFDEEE77A27
:10D7A00080ED7E7A90ED827A27EE067A17EE903A37
:10D7B00027EE267A002BB8BF03F50C43BDEEC77ADF
:10D7C000B8BFA03380ED7F7AC0F80032704700BF49
:10D7D000E02E65420000C8421FB50E4B1B68044690
:10D7E000B3B1684604F0D0FC69462046FFF706FC5A
:10D7F00020B16A4600212046FDF784FF94F87C3270
:10D80000DB0705D504F51B7201212046FDF77AFFE1
:10D8100004B010BD2481002008B502F085F9BDE8F0
:10D82000084001F097BD000010B580F8F8120446DA
:10D8300070F054FCC4F8FC0210BD000010B590F864
:10D84000F832044653B170F049FCD4F8FC32C01AE7
:10D85000B0F57A7F84BF002384F8F83294F800335F
:10D8600053B170F03BFCD4F80433C01AB0F57A7FA2
:10D8700084BF002384F8003310BD000000F5B670AB
:10D880000B4607C883E80700012070470023C0F853
:10D890009C30C0F89830C0F89430C0F8A830C0F878
:10D8A000A430C0F8A030C0F8AC307047704700001A
:10D8B000024B0B604FF07C531360704700004842EE
:10D8C0007047000008B50B4600F12801184616F015
:10D8D000DFFF012008BD000010B500F5C0700C4648
:10D8E0000FC884E80F00204604F03EFC30B1FFF77B
:10D8F00093FD00F51B700FC884E80F00204604F06C
:10D9000033FC80F00100C0B210BD000010B5044629
:10D9100004F090FF204610BD10B5D0F878310446D1
:10D920005BB170F0DBFBD4F87831C01A41F2883378
:10D93000984294BF0020012010BD0120FCE70000A8
:10D9400013B5009303680192D3F890309847DDE94E
:10D950000021044628B90448044B0068C06A11F04D
:10D9600045FE204602B010BD482700209C5E0C08F2
:10D9700013B504460191FDF7D7FD2368019A1B6D8D
:10D98000014608B190F84E11204602B0BDE81040A3
:10D990001847000030B585B000230193029303932C
:10D9A00003680D46DB6D01A99847044620B1039B2F
:10D9B0002B60204605B030BD02F0B6F8417C01F086
:10D9C00005FE04460028F4D002F0AEF801F064FD34
:10D9D000B1EE400A85ED000AEBE7000010B5FDF757
:10D9E000A3FD044658B190F84E11FDF745FB30B148
:10D9F00094F84E112046BDE81040FDF739BC0020D8
:10DA000010BD000038B50D460DF0F4FA0446FEF7DF
:10DA10002BF8022881BF94F82001B02303FB0040BB
:10DA20009C3089BF07C8002085E80700012038BD69
:10DA30002DE9F0432DED028B8FB003680025DB6CE0
:10DA40000395049505950695029502A90446984705
:10DA5000064638B1FFF7E0FEDDED027A27EE800AD8
:10DA60008DED020A0DF0C6FAFDF7FEFF0746002E07
:10DA700050D0DDED027AD4ED6A6A94ED6B7A2368BA
:10DA80000B9527EE877A67EEA67A8DED097ACDEDB4
:10DA90000A7A0C950D959B6C0BA9204609AD984709
:10DAA0000BA9284617F0DAFB012F8DED030ACDED07
:10DAB000040A40F2B3800DF09DFA90F82031DFEDBA
:10DAC0005B7AB02505FB030090ED228A28EE278AB9
:10DAD000B0EE480A9BF006FEF0EE408AB0EE480A2F
:10DAE0009BF056FFCDED0B8A8DED0C0A0DF082FAFE
:10DAF00090F8203105FB030090ED210A0BA817F0E8
:10DB0000CDFB09AD8DED050ACDED060A05A896BB46
:10DB100003C885E00128CED89DED020AB5EEC00A03
:10DB2000F1EE10FA7FDD07AED4F8AC21D4F8A831BD
:10DB300007923046089317F0EDFB23680B950C9580
:10DB40000D959B6C0BA920469847DDED077A9DED5E
:10DB50000B7A77EE877A9DED0C7ACDED077ADDEDC5
:10DB6000087A77EE877A09ABCDED087A96E803005C
:10DB700083E8030049E0236993ED000AB7EE008AC9
:10DB800038EE408A17F08AFB04F5C8798DED090A52
:10DB90004846B0EE480ACDED0A0A17F07FFB0BA904
:10DBA0002846CDED0C0A8DED0B0A17F057FB04F556
:10DBB000D07603AFC4ED650A314684ED640A384679
:10DBC00017F05CFB04F5CC788DED090A4046B0EE09
:10DBD000480ACDED0A0A17F061FB0BA928468DED26
:10DBE0000B0ACDED0C0A17F039FB97E8030084ED22
:10DBF000660AC4ED670A86E803004946404617F006
:10DC00002DFB8DED090ACDED0A0A9DED090ADDED2A
:10DC10000A0A0FB0BDEC028BBDE8F083DDE9030119
:10DC200085E80300F1E709950A95EEE735FA8E3CA1
:10DC300010B590F8F611044604F04CFE7C23C0B2F7
:10DC400003FB0044D4F8940010BD0000044B026FA5
:10DC50001B68DB6A5A60426F9A60826FDA607047B5
:10DC600048270020F0B58FB0044614F085FD00234E
:10DC700002930393049390F8EB1401AB02AA0546B8
:10DC800013F04CFC04F19407D8B39DED010AB5EEF6
:10DC9000C00AF1EE10FA34DD02A817F081FE04F19B
:10DCA000B00684ED2C0AC4ED2D0A84ED2E1A3946F7
:10DCB000304617F085FE04F17C01304617F034FE43
:10DCC00004F1880105A88DED050ACDED060A8DED5C
:10DCD000071A17F029FE08A88DED080A9DED010A24
:10DCE000CDED090A8DED0A1A17F04AFE0BA904F1D1
:10DCF00028008DED0B0ACDED0C0A8DED0D1A15F0F7
:10DD0000E7FF95F8EB040C2303FB0050394600F5C0
:10DD10005C7017F009FE84ED2C0AC4ED2D0A84ED29
:10DD20002E1A0FB0F0BD00002DE9F047824B002500
:10DD30001F682DED028BC0F89C50C0F89850C0F8B9
:10DD40009450C0F88450C0F88050C567C0F8905017
:10DD5000C0F88C50C0F88850C0F8B850C0F8B45023
:10DD6000C0F8B0500446F86A03688AB05B680E4693
:10DD7000984704F12809002854D070F0AFF942F216
:10DD80000F7398424ED8FB6A9FED6C8A93ED010A9F
:10DD900084ED1C0AD3ED020AC4ED1D0A93ED031AAB
:10DDA000484684ED1E1A15F087FE4AF0B9FAD4ED04
:10DDB0001E7A67EE887A054617EE900AF2F7A4FB02
:10DDC000D4ED1D7A67EE887ACDE9040117EE900A4A
:10DDD000F2F79AFBD4ED1C7A67EE887ACDE902015E
:10DDE00017EE900AF2F790FB554ACDE900010621A3
:10DDF000284643F0EFFB94ED1E8AB0EE480A9BF0F4
:10DE000071FC84ED6B0AB0EE480A9BF0C1FD84ED15
:10DE10006A0A70F063F9C4F87C010AB0BDEC028BA9
:10DE2000BDE8F087A6B194ED1C0AB4EE400AF1EE0D
:10DE300010FA0DD6D4ED1D0AF4EE600AF1EE10FAD8
:10DE400006D694ED1E1AB4EE411AF1EE10FA52D72E
:10DE500014F092FC90F8EC344FF00C0A0AFB030328
:10DE600003F50073074693E8070007AE86E807004E
:10DE70004FF01508B2EE028AF2EE068A304618F02C
:10DE80007DF9B4EEC80AF1EE10FA38D508F1FF3882
:10DE900018F0FF083CD1304618F070F9F1EE047A22
:10DEA000B4EEE70AF1EE10FA43DD9DED090ADDED6F
:10DEB000087A9DED078A20EE000AA7EEA70A9BF0DC
:10DEC0007DFFF0EE400AB0EE480A9BF02DFEDDED3E
:10DED000090A84ED1D0A9DED080AF1EE600AB1EE13
:10DEE000400A9BF021FE84ED1C0A9FED161AD4ED2A
:10DEF0001D0A94ED1C0A484615F0DEFD7BE730460E
:10DF000018F03CF9B4EEE80AF1EE10FABEDCC2E714
:10DF1000384613F053F9384613F032FA97F8EC34D8
:10DF20000AFB037303F5007393E8070086E8070014
:10DF3000A4E725676567D8E748270020E02E6542FB
:10DF400010600C08000000000021FFF7EDBE00008B
:10DF500037B5044608461546019118F00FF9B7EE9B
:10DF6000007AC7EE007AB4F8DC3001980133A4F8E7
:10DF7000DC3094ED367A37EE277A84ED367AB0EEDF
:10DF8000007AF4EEC77AF1EE10FA06D5B6EE007A12
:10DF9000F4EEC77AF1EE10FA0DDC9FED0E7AF4EE96
:10DFA000C77AF1EE10FA13D59FED0B7AF4EEC77A2B
:10DFB000F1EE10FA0CDDB0EE670A17F0E1FC01207B
:10DFC00085ED000AC5ED010A85ED021A03B030BDEA
:10DFD0000020FBE700247449BD37863570B52DED70
:10DFE000028B00F1280600F134058AB02946044668
:10DFF000304617F041FDB6EE008A20EE088A28462A
:10E00000B0EE480A17F0BCFC07A93046CDED080A6F
:10E010008DED091A8DED070A17F09CFC30468DED49
:10E02000010AB0EE480ACDED020A8DED031A17F091
:10E03000A7FC07A928468DED070ACDED080A8DED4E
:10E04000091A17F087FC04A901A88DED040ACDED8B
:10E05000050A8DED061A17F023FD324601A9204668
:10E060008DED070ACDED080A8DED091AFFF770FF57
:10E0700058B970F033F80121C4F878012046FFF751
:10E0800053FE0AB0BDEC028B70BD2A4604A920469F
:10E09000FFF75EFF0028ECD004F1400207A92046FC
:10E0A000FFF756FF0028E4D0EBE7000030B52DED78
:10E0B000028B0D4683B091F8F6110446284604F011
:10E0C00009FCC1B27C2000FB0151843104F128001D
:10E0D00015F082FB68468DED000ACDED010A17F0C0
:10E0E0009BF9DFED1C7AB4EEE70AF1EE10FA05D5E4
:10E0F0009FED190A03B0BDEC028B30BD684617F0E6
:10E1000009FA684617F062F90028F1D1284694ED23
:10E11000488A04F08BFCF0EE400AB0EE480A14F096
:10E1200071FF80B9284604F081FC84ED480AB0EE06
:10E13000408A9BF0D7FA84ED490AB0EE480A9BF07A
:10E1400027FC84ED4A0A04F59271684617F00CF931
:10E15000D0E700BF00000034000000009FED0C7A03
:10E16000B4EEC70AF1EE10FA0BD4DFED0A7AB4EE82
:10E17000E70AF1EE10FA07DCC0EE077AB0EE670AA4
:10E180007047F7EE007AF9E7F2EE047AF6E700BF9F
:10E19000F3665F3F58A00B4108B51C3017F03CF9FF
:10E1A000F1EE007AB4EEE70AF1EE10FA9DBFF1EE5F
:10E1B000027A37EEC00ADFED047A9FED040A98BFB9
:10E1C00020EE270A08BD00BFCDCC4C3ECDCCCC3DC7
:10E1D00008B5836993F9000038B10CF00BFFFDF727
:10E1E00043FC012894BF0020012008BDF8B52DEDA7
:10E1F000028B054604F0E4FD04F008FD0446B8B3C4
:10E20000FFF70AF990F8093393B32846FFF7E0FFC8
:10E21000064668B30CF0EEFE90F82031B02707FBFD
:10E22000030090ED217AF0EE087AB4EEE77AF1EE91
:10E2300010FA1DD495ED1E8A0CF0DCFE90F820310A
:10E24000DFED1E7A07FB030090ED220A98EE270A05
:10E2500014F05CFFDFED1A7AB0EEC00AB4EEE70A04
:10E26000F1EE10FA08DC6FF039FF3446C5F86801AA
:10E27000BDEC028B2046F8BD05F5B67017F07EFFA9
:10E28000B0EE408A0CF0B6FE90F820319FED0D7A8A
:10E2900007FB0303D3ED217A67EE877AB4EEE78AB2
:10E2A000F1EE10FADFD56FF019FFD5F86841001BC9
:10E2B000B0F5FA6F8CBF00240124D9E7E02E654247
:10E2C00000003442CDCC4C3F10B50A4B1B68DB6AD2
:10E2D00093F89C3004465BB96FF000FFD4F87C31B2
:10E2E000C01A44F61F6398428CBF0020012010BD65
:10E2F0000020FCE748270020F8B52DED068B0446EA
:10E300000CF078FE054604F05BFD064607F04CF97C
:10E31000002840F0AA802046FFF768FF002800F0A0
:10E32000A7803046FFF784FCD4F8E830984200F02C
:10E3300018813046FFF77CFCD4F8E830DFED8E7AA8
:10E34000C31A08EE903AF8EE688A304668EEA78A5B
:10E35000FFF76EFC94F8BC30C4F8E800F3B930461F
:10E3600004F062FCD0B104F1280796F8F621394692
:10E37000304604F05FFBD4ED1D0AB0EE401A38467B
:10E3800094ED1C0A15F098FB0023C4F89030C4F8F3
:10E390008C30C4F88830012384F8BC3020463146E4
:10E3A000FFF784FE95F8200105EB0015B0EE408ADA
:10E3B000AB6DC4F8EC3004F1B000D4ED129A17F054
:10E3C000DDFE6368DFED6D7A93ED007AB4EEE77AF7
:10E3D000F1EE10FA68EE299AB0EE40AA01D5C3ED2D
:10E3E000007A2046B0EE4A0AFFF7B8FE636820EED6
:10E3F000299A93ED000A29EE009AFFF7CDFE29EE47
